:020000040000FA
:10000000F090032041030000650300006703000037
:10001000690300006B0300006D0300006F03000024
:100020006F0300006F0300006F0300006F03000008
:100030006F0300006F0300000B3C0000BF3E000098
:10004000AF990000B9990000C3990000CD99000054
:10005000D7990000E1990000EB990000F5990000A4
:10006000FF990000099A0000139A00001D9A0000F1
:10007000279A0000319A00003B9A0000459A000040
:100080004F9A0000599A0000639A00006D9A000090
:10009000779A0000819A00008B9A0000959A0000E0
:1000A0009F9A0000A99A0000B39A0000BD9A000030
:1000B000C79A0000D19A0000DB9A0000E59A000080
:1000C000EF9A0000F99A0000039B00000D9B0000CE
:1000D000179B0000219B00002B9B0000359B00001C
:1000E0003F9B0000499B0000539B00005D9B00006C
:1000F000679B0000719B00007B9B0000859B0000BC
:100100008F9B0000999B0000A39B0000AD9B00000B
:10011000B79B0000C19B0000CB9B0000D59B00005B
:10012000DF9B0000E99B0000F39B0000FD9B0000AB
:10013000079C0000119C00001B9C0000259C0000F7
:100140002F9C0000399C0000439C00004D9C000047
:10015000579C0000619C00006B9C0000759C000097
:100160007F9C0000899C0000939C00009D9C0000E7
:10017000A79C0000B19C0000BB9C0000C59C000037
:10018000CF9C0000D99C0000E39C0000ED9C000087
:10019000F79C0000019D00000B9D0000159D0000D4
:1001A0001F9D0000319D00003B9D0000459D00000B
:1001B0004F9D0000599D0000639D00006D9D000053
:1001C000779D0000819D00008B9D0000959D0000A3
:1001D0009F9D0000A99D0000B39D0000BD9D0000F3
:1001E000C79D0000D19D0000DB9D0000E59D000043
:1001F000EF9D0000F99D0000039E00000D9E000091
:1002000000F002F800F074F80AA090E8000C8244B4
:100210008344AAF10107DA4501D100F069F8AFF291
:10022000090EBAE80F0013F0010F18BFFB1A43F0D4
:100230000103184754C2020074C202000A444FF07E
:10024000000C10F8013B13F0070408BF10F8014B35
:100250001D1108BF10F8015B641E05D010F8016B7A
:10026000641E01F8016BF9D113F0080F1EBF10F8DE
:10027000014BAD1C0C1B09D16D1E58BF01F801CB01
:10028000FAD505E014F8016B01F8016B6D1EF9D584
:100290009142D6D370470000002300240025002699
:1002A000103A28BF78C1FBD8520728BF30C148BFD9
:1002B0000B607047642929F08D87752929F08A879A
:1002C00073292AF0DC83002070471FB52AF0A2FCB6
:1002D0009DE803002AF014FB2AF0F6FA040000203F
:1002E00000212AF081FC401C60601FBD10B510BDCC
:1002F0002AF0F0FB1146FFF7E8FF29F08DFD2AF008
:100300000EFC03B4FFF7F2FF03BC2AF03FFC000031
:10031000EFF3108072B67047EFF310807047EFF381
:10032000108062B6704730BF704780F31188704705
:10033000EFF31180704700000138FDD170470000D5
:10034000DFF83C00016841F470010160BFF34F8F9A
:10035000DFF83000016821F040410160BFF36F8F8A
:1003600009480047FEE7FEE7FEE7FEE7FEE7FEE797
:10037000FEE7000005480649064A074B70470000A3
:1003800088ED00E034EF00E001020000F0500320AF
:10039000F0900320F0800320F080032010B5024687
:1003A000F64B1B68F64C2340F64CA34209D1F64BA2
:1003B0009A4202D101F11E0301E001F14003184607
:1003C00011E0EE4B1B68EE4C2340F04CA34209D1E8
:1003D000ED4B9A4202D101F11E0301E001F13E030F
:1003E000184600E0002010BD2DE9F04105460E46FC
:1003F000144631462846FFF7D1FF074621463846C6
:1004000001F05AFE384601F0B3FEBDE8F08170B548
:1004100004460D4629462046FFF7C0FF06463046F3
:1004200001F0E2FE304601F061FE70BD82680123FA
:100430008B409A438260704701228A40C260826882
:1004400001238B401A438260704730B5034632B1B6
:10045000DC684FF001158D4004EA05000FE05C6890
:1004600001258D4045F4803504EA050000F4803410
:100470002CB140F470204FF480348C40A04330BD48
:1004800001228A40C2607047026801238B401A43F0
:1004900002607047026801238B409A4302607047F4
:1004A00070B51446890045690F268E40B54304F0A7
:1004B0000F068E4035434561056A0F268E40B543D1
:1004C00003F003068E403543056204F00F02062A4E
:1004D0000CD3092A0AD8951FEA00C5693026964030
:1004E000B54304F0300696403543C56170BD70B524
:1004F0000C46650140352844920005680F26964059
:10050000B54303F00F0696403543056085690F2615
:100510009640B543C3F3032696403543856146684C
:100520000F25954026EA0505C3F30316964035438B
:100530004560C6690F25954026EA0505C3F30356B5
:1005400096403543C56103F4702575B141690F25A7
:100550009540A943C3F3024595402943416105698C
:10056000012696403543056104E005690126964061
:10057000B543056170BD0246106901238B401840E8
:10058000704701228A400261704702469069012348
:100590008B401840704701228A408261704710B535
:1005A00003464C0140342344002002E09C6810C202
:1005B000401CDC6804F480740CB90828F6D310BD24
:1005C00010B50A0C120401F00F040123A3401A43D2
:1005D000836A1A43826210BDF0B5034600245208B4
:1005E00001E0641C5208002AFBD1674DAB4201D1E7
:1005F000002000E0012000EB4006654F3E447454AB
:10060000F0BD70B5604DA84201D1002400E0012486
:100610004D014035284404EB44055D4E35446E5C85
:100620000425B5406A4304EB4405594E35446E5CDD
:10063000012505FA06F124E005680F269640B5432A
:1006400003F00F0696403543056085690F269640F6
:10065000B543C3F3032696403543856146680F25AD
:10066000954026EA0505C3F30316964035434560D9
:10067000012904D0466806259540AE434660121D08
:10068000491E0029D8D170BDF0B514463E4FB8427E
:1006900001D1002200E001224F014037384419E027
:1006A000002602EB4207DFF8E8C0674417F801C0F4
:1006B000012707FA0CF502E087683E446D1E002D05
:1006C000FAD102EB4207DFF8C8C067447F5C26FA24
:1006D00007F780C41F1EA3F10103E1D1F0BD002282
:1006E000490801E0521C49080029FBD10263704708
:1006F00000F5606343F82120704730B542EA0345B6
:1007000000F5646444F8215030BD70B50446002003
:100710002AB101F11005012606FA05F5284313B1A7
:1007200001258D402843C4F8000D70BD82684FF448
:1007300080338B409A438260704782684FF48033E5
:100740008B401A43826070470146486B7047416393
:10075000704782688A438260704782680A43826079
:100760007047024609B1D06805E0506800F4803354
:100770000BB140F470207047C160704700E00F403B
:100780000000FF70000005100080034000000A1008
:1007900000000020826B22F003020A43826370474C
:1007A0000146886B00F003007047416270470146C4
:1007B000486A704702684FF480738B401A430260A6
:1007C000704702684FF480738B409A430260704711
:1007D00001460868C0F30040704710B5C1F3031329
:1007E000C0F8C43F531E0C4663F31F14C0F8C84F33
:1007F00010BD0246084B186819B1C0F305135B1C05
:100800000B6020F47C70044B1B1F1B6803F00F036C
:1008100040EA031070470000C88F034070B50446DB
:10082000E10901208840C5430A20FFF785FD032028
:10083000D34908600A20FFF77FFDD248C0F8C052B4
:100840000A20FFF779FD0020CD4908600A20FFF754
:1008500073FD70BD10B50A20FFF76EFD0320C84977
:1008600008600A20FFF768FD0020C649C1F8C002F1
:100870000A20FFF761FD0020C14908600A20FFF748
:100880005BFD10BD00BFC048806900F0010000287A
:10089000F9D1704710B50220FFF74EFDFFF7F2FFC8
:1008A000B948C46904F00C0008B1022010BDB74873
:1008B00002F0BBF80220FFF73FFDFFF7E3FFB2486D
:1008C000C46904F00C0008B10220EFE70020EDE756
:1008D000AD4800680004800B7047AB480068C0F367
:1008E0000A40704710B58B09A74C6360C1F38303BE
:1008F000A36092080DE0A44B5B690360001D521ECB
:100900003AB1A14B9B6823B99F4B5B685B1C9E4C23
:100910006360002AEFD110BD2DE9F04107460E4675
:10092000144600BF9848856905F001000028F9D1F8
:10093000B00995494860C6F383008860A40838E090
:1009400093480068934908409349884206D19048EB
:10095000006880B210B93046FFF760FF8A493868F6
:1009600048610A20FFF7E8FC00BF8748856905F069
:1009700001000028F9D105F0100078B18448006822
:10098000844908408449884205D18148006880B282
:1009900008B9FFF75FFF2846BDE8F0813F1D641EE0
:1009A0003CB17948806820B977484068401C764956
:1009B0004860002CC4D176480068764908407649E2
:1009C000884205D17248006880B208B9FFF742FF3B
:1009D0006D488069E0E770B505460C466C480068D4
:1009E0006C4908406C49884206D16948006880B269
:1009F00010B92046FFF712FFA00963494860C4F30D
:100A00008300886008464561806970BD10B5604804
:100A10000068604908406049884205D15C48006828
:100A200080B208B9FFF716FF5C485749803108606B
:100A3000FFF728FF554801F0F8FF0220FFF77CFC84
:100A4000FFF720FF5048806910BD01464E484160C5
:100A5000006B704702464C484260016300BF4A4841
:100A6000806900F001000028F9D14748806970478B
:100A700010B5034644484360434C34340BE00868E7
:100A80002060091D241D521E00BF3F48806900F0F0
:100A900001000028F9D1002AF1D13B48806910BD3E
:100AA0000146394841604FF0FF30374A1062104626
:100AB000006A704710B50346334843604FF0FF307B
:100AC000314C2062501E01EB800104E051F8040912
:100AD0002D4C2062521E002AF8D12B48006A10BD0E
:100AE00001218140284A116570472749096C41F06E
:100AF0000101254A11642249FC39096941F00401C8
:100B00001F4AFC3A116170471D49FC39096921F0FF
:100B100004011B4AFC3A11611B49096C21F00101D7
:100B2000194A11647047014649B11548FC384069BB
:100B300000F0040008B1042070470020FCE71248D0
:100B4000806900F0010008B10020F5E70420F3E718
:100B500010B5044604200A49FC3948610C48006875
:100B60000C4908400C49884205D10948006880B208
:100B700008B9FFF76FFE10BD034880697047000099
:100B8000FCD00F4000E00A4000F00A40005800F09E
:100B900000E00F400000FF700000051001007BE343
:100BA000F0B50446DDE9055700BFDFF8B0C4DCF856
:100BB00000C00CF0010CBCF1000FF6D142EA870C2A
:100BC0004CF08000202D01D8202B03D940F08070FC
:100BD000ED08DB08AB4202D140EA052007E04FF404
:100BE000000C4CEA052C4CEA434C4CEA0000C4F8DB
:100BF000000CDFF86CC4DCF8146000200DE0DFF8B6
:100C000060C45CF830C08C4506D3DFF854C40CEBEC
:100C1000C00CDCF8046002E0401C0328EFD300BFE6
:100C2000D4F810C02CF03C0C4CEA060CC4F810C0F0
:100C30004FF0FF3CC4F80CC1C4F810C1F0BDD0F8AF
:100C4000001C41F00101C0F8001C00BFD0F8001CDE
:100C500001F001010029F9D1704770B505460C4635
:100C6000C5F8C44F04F0404060B9FE4801F0DDFE15
:100C700000BFFC4801F091FE0028FAD042F210704B
:100C8000FFF75AFB04F04040B0F1404F06D1F64860
:100C9000006840F48030F449086005E0F2480068DC
:100CA00020F48030F0490860F048FFF7C8FF4FF4A7
:100CB0007A70FFF741FB70BD30B50468EC4D2C40F5
:100CC0000C4344F40044046023B143F48034C0F87E
:100CD000DC4005E0D0F8DC4024F48034C0F8DC408F
:100CE000C0F8182C30BD70B5D0F8185C15600568D8
:100CF000E04E35400D60D0F8DC4004F480351DB185
:100D0000C4F30D051D600AE0056805F480151DB1EA
:100D10004FF420551D6002E04FF400651D6070BD6A
:100D200010B5CB004033C3586FF30F03147923433E
:100D3000547943EA0424CB004033C45013785478E8
:100D400043EA0423947843EA0443D47843EA0464EE
:100D5000CB004433C45010BD10B50346CC0044341E
:100D600018591070040A5470040C9470040ED47056
:100D7000CC00403418591071040A547110BD01465A
:100D80000420704730B5CC0040340459A4B2144359
:100D9000CD0040354451CC0044340359CC00443498
:100DA000035130BD0246C8004030105800F07F406B
:100DB00070474268B04B1A400A4342607047014690
:100DC0004868AD4AD24310407047C26081607047A6
:100DD000C368136083680B6070472DE9F0410646D5
:100DE00006223146D01F01F0E0FC0446E443002512
:100DF000002705E06D0004F00100054364087F1C36
:100E0000062FF7D32846BDE8F081C0F8241C7047B0
:100E10000146486A70470021C0F8041C7047002151
:100E2000C0F8081C7047C0F80C1C70470146D1F888
:100E30000C0C70470146D1F84C0C70470146D1F8B4
:100E4000540C7047C0F8101C70470146D1F8100CC4
:100E500070470146D1F8480C70470146D1F8500C54
:100E600070470146D1F8140C844A10407047416A1B
:100E700001F0807161B1D0F8181C41F48011C0F804
:100E8000181C00BFD0F8181C01F480110029F9D1FA
:100E90007047D0F8181C41F40051C0F8181C0168C4
:100EA00041F0080101607047016821F0080101600C
:100EB000D0F8181C21F40051C0F8181C7047D0F865
:100EC000181C41F00201C0F8181C016841F004012F
:100ED00001607047016821F004010160D0F8181C1E
:100EE00021F00201C0F8181C704770B505460C4689
:100EF0002146382001F0E0F8382001F039F970BDC2
:100F000010B50446382001F06FF9382001F0EEF8F2
:100F100010BD44F245020A400AB141F4803142F268
:100F2000BA720A400AB141F4004121F0004232B1E4
:100F3000D0F81C2C21F000431A43C0F81C2C01F0FF
:100F400000422AB1D0F8D42F42F00102C0F8D42FC9
:100F500070470246D2F81C0C21F00043984344F23B
:100F6000450303400BB920F4803042F2BA730340CA
:100F70000BB920F40040C2F81C0C01F000432BB167
:100F8000D2F8D43F23F00103C2F8D43F704710B524
:100F90000246D2F8140C3A4C204021B1D2F81C4C35
:100FA00044F0F044204011B1D2F8D83F01E0D2F82B
:100FB000D03F03F001040CB140F0004010BD44F2FA
:100FC00045020A400AB141F4803142F2BA720A4045
:100FD0000AB141F4004121F000421AB121F000426F
:100FE000C0F8142C01F000422AB1D0F8D82F42F0FA
:100FF0000102C0F8D82F704710B500BF046904F093
:101000000104002CFAD14361046904F03C0444EA71
:10101000821444EAC124E41C046100BF046904F0A2
:101020000104002CFAD110BD034600BF186900F07E
:1010300001000028FAD1186900F03C0040EA821053
:1010400040EAC120401C186100BF186900F001008F
:101050000028FAD1586980B27047000000CC0E40D9
:1010600020AC0200003000F0C8CF0E4000C00E409F
:101070000C81A085FF7E5F7A00F8FE7F0020FE03D2
:10108000FFFF01FC70B506460D4614461F230D22D6
:101090002946FE48FFF7B0FF23460E222946FB48AB
:1010A000FFF7AAFF44F21F030D222946F748FFF776
:1010B000A3FF0E222946F548FFF7B6FF70BDF0B535
:1010C00007460D4614461E461F230D222946EF48AB
:1010D000FFF792FF23460E222946EC48FFF78CFFCC
:1010E00044F21F030D222946E848FFF785FF3346E7
:1010F0000E222946E548FFF77FFFF0BD70B5044694
:101100000D46002229462046FFF78EFF20F480502E
:1011100040F400663346002229462046FFF76CFF64
:1011200070BD70B504460D46002229462046FFF7E3
:101130007BFF20F4006040F48056334600222946AD
:101140002046FFF759FF70BDD0F8C83F43F4802315
:10115000C0F8C83FD3B2C0F80437C0F800177047D2
:101160000246D2F80407C0B20860D2F80007704700
:10117000D0F8001741F00101C0F80017D0F80017AF
:1011800001F0040129B9D0F8001741F00401C0F8BA
:1011900000177047D0F8001721F00101C0F80017C0
:1011A0007047C0F81017C0F8142700BFD0F80037F8
:1011B00003F00403002BF9D1D0F8003743F0040307
:1011C000C0F80037704710B500BFD0F808370B6083
:1011D000D0F80C3713601368D0F80C47A342F4D84A
:1011E00010BD10B5C0F810170BB1002401E04FF08E
:1011F00000441443C0F8144700BFD0F8004704F07F
:101200000804002CF9D1D0F8004744F00804C0F8D5
:10121000004710BDC0F8181700BFD0F8002702F033
:101220002002002AF9D1D0F8002742F02002C0F8AD
:101230000027704700BFD0F8203703F00043002B91
:10124000F9D1C0F81C17C0F820277047D0F8001754
:1012500041F01001C0F800177047D0F8001721F0D6
:101260001001C0F8001770470146D1F828077047F1
:10127000D0F80037C3F3402209B102B9491EC0F8C3
:101280002C17704700BFD0F82C2702F00F02002A5D
:10129000F9D141F01002C0F82C27704700BFD0F8F8
:1012A0002C2702F00F02002AF9D141F01002C0F8F9
:1012B0002C277047C0F86017C0F86427704742EACF
:1012C0000103C36170470246D3690B80180C000408
:1012D000704742EA0103C0F8843570470246D2F8ED
:1012E00084350B80180C00047047F1B50222694662
:1012F000D01E01F05AFA0446E4430025002605E01A
:101300006D0004F0010005436408761C042EF7D339
:101310002846F8BDC0F8881570470146D1F8880501
:10132000704710B50A46C46A44F00044C4621346CC
:10133000002103E053F821408462491C0829F9D3B5
:1013400010BD10B50A46C46A44F00044C462134696
:10135000002103E0846A43F82140491C0829F9D39D
:1013600010BD0A46C16A40F2072399431143C16286
:1013700070470146C86A40F2072210407047014694
:10138000C86A00F06100704700BFD0F8141C012942
:10139000FBD0016821F008010160D0F8181C21F48D
:1013A0000051C0F8181C00BF416A01F440710029C7
:1013B000FAD0D0F8181C21F00201C0F8181C7047B0
:1013C00030B5334D05EA02449DB22C43446321B14C
:1013D000056B45F40025056301E00025056330BD7C
:1013E000016B41F48031016370470146086B80B2A4
:1013F0007047016B41F4003101637047016B21F4C8
:10140000003101637047F0B505460E4614461F468D
:10141000230B0D2231462846FFF7EEFDC4F30B03E4
:101420000E2231462846FFF7E7FD4FF4804040EAA0
:1014300014330D2231462846FFF7DEFD3B460D22D0
:1014400031462846FFF7D8FDF0BD70B505460E467B
:101450001446230B0D2231462846FFF7CDFDC4F379
:101460000B030E2231462846FFF7C6FD4FF480409D
:1014700040EA14330D2231462846FFF7BDFD0E2207
:1014800031462846FFF7D0FD70BD000000C00E4079
:101490000000FF0330B50246F74B1824F7480068F8
:1014A000F74D2840F74DA84201D1F74B1B240021EE
:1014B00008E053F83100904203D103EBC1004068CB
:1014C00030BD491CA142F4D30020F9E702F001032A
:1014D0001BB1D0F800340B4302E0D0F800348B434A
:1014E000C0F8003402F002031BB1D0F820340B43E3
:1014F00002E0D0F820348B43C0F82034704730B578
:10150000024601208840C1B2D2F80034D2F820440B
:1015100003EA010008B1012000E0002004EA01050F
:101520000DB1022500E00025284330BD02F0010383
:101530001BB1D0F808340B4302E0D0F808348B43D9
:10154000C0F8083402F002031BB1D0F804340B4396
:1015500002E0D0F804348B43C0F8043402F00403F2
:101560001BB1D0F80C340B4302E0D0F80C348B43A1
:10157000C0F80C3402F4803323B1D0F8383543F08E
:10158000010303E0D0F8383523F00103C0F8383503
:101590007047F0B5024601208840C1B2D2F8083445
:1015A000D2F80444D2F80C64D2F8385503EA0100AA
:1015B00008B1012000E0002004EA01070FB1022772
:1015C00000E00027384306EA01070FB1042700E0D6
:1015D0000027384305F0010717B14FF4803700E0CA
:1015E00000273843F0BDF0B5A44D2D68A44E35401A
:1015F000A64EB5421AD0002416E00125A5400D40A4
:1016000085B1D0F8C45F67000326BE40B543C0F87B
:10161000C45FD0F8C45F6700C2F34116BE403543D3
:10162000C0F8C45F651CECB2082CE6DB02F00105D3
:101630001DB1D0F800550D4302E0D0F800558D43A0
:10164000C0F8005502F002051DB1D0F804550D4355
:1016500002E0D0F804558D43C0F8045502F00405AB
:101660001DB1D0F808550D4302E0D0F808558D4360
:10167000C0F8085502F008051DB1D0F818550D4303
:1016800002E0D0F818558D43C0F818557B4D2D68F1
:101690007B4E35407D4EB5420BD002F010051DB19A
:1016A000D0F83C550D4302E0D0F83C558D43C0F8CE
:1016B0003C5503F001051DB1D0F80C550D4302E077
:1016C000D0F80C558D43C0F80C5503F002051DB140
:1016D000D0F810550D4302E0D0F810558D43C0F8F6
:1016E000105503F004051DB1D0F814550D4302E068
:1016F000D0F814558D43C0F8145503F008051DB1FA
:10170000D0F81C550D4302E0D0F81C558D43C0F8AD
:101710001C555A4D2D685A4E35405C4EB54217D077
:1017200003F400751DB1D0F844550D4302E0D0F824
:1017300044558D43C0F8445503F440751DB1D0F8AD
:1017400040550D4302E0D0F840558D43C0F8405558
:101750001BB9D0F828550D4302E0D0F828558D4329
:10176000C0F82855F0BDF0B514461D4601268E4040
:10177000F1B2D0F800650E400EB1012600E000265F
:101780003246D0F804650E400EB1022600E0002675
:101790003243D0F808650E400EB1042600E0002662
:1017A0003243D0F818650E400EB1082600E000263E
:1017B0003243324E3668324F3E40344FBE420FD035
:1017C000D0F83C650E400EB1102600E000263243F2
:1017D000D0F8C46F4F00FE4006F0030642EA4612FE
:1017E0002260D0F80C650E400EB1012600E0002604
:1017F0003346D0F810650E400EB1022600E00026F8
:101800003343D0F814650E400EB1042600E00026E4
:101810003343D0F81C650E400EB1082600E00026C8
:101820003343164E3668164F3E40184FBE420CD01A
:10183000D0F840650E4046B1D0F844650E400EB178
:10184000FE1401E04FF4807633432B60F0BDD0F8F6
:1018500010240A43C0F810247047D0F810248A439B
:10186000C0F810247047024611B1D2F8180470472E
:10187000D2F81404FBE7000038AC020000E00F408F
:101880000000FF7000000A10F8AC02000000051014
:10189000C0F81C14704770B504460D462046FFF78B
:1018A000F9FD06462946304600F006FC304600F0B9
:1018B0005FFC70BD70B504462046FFF7EBFD0546A2
:1018C000284600F091FC284600F010FC70BD2DE980
:1018D000F04107460C4615463846FFF7DBFD064645
:1018E0003019294600F0E8FB301900F041FCBDE852
:1018F000F08170B506460C463046FFF7CBFD054635
:10190000281900F071FC281900F0F0FB70BD0246A8
:10191000002000EB810010587047002303EB810387
:10192000C250704730B504460D4600222946204675
:10193000FFF7CCFD0023012229462046FFF753FE86
:1019400030BD30B504460D46022229462046FFF739
:10195000BDFD0823662229462046FFF744FE30BD20
:1019600030B504460D46002229462046FFF7AEFD5D
:101970000023012229462046FFF735FE30BD30B551
:1019800004460D46022229462046FFF79FFD082304
:10199000012229462046FFF726FE30BD30B5044619
:1019A0000D46022229462046FFF790FD082301221A
:1019B00029462046FFF717FE30BD30B504460D46D8
:1019C000022229462046FFF781FD08236622294688
:1019D0002046FFF708FE30BD30B504460D46022212
:1019E00029462046FFF772FD082366222946204635
:1019F000FFF7F9FD30BD30B504460D4602222946F9
:101A00002046FFF763FD0823662229462046FFF79C
:101A1000EAFD30BD30B504460D4600222946204679
:101A2000FFF754FD0823012229462046FFF7DBFD7E
:101A300030BD30B504460D46082301222946204614
:101A4000FFF7D1FD012229462046FFF73FFD30BDBB
:101A500030B504460D460923012229462046FFF7EA
:101A6000C2FD012229462046FFF730FD30BD30B5CA
:101A700004460D46022229462046FFF727FD08238B
:101A8000012229462046FFF7AEFD30BD30B50446A1
:101A90000D46022229462046FFF718FD09230122A0
:101AA00029462046FFF79FFD30BD30B504460D4660
:101AB000022229462046FFF709FD08230122294674
:101AC0002046FFF790FD30BD30B504460D4602229A
:101AD00029462046FFF7FAFC0823662229462046BD
:101AE000FFF781FD30BD30B504460D460222294680
:101AF0002046FFF7EBFC0823012229462046FFF78A
:101B000072FD30BD30B504460D46022229462046FE
:101B1000FFF7DCFC0823012229462046FFF763FD7E
:101B200030BD30B504460D46022229462046FFF757
:101B3000CDFC0A23012229462046FFF754FD30BD83
:101B400030B504460D46022229462046FFF7BEFC6A
:101B50000823012229462046FFF745FD30BD30B558
:101B600004460D46022229462046FFF7AFFC082313
:101B7000012229462046FFF736FD30BD30B5044628
:101B80000D46022229462046FFF7A0FC0823012229
:101B900029462046FFF727FD30BD30B504460D46E7
:101BA000022229462046FFF791FC082301222946FC
:101BB0002046FFF718FD30BD30B504460D46002223
:101BC00029462046FFF782FC0023012229462046B1
:101BD000FFF709FD30BD30B504460D460222294607
:101BE0002046FFF773FC0823012229462046FFF711
:101BF000FAFC30BD30B504460D4600222946204689
:101C0000FFF764FC4FF40273012229462046FFF7D8
:101C1000EAFC30BD30B504460D4600222946204678
:101C2000FFF754FC4FF48473012229462046FFF746
:101C3000DAFC30BD0146D1F84805704710B50146C1
:101C4000C1F307401F4BDB6E01248440234033B1B6
:101C5000012303EB40031C4C54F8230003E0430032
:101C6000194C54F82300C1F30722D0F82C350F2467
:101C70009440A34301F00F0494402343C0F82C3553
:101C800010BDD0F834250A43C0F834257047D0F889
:101C900034258A43C0F834257047D0F830250A43EC
:101CA000C0F830257047D0F830258A43C0F8302579
:101CB0007047064AC0F82025D0F824250A43C0F80A
:101CC0002425704700E00F40D0AD02004B434F4C3D
:101CD00030B50246E64B0624E6480068E64D28404B
:101CE000E64DA84201D1E64B0A24002108E053F852
:101CF0003100904203D103EBC100406830BD491C64
:101D0000A142F4DB0020F9E7016A41F01001016211
:101D1000704770B503460C4616461846FFF7F4FFA9
:101D2000012E01D1D74A00E0D74A142000FB02401F
:101D3000401E02EB82018900B0FBF1F0451EDD6020
:101D4000D3F8C00F00F0010048B1D0482044401E35
:101D5000CE49B0FBF1F0451E45F08000D86070BD63
:101D6000016A41F0200101620121C0F804187047A6
:101D700000B502460B461046FFF7F2FFC2F80038E6
:101D800000BD11B1012908D102E0C0F8002804E02B
:101D900042F08003C0F81C3800BF00BF7047016AE2
:101DA00021F01001016270470021C0F80418016A97
:101DB00021F020010162704770B504460D462046AF
:101DC000FFF786FF06462946304600F075F9304693
:101DD00000F0CEF970BD70B504462046FFF778FFDD
:101DE0000546284600F000FA284600F07FF970BD4D
:101DF00001210161704702690A4302617047D0F80E
:101E00000C1841F00101C0F80C187047D0F80C28EC
:101E10000A43C0F80C28704700210161704702692D
:101E20008A4302617047D0F80C1821F00101C0F814
:101E30000C187047D0F80C288A43C0F80C2870475B
:101E4000024629B1906908B1012070470020FCE7E3
:101E5000506908B10120F8E70020F6E7024609B111
:101E6000906970475069FCE7024631B1D2F8140816
:101E700008B1012070470020FCE7D2F8100808B133
:101E80000120F7E70020F5E7024611B1D2F8140867
:101E90007047D2F81008FBE70121C16181617047EA
:101EA000C16170470121C0F818187047C0F81818B0
:101EB000704742EA4103036070470146C86A7047B1
:101EC0000146486800F0010008B101207047002079
:101ED000FCE70146486800F0400008B10120704767
:101EE0000020FCE7416070470246516801F00100A4
:101EF00008B10020704701F0120010B101F01C0081
:101F0000F8E70020F6E7816070470146886870476F
:101F10004162704731B1D0F8202842F00102C0F888
:101F2000202805E0D0F8202822F00102C0F820285F
:101F3000704731B1D0F8202822F00202C0F82028E2
:101F400005E0D0F8202842F00202C0F820287047AF
:101F50000146D1F804087047C0F8081870470146D8
:101F6000D1F808087047D0F8042F6FF30F02C0F8BB
:101F7000042FD0F8042F0A43C0F8042F7047D0F87C
:101F8000041F41F48041C0F8041F7047D0F8042FAB
:101F900092B2C0F8042FD0F8042F0A43C0F8042FDF
:101FA0007047D0F8041F41F08041C0F8041F70470B
:101FB0000146D1F8080F704700BFD0F8082F02F093
:101FC0000202002AF9D1C0F8001F70470246D2F879
:101FD000080F00F0020008B100207047C2F8001F8F
:101FE0000120FAE7014600BFD1F8080F00F4803065
:101FF0000028F9D1D1F8000F70470246D2F8080F37
:1020000000F4803008B100207047D2F8000F08704B
:102010000120F9E7016370470146486B7047154A94
:102020001268154B1A40154B9A4202D1C2680A43F6
:10203000C260104A1268104B1A40154B9A4207D1E1
:10204000826B42EA11328263026A42F0400202620B
:10205000704741F00102C0F8042870470121C0F820
:1020600004187047016A41F00101016270470000E5
:1020700060AE020000E00F400000FF7000000A1098
:1020800090AE0200801A0600A0860100804737014A
:102090000000051000BFFEE710B5FEF740F908B1DB
:1020A000012010BD0020FCE710B5FEF731F908B1A2
:1020B000012010BD0020FCE730B50246B64C246874
:1020C000B64DAC420ED0B44C2368002005E053F866
:1020D0002040B24D45F82040401C9B28F7D3AF4C20
:1020E000AD4D2C60AD4C44F8221030BDAC49AB4A2C
:1020F00042F820107047AB4951F82010AA4A11430A
:10210000A54A121D11607047A34A121D126802F4FD
:10211000E061002006E0A34A52F820208A4200D164
:1021200002E0401C0828F6D300BF704710B50A46ED
:1021300083089E4C54F8233019688307DC0EFF2374
:10214000A34099438307DB0E02FA03F31943830884
:10215000964C54F82330196010BD01468808934A04
:1021600052F8200000688A07D20ED040C0B27047F3
:10217000042808D188491C31096841F48031864A15
:102180001C3211602FE0052808D183491C310968F1
:1021900041F40031804A1C32116024E0062808D145
:1021A0007D491C31096841F480217B4A1C32116051
:1021B00019E00F2808D14FF0E021096941F0020130
:1021C0004FF0E02211610EE010280CD3A0F11001B5
:1021D00001F01F0201219140A0F110025209744B3D
:1021E00053F8222011607047042808D16A491C3135
:1021F000096821F48031684A1C3211602FE00528FB
:1022000008D165491C31096821F40031624A1C3249
:10221000116024E0062808D15F491C31096821F4C7
:1022200080215D4A1C32116019E00F2808D14FF05F
:10223000E021096921F002014FF0E02211610EE076
:1022400010280CD3A0F1100101F01F0201219140D0
:10225000A0F110025209574B53F822201160704729
:1022600010B501460020042905D14B4A1C321268E2
:1022700002F4803028E0052905D1474A1C32126853
:1022800002F4003020E0062905D1434A1C321268CE
:1022900002F4802018E00F2905D14FF0E0221269E6
:1022A00002F0020010E010290ED3A1F11002520931
:1022B0003F4B53F822201268A1F1100303F01F04D2
:1022C0000123A34002EA030010BD022808D13249CD
:1022D000091F096841F000412F4A121F116024E0D4
:1022E0000E2808D12C49091F096841F080512A4A5B
:1022F000121F116019E00F2808D12749091F09682A
:1023000041F08061244A121F11600EE010280CD3A6
:10231000A0F1100101F01F0201219140A0F1100273
:102320005209254B53F82220116070470E2808D11E
:102330001949091F096841F00061174A121F11600D
:1023400019E00F2808D11449091F096841F00071EC
:10235000114A121F11600EE010280CD3A0F11001D9
:1023600001F01F0201219140A0F110025209134B0C
:1023700053F822201160704710B504462046FDF73F
:10238000D4FF10BD10B5FDF7D3FF10BDA0F11001B3
:102390000B4A11607047000008ED00E000080020C3
:1023A00095200000E0AE02000000FA0500AF020038
:1023B0009CAF0200B0AF0200C4AF0200D8AF020071
:1023C00000EF00E030B50246744B04247448006806
:1023D000744D2840744DA84201D1744B00BF0021B8
:1023E00008E053F83100904203D103EBC10040688C
:1023F00030BD491CA142F4D30020F9E72DE9F04F8C
:102400000C461D46DDE909C815B94FF0000A01E088
:102410004FF0040A57464760B4FBFCF6002100BFAA
:10242000891CB6FBF1FAAAF10103FF2BF8D8016170
:102430004FEA827A4FEA1A6902F0300249EA032A27
:102440004AEA020AA8F1010B4AEA0B070760BDE855
:10245000F08F416841F0020141607047416821F00E
:1024600002014160704770B504460D462046FFF7F3
:10247000A9FF064629463046FFF71EFE3046FFF705
:1024800077FE70BD70B504462046FFF79BFF0546FA
:102490002846FFF7A9FE2846FFF728FE70BD4269CF
:1024A0000A434261704742698A434261704702466B
:1024B00009B1D06970479069FCE70162704700BFBD
:1024C000C26802F00202002AFAD081607047024618
:1024D000D06800F0020010B1916001207047002028
:1024E000FCE700BFC26802F00402002AFAD082684A
:1024F0000A6070470246D06800F0040018B1906886
:102500000860012070470020FCE7426A0A434262EB
:102510007047426A8A43426270470146C868C0F306
:1025200000107047C0F8C81F70470146D1F8C80FA7
:102530007047426822F4E0720A434260704700BF6D
:10254000C26802F00202002AFAD0426842F4006235
:102550004260816070470246D06800F0020030B1EE
:10256000506840F400605060916001207047002086
:10257000FCE7416841F4806141607047416821F4A3
:10258000806141607047416841F0010141607047DE
:10259000416821F00101416070470000ECAF02008A
:1025A00000E00F400000FF7000000A100CB00200B5
:1025B00030B501F001042CB10C784440AE4D285DDB
:1025C000491C521E01F0020464B1012A0AD90B8889
:1025D00080EA0304E4B2A84D285D80EA1324285D54
:1025E000891C921E12E00B6880EA0304E4B2A24D3B
:1025F000285D80EA1324E4B2285D80EA1344E4B243
:10260000285D80EA1364285D091D121F032AEAD899
:10261000012A0AD90B8880EA0304E4B2964D285DAA
:1026200080EA1324285D891C921E1AB10C7844405C
:10263000914D285D30BD30B501F001044CB10C78EE
:102640004440E4B28D4D35F8144084EA2020491C02
:10265000521E01F002049CB1012A11D90B8880EAB4
:102660000304E4B2854D35F8144084EA202080EA62
:102670001324E4B235F8144084EA2020891C921E09
:102680001FE00B6880EA0304E4B27C4D35F8144087
:1026900084EA202080EA1324E4B235F8144084EA66
:1026A000202080EA1344E4B235F8144084EA202064
:1026B00080EA1364E4B235F8144084EA2020091D4E
:1026C000121F032ADDD8012A11D90B8880EA0304DE
:1026D000E4B26A4D35F8144084EA202080EA1324DD
:1026E000E4B235F8144084EA2020891C921E3AB1E5
:1026F0000C784440E4B2614D35F8144084EA20205F
:1027000030BD30B504460D46A20029460020FFF733
:1027100092FF30BDF0B506460D461446002000225B
:1027200000233AE002CD80EA0107FFB2DFF84CC196
:102730003CF8177087EA202080EA1127FFB23CF8A6
:10274000177087EA202080EA1147FFB23CF8177023
:1027500087EA202080EA1167FFB23CF8177087EA09
:10276000202083EA0107FFB23CF8177087EA232391
:1027700083EA1147FFB23CF8177087EA232382EA05
:102780001127FFB23CF8177087EA222282EA11670C
:10279000FFB23CF8177087EA2222371EA6F1010625
:1027A000C0D120806380A280F0BD30B501F001046B
:1027B0004CB1C4B20D786C40314D55F8244084EAD8
:1027C0001020491C521E01F002049CB1012A11D9AB
:1027D0000B8880EA0304E4B2294D55F8244084EACA
:1027E000102080EA1324E4B255F8244084EA102033
:1027F000891C921E1FE00B6880EA0304E4B2204D9E
:1028000055F8244084EA102080EA1324E4B255F8F5
:10281000244084EA102080EA1344E4B255F82440AE
:1028200084EA1020C4B284EA136455F8244084EA90
:102830001020091D121F032ADDD8012A11D90B8887
:1028400080EA0304E4B20E4D55F8244084EA1020D7
:1028500080EA1324E4B255F8244084EA1020891C4D
:10286000921E3AB1C4B20D786C40054D55F8244023
:1028700084EA102030BD00002CB002002CB1020010
:102880002CB30200024600210AE0F74850F831005C
:10289000904204D3F44800EBC10040687047491CE3
:1028A0000629F2D30020F9E7F0B50146DFF8BCC3F2
:1028B000DCF860C1CCF38923DFF8B0C3DCF860C179
:1028C000CCF30905DFF8A4C3DCF864C1CCF3042C15
:1028D0000CF10106DFF894C3DCF864C10CF01F0CA6
:1028E0000CF10107B1FBF7F15A09A3EB421401FB0C
:1028F00005F001FB02FC00EB5C1001FB04FC00EBAB
:102900009C20B0FBF6F0F0BDD8483C380068401C75
:1029100000027047D5480068D5490840D54988422B
:1029200006D1D24880680004400900F50060704775
:10293000CE484038006880B2401CC002F7E7CB4860
:102940000068CB490840CC49884209D1C748403883
:102950000068C0F302400A30012101FA00F070471C
:102960004FF48060FBE70146C1F30720C34A1044DF
:1029700000F0704040F00070C1F30722BF4B1A44D2
:10298000C2F3130240EA4210CAB240EA8200006871
:1029900008B1012070470020FCE70146C1F3072081
:1029A000B74A104400F0704040F00070C1F30722B5
:1029B000B34B1A44C2F3130240EA4210CAB240EACF
:1029C0008200006808B1012070470020FCE710B5C4
:1029D0000121C0F30722AB4B1A4402F0704242F0CF
:1029E0000072C0F30723A74C2344C3F3130342EA46
:1029F0004312C3B242EA8302116010BD10B5002138
:102A0000C0F307229F4B1A4402F0704242F000725A
:102A1000C0F307239B4C2344C3F3130342EA43123E
:102A2000C3B242EA8302116010BD18B50121C0F3A0
:102A30000722954B1A4402F0704242F00072C0F334
:102A40000723914C2344C3F3130342EA4312C3B256
:102A500042EA830211600021009102E00099491CC2
:102A6000009100991029F9D30021C0F30722864B69
:102A70001A4402F0704242F00072C0F30723824C05
:102A80002344C3F3130342EA4312C3B242EA83026C
:102A9000116018BD10B50121C0F307227B4B1A4409
:102AA00002F0704242F00072C0F30723774C2344D7
:102AB000C3F3130342EA4312C3B242EA8302116032
:102AC00010BD10B50021C0F30722704B1A4402F06C
:102AD000704242F00072C0F307236C4C2344C3F3EE
:102AE000130342EA4312C3B242EA8302116010BDEB
:102AF00010B50121C0F30722654B1A4402F0704261
:102B000042F00072C0F30723614C2344C3F3130364
:102B100042EA4312C3B242EA8302116010BD10B50B
:102B20000021C0F307225A4B1A4402F0704242F0CF
:102B30000072C0F30723564C2344C3F3130342EA45
:102B40004312C3B242EA8302116010BD10B50121E5
:102B5000C0F307224F4B1A4402F0704242F0007259
:102B6000C0F307234B4C2344C3F3130342EA43123D
:102B7000C3B242EA8302116010BD10B50021C0F358
:102B80000722444B1A4402F0704242F00072C0F334
:102B90000723404C2344C3F3130342EA4312C3B256
:102BA00042EA8302116010BD30490968304A114081
:102BB000304A91420ED130B12C49096E41F000618A
:102BC0002A4A116618E02949096E21F00061274A56
:102BD000116611E040B12549B031096841F000515A
:102BE000224AC2F8B01007E02049B031096821F04C
:102BF00000511E4AC2F8B010704710B50446214675
:102C00002C20FFF759FA2C20FFF7B2FA10BD10B5AF
:102C10002C20FFF7E9FA2C20FFF768FA10BD1349C2
:102C2000496D0143114A516570471049496D81430F
:102C30000E4A516570470D4988657047014611B1CC
:102C40000A48806D70470948006DFBE7124908602B
:102C500070471148006870470F4908310860704795
:102C60000D4808300068704748B9020000E00F4086
:102C70000000FF700000051000000A1000E30F4084
:102C800000EA0F4000E90F4000E50F4000E60F406A
:102C900000E70F4000E80F40B4E10F40FE49086034
:102CA0007047FD49091D08607047FC48FC490860F1
:102CB00000BFFEE710B5FDF736FB10BD10B5F848B4
:102CC000001D006840F00400F549091D0860FDF78B
:102CD0002AFBF348001D006820F00400F049091D9C
:102CE000086010BDEF48C06D7047EE49C96D814363
:102CF000EC4AD1657047EB49C86770470146EA481E
:102D0000084050B101F00040E34A383A1060E6480C
:102D100081380840E34AC2F85001DF483838016082
:102D200001F4007088B100BFDB483438006800F45B
:102D300040700028F8D0D8483438006800F440705B
:102D4000B0F5807F01D0002070470120FCE7D24918
:102D5000503108607047D0485030006870472DE906
:102D6000FE4F05468A46CF480068D0490840D04902
:102D7000884202D10020BDE8FE8FC5F3841705F01C
:102D80003800102805D1DFF82C93002600BF152746
:102D900048E005F03800302804D147F230594FF4AC
:102DA00000163FE005F03800382804D14FF4004900
:102DB0004FF4800636E005F0380078BB1A2F01DCAE
:102DC000092F01DA0020D6E7BB4850F827904FF4CE
:102DD000401646F04076B348C06F20F01C000190CA
:102DE000072F03DB019840F010000190AD490198D6
:102DF000C8674FF40020009005E00098401E009046
:102E0000009800B905E0A748006D00F48070002824
:102E1000F3D000BF009828B90020ACE7FFE74FF0DF
:102E20000009002605F46050002874D105F0380030
:102E300028B105F03800102801D000209BE7C5F329
:102E4000026002909D48FFF71DFD9649C031086061
:102E50009448D0F8B0009A4900EA010444F00044D4
:102E60009048B0300460093F9649029851F820001C
:102E70005044401EB0FBFAF88A48D0F8B000304306
:102E80008849B0310860029800EBC00000EB4000B8
:102E90008D4901EBC00007EB470100EB8100406862
:102EA0008049C1F864017C4824380168A8F1010018
:102EB00041EA00207B49C1F86401029800EBC000A0
:102EC00000EB4000804901EBC00007EB470150F8E0
:102ED000210071492839096801F4000108436E494D
:102EE000283908604846FFF7DFFC4FEA500A504691
:102EF000FFF7C8FC6B49C1F8C0000846D0F8600174
:102F000000F4000040B16748B030006840F08040F5
:102F1000C1F8B00008E02BE05F482838006840F4B2
:102F200000006049C1F860014FF4004B08E05A48C6
:102F30002038006800F0010000B104E0ABF1010BA3
:102F4000BBF1000FF3DC00BFBBF1000F0DD0554803
:102F5000B030046846F0010040F08050044344F073
:102F600000445048C0F8B0403CE04FF0000A39E05F
:102F70005048FFF787FC4B49C03108604948D0F8FA
:102F8000600120F400004749C1F860010846D0F80C
:102F9000B0404E48044044F000444248B030046021
:102FA000BAF1000F02D14FF000080AE0B9FBFAF8BD
:102FB000B8F1000F01D0A8F1010808F10100B9FB38
:102FC000F0FA5046FFF75EFC3649C03108603548DC
:102FD000D0F8B04046EA8820044344F00044314829
:102FE000B03004602F48B030006820F470002D49E4
:102FF000C1F8B0005046BEE62DE9F041064629482A
:10300000046E056F44F4006424F4800445F4006504
:103010000466056704F00100D8B106F00100C0B9EC
:1030200066F0010004404FF480701E498865084630
:1030300004664FF4002702E07F1E07B905E0194837
:10304000006D00F480700028F6D000BF0FB9BDE815
:10305000F08124F4FE6406F4FE6004431C4805403D
:103060001B49A13106EA0100054306F0080045EAC4
:10307000C0050C480466056724F4005406F40050AB
:10308000044325F4005506F400500543402005494B
:10309000886505F000401DE088E10F400400FA0556
:1030A0000CED00E000E00F40000100800000FF7028
:1030B000000005100024F4002CB7020040787D01C8
:1030C00000FC0FE078B9020098B70200FF0300EFA0
:1030D0008FFFFF7F18B108460567046602E0D648F7
:1030E00004660567D5480440C14306EA010004436D
:1030F00025F0FC5506F0FC50054306F0804040B139
:1031000044F4800425F48005CD4906EA0100054316
:1031100001E025F0804506F4006080B94FF40047D7
:1031200006E0C848006800F0010000B102E07F1E20
:10313000002FF6D100BF24F4006425F40065BE48DA
:10314000046605671020FDF7F7F800BF7FE7F0B5CC
:10315000B948036E026F02F0004010B102F0700037
:1031600001E003F03000202811D003DC38B1102832
:1031700015D10AE030280CD0702810D10CE0B248EC
:10318000C3F3841750F827100BE0B04909E0B049A9
:1031900007E047F2305104E04FF4004101E0002025
:1031A000F0BD00BF4FF0FF3402F0004010B102F458
:1031B000006028B102F0004098BB03F4006080BBBF
:1031C000A048083805689C48D0F8646106F01F00E4
:1031D000401CC6F304277F1C10FB07F04000B1FB26
:1031E000F0F1C5F309004843C5F389274F4300EBCD
:1031F000972143F480039048006900F47040B0F5D3
:10320000804F13D006DCB0F5005F0BD0B0F5405F07
:1032100012D109E0B0F5E04F0AD0B0F5104F0BD154
:1032200008E00BE08B4C08E08B4C06E08B4C04E094
:103230008B4C02E08B4C00E000BF00BF03F4800029
:1032400018B302F00040D8B102F0804090B102F013
:10325000004010B102F4006028B102F0004048B90B
:1032600003F4006030B94F00C2F38650401CB7FB36
:10327000F0F10AE0C2F3C550401CB1FBF0F104E0EC
:10328000C3F3C350401CB1FBF0F18C4200D2214685
:10329000084685E76B4924390860704710B5024637
:1032A000654B1B68704C2340704CA34208D121F041
:1032B000FC54531E44EAC353624C243C236023E075
:1032C000501E01F0700333B1102B0ED0302B05D0FF
:1032D000702B09D105E040F4401007E040F40010E5
:1032E00004E040F4800001E000BF00BF00BF01F037
:1032F00002030BB140F0004001F080430BB140F0FD
:103300008040504B243B186010BD4B49096E21F49E
:10331000F0110143484A116670474748006E00F4B7
:10332000801008B9002070474348006E00F4F01088
:10333000F9E74149C96E00F00F0301229A40114399
:103340003D4AD16670473C49C96E00F00F03012227
:103350009A409143384AD16670473748006F20F44D
:1033600080403549086770473348006F40F480401B
:103370003149086770473049886370472E48006EAE
:1033800070472D49096E01432B4A116670472DE99C
:10339000F04F054628480068DFF8CCE000EA0E0050
:1033A000DFF8C8E0704503D100200860BDE8F08F69
:1033B0002148B030076807F08050B0F1805F02D03C
:1033C00000200860F2E7C5F384161F4850F8264035
:1033D0001C48083802681848D0F86431C2F3090C58
:1033E000C2F3892803F01F09C3F3042A04FB0CF07D
:1033F00004FB08FE00EB9E2B09F101000AF1010E0F
:1034000010FB0EF0BBFBF0FBC1F800B00120CDE7D4
:103410000948406E70470849496E8143064A516623
:1034200070474A1ED2B20243064B203B1A607047D7
:10343000044930390860704700E00F40FEFF3FF854
:103440000000404068E10F402CB702000024F40067
:1034500000093D0000B4C40480F0FA02005A620280
:1034600040787D01002D31010000FF700000051043
:10347000F0B503460C46C24D0C26C2480068C24F48
:103480003840C24FB84201D1C14D082600210DE09D
:1034900055F83100984208D105EBC1004268B4F5F7
:1034A0007F4F00D1521C1046F0BD491CB142EFD3F2
:1034B0000020F9E7C26840F201130B401A43C260D2
:1034C0007047C26840F201130B409A43C2607047D4
:1034D000C26840F201139A43C2600A0E0260A94A10
:1034E0001268A94B1A40A94B9A4211D1CAB201F4F1
:1034F000702342EA131242F40072426001F4700237
:10350000C1F3072343EA122242F40072826008E00A
:10351000CAB242F400724260C1F3072242F4007260
:103520008260704744F24003194012B1C3680B43F4
:1035300001E0C3688B43C360704710B5914B1B68B3
:10354000914C2340914CA3420AD140F201130B400D
:1035500012B1046F1C4301E0046F9C43046700BF79
:1035600042F22003194012B1C3680B4301E0C36863
:103570008B43C36010BD10B540F60C431940C368BF
:103580008B4302EA01042343C36010BD40F20223CF
:10359000194012B1C3680B4301E0C3688B43C36099
:1035A0007047CBB24BB122B1436843F04003436054
:1035B00003E0436823F04003436001F47F434BB1D1
:1035C00022B1836843F04003836003E0836823F003
:1035D000400383607047C16841F01001C1607047CB
:1035E000C16821F01001C1607047C0F8C81F704762
:1035F0000146D1F8C80F7047CBB203B1826301F422
:103600007F4303B1C26370470246FF2901D1906B2B
:103610007047D06BFCE7CBB203B1026401F47F4387
:1036200003B1426470470246FF2901D1106C704714
:10363000506CFCE7CBB203B1826201F47F4303B16B
:10364000C26270470246FF2901D1906A7047D06A72
:10365000FCE7C3628262704730B5034600BFDA6A96
:103660009C6ADD6AAA42FAD1002001462043114338
:1036700030BD0246FF2901D1906C7047D06CFCE749
:1036800030B5034600BFDA6C9C6CDD6CAA42FAD1FF
:10369000002001462043114330BDCBB203B1026389
:1036A00001F47F4303B1426370470246FF2901D111
:1036B000106B7047506BFCE743630263704730B593
:1036C000034600BF5A6B1C6B5D6BAA42FAD1002007
:1036D00001462043114330BD2DE9F04105460E4619
:1036E000144631462846FFF7C3FE074621463846B2
:1036F000FEF7E2FC3846FEF73BFDBDE8F08170B511
:1037000004460D4629462046FFF7B2FE06463046DF
:10371000FEF76AFD3046FEF7E9FC70BD82690A4398
:103720008261704782698A4382617047024609B1AB
:10373000106A7047D069FCE74162704701617047C9
:10374000016770470146086F7047C16670470146C0
:10375000C86E704710B50B46DCB2FF2C04D144682C
:1037600024F4A0611143416003F47F44B4F57F4F1A
:1037700004D1846824F4A0611143816010BD00006D
:1037800080B9020000E00F400000FF7000000A1046
:10379000E0B9020030B50246C74B0824C7480068AC
:1037A000C74D2840C74DA84201D1C74B00BF0021DB
:1037B00008E053F83100904203D103EBC1004068A8
:1037C00030BD491CA142F4D30020F9E7C26A22F0BF
:1037D00086020A43C26270470146C86A00F086004A
:1037E000704741EA02034363704710B5436B03F02F
:1037F00007040C6003F03804146010BDC16A41F086
:103800001001C162016B40F2013211430163704744
:1038100000BF816901F008010029FAD1C16A21F0D5
:103820001001C162016B40F20132914301637047A4
:10383000F0B504460E4615461F462046FFF7E8FF42
:10384000B6EB051F05D2206B40F0200020636D0809
:1038500003E0206B20F020002063F000B0FBF5F0C7
:10386000401C43089809606203F03F00A062E762D1
:103870000020A0612046FFF7C1FFF0BDF0B5446A0B
:10388000856A8E00402707FB0457B6FBF7F61660E3
:10389000066B06F0200616B1166876001660C66A3A
:1038A00006F0EE061E60F0BDC16A41F01001C16273
:1038B0007047C16A21F01001C162704721B1026BEB
:1038C00042F00602026303E0026B42F0020202636E
:1038D0007047016B21F0060101637047C16A21F056
:1038E000E60141F06E01C162026B42F00802026320
:1038F0007047016B21F0080101637047026B01F40E
:1039000040631A4302637047026B01F440639A43B9
:10391000026370470146086B00F44060704701463F
:10392000886940F2071210407047026B22F440424F
:103930000A43026370470146086B00F44040704739
:10394000026B22F010020A43026370470146086BC3
:1039500000F01000704701468869012222EA101029
:10396000704701468869012222EA501070470146DB
:10397000886900F0100008B9086870474FF0FF3000
:10398000FBE7014600BF886900F010000028FAD16B
:10399000086870470246906900F0200010B9116075
:1039A000012070470020FCE700BF826902F020027E
:1039B000002AFAD10160704719B1C26A42F00102CF
:1039C00002E0C26A22F00102C262704701468869C1
:1039D000C0F3C000704770B504460D462046FFF79F
:1039E000D9FE064629463046FEF766FB3046FEF70E
:1039F000BFFB70BD70B504462046FFF7CBFE054601
:103A00002846FEF7F1FB2846FEF770FB70BD826B7F
:103A10000A4382637047826B8A438263704702461F
:103A200009B1106C7047D06BFCE741647047826C41
:103A30000A4382647047826C8A43826470470146FD
:103A4000486800F00F007047002141607047C0F8DF
:103A5000C81F70470146D1F8C80F7047D0F8A410AE
:103A600041F40041C0F8A4107047D0F8A41021F42C
:103A70000041C0F8A4107047C0F8A410C0F8A820F6
:103A800070470A4600BF836903F08803802BFAD190
:103A9000C16A21F0040343F08203C362026000BFE5
:103AA000836903F08803802BFAD1C1627047016BF0
:103AB00041F080010163704720BA020000E00F402E
:103AC0000000FF7000000A1060BA0200014688681A
:103AD00000F001007047816841F00101816070478A
:103AE000816841F0020181607047816821F0020124
:103AF000816070470121C0F8001C70472449C0F85C
:103B0000001C70470146D1F8000C012800D1704715
:103B10000020FCE7016070470146086870470146D5
:103B20004868704770B505460C4621462220FEF7CE
:103B3000C3FA2220FEF71CFB70BD10B504462220FC
:103B4000FEF752FB2220FEF7D1FA10BD816841F04A
:103B5000010181607047024609B1506970471069E0
:103B6000FCE70121C1607047826822F004020A4329
:103B700082607047D0F8181441F48071C0F81814AE
:103B80007047D0F8181421F48071C0F818147047E9
:103B900051E5CC1AEFF3098141B1F1EE101A40F86A
:103BA000041D20ED200A29490A6810607047B0EC16
:103BB000200A02C8E1EE101A25490A681060704711
:103BC000EFF3108072B6704780F310887047214879
:103BD0004FF0FF010170002080F309881E48016842
:103BE00081F308881D48012101701D484FF0805164
:103BF000016062B6FEE71A484FF0805101607047DD
:103C000017484FF080510160704772B6EFF309809A
:103C100028B1203880E8F00F0C490968086000B529
:103C2000104880475DF804EB0F4810490A7802708D
:103C3000064807490A680260106890E8F00F2030D3
:103C400080F309884EF0F40E62B670473C00002005
:103C50004400002022ED00E0080000203600002093
:103C600004ED00E08B3E00002B0000202C00002023
:103C7000A648802102E0491E002204C00029FAD192
:103C8000A34AA44B1A601A46126822F007021A606F
:103C90000022A14B1A807047704710B50446204699
:103CA00025F0FAFC10BD10B50446204625F0F5FCC1
:103CB00010BD10B525F0F2FC10BD10B5044620462D
:103CC00025F0EEFC10BD10B525F0E9FC10BD70B577
:103CD0000446101D20F007004FF08076051F28468F
:103CE0002E60051F28462C608C4E051F28462E602E
:103CF0004FF01236051F28462E604FF00336051F81
:103D000028462E604FF00236051F28462E6076109A
:103D1000051F28462E60051F284629604FF01136E2
:103D2000051F28462E604FF01036051F28462E60CE
:103D30004FF00936051F28462E604FF00836051F44
:103D400028462E604FF00736051F28462E604FF09C
:103D50000636051F28462E604FF00536051F2846FB
:103D60002E604FF00436051F28462E6003F0040530
:103D7000002D7DD0F605051F28462E60684E051FD4
:103D800028462E60674E051F28462E60664E051F8A
:103D900028462E60654E051F28462E60644E051F7E
:103DA00028462E60634E051F28462E60624E051F72
:103DB00028462E60614E051F28462E60604E051F66
:103DC00028462E605F4E051F28462E605E4E051F5A
:103DD00028462E605D4E051F28462E605C4E051F4E
:103DE00028462E605B4E051F28462E605A4E051F42
:103DF00028462E604FF08346051F28462E60574EFA
:103E0000051F28462E60564E051F28462E60554E2B
:103E1000051F28462E60544E051F28462E60534E1F
:103E2000051F28462E60524E051F28462E60514E13
:103E3000051F28462E604FF08246051F28462E603B
:103E40004D4E051F28462E604C4E051F28462E60FD
:103E50004B4E051F28462E604FF08146051F284611
:103E60002E60484E051F28462E603602051F00E0D2
:103E70000AE028462E604FF07E56051F28462E6029
:103E80000026051F28462E6070BD10B525F009FCE0
:103E900010BD10B50446204625F004FC10BD10B539
:103EA00025F001FC1C480088401C1B49088008467E
:103EB000008818B10020088003F0E0F810BD10B5AC
:103EC000FFF77EFE044630480078401C2E490870FB
:103ED0002046FFF779FE00F0CDFD00F0CFFC10BDCD
:103EE00001464A1E4FF0E0235A61284A106820F02C
:103EF0007F4000BF10601A46126942F005021A6145
:103F00001A46126942F002021A6170476C0A0020D8
:103F10006C0C0020080000200C000020E969000063
:103F20000000F8410000F0410000E8410000E041DD
:103F30000000D8410000D0410000C8410000C0414D
:103F40000000B8410000B0410000A8410000A041BD
:103F5000000098410000904100008841000070413D
:103F6000000060410000504100004041000030412D
:103F700000002041000010410000E0400000C0406F
:103F80000000A040000040402900002020ED00E09B
:103F90001D481E481E481F481F48204820482148E9
:103FA00021482248224823482348244824482548B9
:103FB0002548264826482748274828482848294889
:103FC00029482A482A482B482B482C482C482D4859
:103FD0002D482E482E482F482F4830483048314829
:103FE00031483248324833483348344834483548F9
:103FF00035483648364837483748384838483948C9
:10400000394800BF70470000A0BA0200A4BA0200FD
:10401000AABA0200ACBA0200A8BA0200AEBA020004
:10402000B0BA0200B2BA0200B4BA0200B6BA0200D4
:10403000B8BA0200BABA0200BCBA0200BEBA0200A4
:10404000C0BA0200C2BA0200C4BA0200C6BA020074
:10405000C8BA0200CABA0200CCBA0200CEBA020044
:10406000D0BA0200D2BA0200D4BA0200D6BA020014
:10407000D8BA0200DABA0200DCBA0200DEBA0200E4
:10408000E0BA0200E2BA0200E4BA0200E6BA0200B4
:10409000E8BA0200EABA0200ECBA0200EEBA020084
:1040A000F0BA0200F2BA0200F6BA0200F8BA020050
:1040B000FABA0200FCBA0200B42B0020343000200F
:1040C00000BB020002BB020004BB020006BB0200F0
:1040D00008BB02000ABB02000CBB02000EBB0200C0
:1040E00010BB0200FEBA020012BB02000146002013
:1040F00002E0491C421CD0B20A78002AF9D170476C
:104100002DE9F04105460E4614460027FB4800788D
:1041100020B1112020700020BDE8F081287801280E
:1041200008D0022807D0032802D0042804D100E0D8
:1041300000BF00BF00BF03E0012020700020EBE7BC
:1041400000BFFFF73DFD0746686930603068FFF744
:10415000CDFF80463846FFF737FD002020704046EF
:10416000DAE72DE9F04105460E4614460027E348FC
:10417000007818B112202070BDE8F081287801285D
:1041800008D0022807D0032802D0042804D100E078
:1041900000BF00BF00BF02E001202070ECE700BFBD
:1041A000FFF70EFD07466E613846FFF70DFD002054
:1041B000207000BFE0E7F0B5024612F8384F95785E
:1041C0005678383A0B4618680FE000F10B073F5D50
:1041D000B74300F10B0C0CF8047067463F5D17B94C
:1041E000877AAF4387721B1D18680028EDD1F0BD98
:1041F000C349C44A1278885CC349095CC04A515C0F
:1042000001EBC001C14A1170704710B50024FFF7DF
:10421000D7FC0446B9480078F8B9BD480078E0B941
:10422000FFF7E6FFBB48B949097850F82100BA49C1
:104230000860B6480078B949097888420DD0B64878
:104240000068C06B401CB4490968C863B448006882
:10425000401CB3490860FFF7CEFC2046FFF7B4FCD2
:1042600010BD70B501460024AE4D2D68EC61AD4C1B
:10427000246821620B4618681BE0AA4C246894F855
:10428000385000F10B04645DA64D2D6895F8395047
:104290002C43A44D2D6895F8386000F10B05AC5502
:1042A000847AA04D2D6895F83A502C4384721B1DDA
:1042B00018680028E1D19B4C246894F83820924C6F
:1042C000A45C984D2D6895F83950AC438E4DAC5494
:1042D0002C46A45C44B9934C246894F83A50894C19
:1042E0002478AC43874D2C7070BD2DE9FF4F83B00F
:1042F00081460E461546DDF8408000200090306073
:10430000CA46DAF8004018E02078062807D2DFE82D
:1043100000F00604050307080AE009E008E000BF12
:1043200000BF012088F80000002007B0BDE8F08F32
:1043300000BF0AF1040ADAF80040002CE4D16F480B
:10434000007820B1022088F800000020EDE77048D6
:10435000007820B10D2088F800000020E5E700205B
:10436000029001908346CA46DAF80040FFF728FC25
:10437000009057E02078062843D2DFE800F042158D
:1043800026034344208960B12089401E208110C645
:1043900001200290002001C50198401C80B20190CC
:1043A00001E04BF0010B38E0606858B1606801C56E
:1043B0000020606010C6012002900198401C80B26D
:1043C000019001E04BF0020B27E06768F88AA8B182
:1043D0003969081D3861086801C5B96838698842BB
:1043E00001D178683861F88A401EF88210C6012031
:1043F00002900198401C80B2019001E04BF0040B48
:104400000BE000BF00BF0098FFF7DEFB002030602C
:10441000012088F80000019887E700BF0AF1040A2C
:10442000DAF80040002CA5D10298012809D100201B
:1044300030600098FFF7C8FB002088F80000019862
:1044400073E73848006890F834004BF08001084367
:104450003449096881F8340000203249096881F83C
:10446000350030490698096808634846FFF7F9FEA9
:104470000098FFF7A9FBFFF7C8FEFFF7A1FB00902C
:104480002848006890F8350020B1012819D002288A
:1044900016D100E000BF23480068C4692CB110C6E3
:1044A000002030600120019009E001201D490968C9
:1044B00081F8350049461B480068FFF77CFE06E09E
:1044C00000BF494617480068FFF775FE00BF00BFF0
:1044D0001448006890F8350020B1012842D0022825
:1044E0003FD138E02078062824D2DFE800F0231DF1
:1044F0001E032425002001C528E00000290000201B
:1045000014BB02002D0000202E0000202C000020F3
:104510002A000020F4160020440000202B00002078
:10452000100000203C00002000BFFD480068406AE9
:1045300001C50BE000BF00BF0098FFF745FB00205E
:104540003060012088F800000198EEE600BF0020EE
:1045500088F800000CE0002001C50E2088F800005B
:1045600006E000BF002001C50A2088F8000000BF57
:1045700000BF0020EA49096881F83400E849096869
:1045800081F83500E6490968C861E54909680862AB
:10459000E349096848620098FFF716FB0198C4E6F2
:1045A0007CB5002514E06946284602F00EF906465F
:1045B00066B9DC4850F8254044B1012C06D0D4E956
:1045C000020100EB8100A0640198E064681CC5B2A0
:1045D0003F2DE8D97CBD00BF00BF02E0C82002F03B
:1045E0001BFAD14800780028F8D0D0480068642130
:1045F000B0FBF1F0CD4908600846006828B90020FA
:10460000CB490870FF2002F020F9FFF7D9FA0446E1
:10461000C648006864214843C64908602046FFF741
:10462000D3FA00BFFFF7CCFA0446C2480068C2497B
:1046300008600020BF4908602046FFF7C5FABE4861
:104640000068BA490968B0FBF1F0C0F16400B849EC
:104650000870FFF738FBFFF7A3FF642002F0DCF9D6
:10466000E0E700B587B0032000218022B34BCDE9FD
:104670000132CDE903104FF6FE703E23B04A0090A0
:10468000AFF2AD0001F0B3FE06AAAEA13E2002F0EB
:104690001EF807B000BD002400BF00BFFFF790FA6E
:1046A0000446A4480068401CA24908602046FFF761
:1046B0008BFAFFF7FEFAF1E700B587B0032000217F
:1046C0008022A44BCDE90132CDE903104FF6FF70F3
:1046D0003F23A14A0090AFF2410001F088FE06AAF4
:1046E0009EA13F2001F0F3FF07B000BD04E00022CF
:1046F00000F8012B4A1E91B20029F8D1704770B51D
:104700004FF4BD619948FFF7F1FF002411E0601CF0
:1047100085B204EB4400954901EBC00305EB45006D
:1047200001EBC006002018705E6091A05861601C0B
:1047300084B23E2CEBD304EB44008C4901EBC00364
:104740000020187058608AA058610846894908609E
:1047500070BD70B54FF48F518748FFF7C7FF4FF416
:1047600080717048FFF7C2FF002413E0601CC5B2DF
:1047700004EB440000EBC4007F4901EBC00305EBF0
:10478000450000EBC50001EBC0065E6178A018652E
:10479000601CC4B2332CE9D304EB440000EBC4002A
:1047A000754901EBC0030020586171A01865002015
:1047B0007249086070487249086070BD0021714AF2
:1047C0001170002004E000216F4A1154411CC8B24E
:1047D0000828F8D300216D4A11706D4A11706D4A96
:1047E00011604F4A1160704700206B4908606B49A7
:1047F00008706B4908706B4908706B4908706B4909
:1048000008604C4908604C490860484908604649BE
:10481000087067490870704710B5FFF729FAFFF76D
:10482000E3FFFFF7CBFFFFF794FFFFF768FF00F010
:10483000CFFE00F0C0FF01F0C2FAFFF73DFFFFF727
:1048400010FF02F075FCFFF727FAFFF7A1FB10BD80
:1048500010B50024FFF7B4F9044653480078012846
:1048600008D14E480078FF2804D24C480078401CFC
:104870004A4908702046FFF7A7F910BD10B500247B
:1048800049480078012830D1FFF79AF90446434897
:10489000007820B141480078401E404908703F48E8
:1048A0000078F8B93E480078E0B9FFF7A1FC1D4850
:1048B0003749097850F821003649086034480078B3
:1048C0003249097888420DD032480068C06B401CDC
:1048D00030490968C86335480068401C334908609E
:1048E000FFF78EF92046FFF76FF910BD10B50024D1
:1048F0002D480078012811D1FFF762F904462748B6
:10490000007840B926480078FF2804D2244800786F
:10491000401C234908702046FFF756F910BD0000DF
:104920003C000020F4160020280000202000002079
:104930001C0000203800002024000020F412002079
:10494000F014002075432F4F532D494920537461B3
:1049500074000000F4140020F016002075432F4F5F
:10496000532D49492049646C650000006C0C0020FF
:104970003F00000014000020F41700204800002031
:10498000400000202D0000202E0000202B000020E1
:104990002C000020440000205C00002029000020A2
:1049A0002A000020370000203600002010000020E0
:1049B0005800002010B50024FD480078012821D1BE
:1049C000FFF7FEF80446FB480078C0B9FA480078C3
:1049D00088B1F9480078401EF74908700846007809
:1049E00028B92046FFF7F0F8FFF70FFC0AE0204651
:1049F000FFF7EAF806E02046FFF7E6F802E0204677
:104A0000FFF7E2F810BD10B5E948007890B9FFF75C
:104A1000EFFBEA480078EA490870EA48E749097874
:104A200050F82100E849086008460068E749086036
:104A3000FFF7CDF810BD10B50024022001F0ECFF07
:104A4000FFF7BEF804460020E14908602046FFF762
:104A5000BBF8642001F0E0FFFFF7B2F80446DC4841
:104A60000068DC4908600120DB4908702046FFF738
:104A7000ABF810BD70B50026FFF711FAFFF7A0F8EC
:104A80000646D6480068401CD44908603046FFF707
:104A90009BF8C7480078012853D1D148007820B14D
:104AA000012804D0022809D103E001250BE00025EC
:104AB00009E001250120CA49087004E00125002011
:104AC000C749087000BF00BF05B970BDC54804687C
:104AD00033E0FFF775F80646206B50B3206B401E9D
:104AE0002063206B28BB94F8340000F0370040B1FD
:104AF00014F8340F00F0C800207001206070343CBE
:104B000002E0002084F8350094F8340000F008003A
:104B100078B93834A078B44909780843B2490870A4
:104B20002078B249085C6178084314F83819AF4A14
:104B3000505464693046FFF747F894F836003F2830
:104B4000C7D100BFC1E747F21A207047704710B5C0
:104B500090F8382001F10B039B5C90F83940A34397
:104B600001F10B04A35423469B5C23B98B7A90F884
:104B70003A40A3438B720023C36110BD2DE9F04F6F
:104B800005460F4690469946A87A99490E5C05F16C
:104B90000B00805D11F800B00BEBC60000F0FF0ABF
:104BA000884850F82A4000202434E0602760207CA8
:104BB00020EA0800207484F81190207C243C00F046
:104BC000080068B994F83A0087490978084386498B
:104BD00008708648805D94F83910084383498855E9
:104BE00029462046FFF7B3FF206A20B12046216AFC
:104BF000FFF7E1FAE5615046BDE8F08F10B5734A62
:104C00001268D061714A126892F8383000F10B02D4
:104C1000D25C6E4B1B6893F839301A436B4B1B68A0
:104C200093F8384000F10B031A55827A674B1B68E2
:104C300093F83A301A438272644A126892F8381034
:104C40006A4A525C614B1B6893F839309A43674B50
:104C50005A541A46525C42B95C4A126892F83A3089
:104C6000614A12789A43604B1A7010BD01460022C7
:104C70008A72002005E0002301F10B021354421C4C
:104C8000D0B20828F7D3704705E011F8013B00F8CF
:104C9000013B531E9AB2002AF7D170472DE9F84F15
:104CA00005460F4690469946DDE90AAB0020009084
:104CB000FEF786FF00904F480468002C77D01C3424
:104CC00054F8080C4B4908600098FEF77DFF44F843
:104CD0001C7CA576002020766076606144F818BCC4
:104CE00044F810AC44F8148C0C9824F80C0C24F8FC
:104CF0000A9C0020E077E810207705F00700E076B6
:104D0000217F01208840A077E17E012088406077E4
:104D1000002020606060E060A0602062A0626062AD
:104D2000E0622063AFF2B83060631C3C002606E00E
:104D3000002104F1540040F82610701CC6B2002E69
:104D4000F6D02046FFF7A5F8FEF73AFF00901D4881
:104D500040F825400098FEF737FF2046FEF79DFFFC
:104D6000FEF72EFF00901F48006860610020A061E0
:104D70001C48006810B11B48006884611948046031
:104D80003834A07818490978084317490870207802
:104D90001649085C6178084314F83819134A5054CE
:104DA00015480078401C14490870009826E02AE055
:104DB00036000020290000202A0000202C000020BE
:104DC0002B000020F4160020440000203C000020AE
:104DD0003800002020000020280000205C00002077
:104DE0004C000020480000202D0000202E00002054
:104DF00014BB02004000002037000020FEF7E4FE54
:104E00000020BDE8F88F0098FEF7DEFE4220F8E7AC
:104E10002DE9F05F04460F4691461E464FF0000B09
:104E20002078052804D0012030700020BDE8F09FD4
:104E300009F0800ABAF1000F04D029F080094FF080
:104E4000010801E04FF0000800203070FEF7B8FEC6
:104E50008346B9F1000F2CD0B9F1010F3BD0B9F165
:104E6000020F03D0B9F1030F46D111E0208900EA07
:104E70000705BD4206D1B8F1010F05D12089A8432D
:104E8000208101E0702030705846FEF79DFE3AE028
:104E9000208900EA070535B1B8F1010F05D1208955
:104EA000A843208101E0702030705846FEF78CFE48
:104EB00029E0208927EA0005BD4206D1B8F1010F9B
:104EC00005D120892843208101E0702030705846A8
:104ED000FEF77AFE17E0208927EA000535B1B8F120
:104EE000010F05D120892843208101E07020307016
:104EF0005846FEF769FE06E05846FEF765FE0025B7
:104F00006F20307000BF00BF28468FE72DE9F041C9
:104F100006460D460027FC48007820B11020287076
:104F20000020BDE8F081FEF74BFE0746F748046815
:104F300084B100684068F54908600520207026812A
:104F400000206060F2A0E0603846FEF73DFE0020E1
:104F5000287004E03846FEF737FE7220287020469D
:104F6000DFE730B501464A6808682AB9CC68606056
:104F700028B10025456002E0106000B142608B68F6
:104F800000259D6230BD2DE9F04106468846174652
:104F9000B468002044F8300F24F8048C207900F025
:104FA000DF00207167712079303C88B93834A078EF
:104FB000D84909780843D74908702078D649085C51
:104FC0006178084314F83819D34A5054012500E099
:104FD00000253046FFF7C5FF2846BDE8F0812DE9E2
:104FE000F0470446894615464FF0000AC648007847
:104FF00020B10F2028702046BDE8F08720780528D2
:1050000003D0012028702046F6E7FEF7D9FD82463E
:10501000606808B1012700E00027B9F1000F03D054
:10502000B9F1010F3DD119E08FB9B9A0E0600020BE
:105030002070B6480068606000202081B34804609A
:105040005046FEF7C1FD00202870002605E05046BE
:10505000FEF7BAFD49202870264629E0D4F80480DE
:1050600006E0022200214046FFF78DFFD8F80080BD
:10507000B8F1000FF5D1A6A0E06000202070A34891
:105080000068606000202081A04804605046FEF760
:105090009BFD012F01D1FFF7B8F8002028700026F2
:1050A00006E05046FEF790FD07202870264600BF18
:1050B00000BF3046A0E72DE9F04105460E461446F4
:1050C00000279148007820B1112020700020BDE811
:1050D000F081FEF775FD07462878052806D038468A
:1050E000FEF772FD012020700020F0E7E8683060D4
:1050F0003068FEF7FBFF80463846FEF765FD00206E
:1051000020704046E3E72DE9F04105460E4614467F
:1051100000277D48007818B112202070BDE8F0818A
:10512000FEF74EFD07462878052805D03846FEF7DD
:105130004BFD01202070F1E7EE603846FEF744FD9C
:105140000020207000BFE9E7F0B51446059E734FBC
:105150003F6897F8347047F02007DFF8C0C1DCF8EB
:1051600000C08CF834700027DFF8B0C1DCF800C054
:105170008CF83570694F3F683E63684F3F68B9628D
:105180000C828B74654F3F688F6047680F60002703
:105190004F60C860456805B1696041605F4F3F6816
:1051A00097F838205C4FBF5CDFF870C1DCF800C0B6
:1051B0009CF839C027EA0C07DFF85CC10CF80270D4
:1051C0006746BF5C5FB9554F3F6897F83AC0514F8B
:1051D0003F7827EA0C07DFF83CC18CF80070F0BD7F
:1051E0002DE9F04F89B005460F4691469A46129E2A
:1051F000002002904448007828B10220307000203E
:1052000009B0BDE8F08F4648007818B10D20307025
:105210000020F5E72878052803D001203070002011
:10522000EEE709F0800BBBF1000F04D009F07F0915
:105230004FF0010801E04FF00008FEF7C1FC0290BA
:10524000B9F1000F4AD0B9F1010F78D0B9F1020FCE
:1052500003D0B9F1030F71D120E0288900EA0704D7
:10526000BC420FD1B8F1010F02D12889A043288197
:105270002A48006884850298FEF7A6FC002030705A
:105280002046BDE74B463A4604A92846CDF800A083
:10529000FFF75AFF0298FEF797FC78E0288900EAAA
:1052A00007047CB1B8F1010F02D12889A0432881FD
:1052B0001A48006884850298FEF786FC002030704A
:1052C00020469DE74B463A4604A92846CDF800A063
:1052D000FFF73AFF0298FEF777FC58E0288927EAA3
:1052E0000004BC421ED1B8F1010F02D1288920432D
:1052F00028810A48006884850298FEF765FC002032
:10530000307020467CE71AE02900002018000020B9
:105310003F0000002D0000202E0000203C00002057
:105320002A0000204B463A4604A92846CDF800A0A2
:10533000FFF70AFF0298FEF747FC28E01FE02889E4
:1053400027EA00047CB1B8F1010F02D1288920437B
:105350002881B348006884850298FEF735FC002058
:10536000307020464CE74B463A4604A92846CDF813
:1053700000A0FFF7E9FE0298FEF726FC07E002987E
:10538000FEF722FC00246F203070204638E700BF73
:10539000FEF73BFFFEF714FC0290A148006890F86E
:1053A000350020B39E48006890F835000390002037
:1053B0009B49096881F8350004A8FFF7D2FD002059
:1053C0009749096881F834000298FEF7FDFB002434
:1053D0000398012805D0022802D10E20307003E086
:1053E00000BF0A20307000BF00BF204608E78C488D
:1053F0000068848DB8F1010F1ED1B9F1000F0ED0F5
:10540000B9F1010F0CD0B9F1020F03D0B9F1030FBC
:105410000AD100E000BF2889A04328810BE000BF2B
:1054200028892043288106E00298FEF7CDFB6F20F3
:1054300030700020E4E600BF0298FEF7C5FB0020B4
:1054400030702046DCE670B50025FEF7B9FB054656
:1054500073480068848D2846FEF7B6FB204670BD71
:105460002DE9FC5F0446894692461E4600200090C6
:105470002078052804D0012030700020BDE8FC9F72
:10548000FEF79EFB0090BAF1000F03D0BAF1010FB6
:105490000AD104E0208920EA090020810BE020895C
:1054A00040EA0900208106E00098FEF78DFB71209C
:1054B00030700020E2E700BF4FF0000B656859E054
:1054C000A87C50B301283BD0022802D0032848D141
:1054D00012E02089298A00EA0107288AB8420AD105
:1054E000002239462846FFF74EFD8046B8F1010FED
:1054F00001D14FF0010B3BE02089298A00EA010726
:1055000057B1002239462846FFF73DFD8046B8F1E5
:10551000010F01D14FF0010B2AE0288A218920EAEE
:105520000107288AB8420AD1002239462846FFF7E7
:105530002AFD8046B8F1010F01D14FF0010B17E0B1
:10554000288A218920EA010757B1002239462846D6
:10555000FFF719FD8046B8F1010F01D14FF0010BA3
:1055600006E00098FEF730FB6F203070002085E7E2
:1055700000BF2D68002DA3D10098FEF725FBBBF1DD
:10558000010F01D1FEF741FEFEF71AFB00902089C2
:1055900001900098FEF718FB0020307001986DE72D
:1055A0002DE9F04104460D4600272078052804D057
:1055B000012028700020BDE8F081FEF701FB0746BE
:1055C00026893846FEF700FB002028703046F2E7B7
:1055D0002DE9F041A0211348FFF788F800250EE0DF
:1055E000681C86B20F4800EB051400EB061700207C
:1055F00020706760AFF2E820E060681C85B2092D7A
:10560000EED3084800EB0514002020706060AFF274
:105610000030E060034804490860BDE8F081000004
:105620003C00002054120020180000202DE9FC5FEF
:1056300005460F4691469A4600200090FEF7C0FAB4
:1056400000906F480468006820B16D4800684068A9
:105650006B4908600098FEF7B7FA2CB95A208AF80F
:1056600000000020BDE8FC9FA8462E46781E019051
:105670004FF0000B05E04E44C8F80060B0460BF157
:10568000010B01988345F6D30020C8F8000025607F
:1056900065602761E760C4F808908AF8000020463A
:1056A000E0E72DE9F04104460D460027FEF788FAB1
:1056B0000746206968B16668306860602069401EEE
:1056C00020613846FEF780FA002028703046BDE899
:1056D000F0813846FEF778FA5D2028700020F6E762
:1056E0002DE9F04106460C4615460027454800784E
:1056F00020B1112028700020BDE8F081FEF760FA8B
:105700000746706920602068FEF7F0FC8046384646
:10571000FEF75AFA002028704046EDE72DE9F041E7
:1057200005460E46144600273648007818B1122068
:105730002070BDE8F081FEF743FA07466E613846F7
:10574000FEF742FA0020207000BFF2E770B5044671
:105750000D460026FEF734FA0646D4E903108842C7
:1057600004D33046FEF730FA5E2070BD60682860D2
:1057700065602069401C20613046FEF725FA002054
:10578000F3E770B505460C460026FEF719FA064603
:105790002868206068686060A868A060E868E060C9
:1057A000286920613046FEF70FFAD4E90301401A58
:1057B0006061002070BD70B5F0211348FEF796FFC0
:1057C00000240EE004EB44000F4901EBC005601C0F
:1057D00000EB400001EBC00068600CA06861601C39
:1057E00084B2092CEED304EB4400074901EBC00559
:1057F0000020686005A0686108460149086070BD26
:105800005000002029000020D42900203F00000083
:105810002DE9F04106460D464FF000083078022889
:1058200004D0012028700020BDE8F081FEF7C8F9FF
:1058300080467468E08A78B12169081D20610F688C
:10584000E08A401EE082A1682069884201D1606838
:1058500020610020287002E01F20287000274046A9
:10586000FEF7B2F93846DFE72DE9F04106460F466C
:105870004FF00008F748007810B10020BDE8F08133
:10588000FEF79EF98046F4480468006820B1F248AB
:1058900000684068F04908604046FEF795F9FCB1A1
:1058A000FEF78EF98046ED480568D5B100680068BE
:1058B000EA4908604046FEF787F96E6006EB87000C
:1058C000A860EE602E61AF820020E8820220207086
:1058D000002020816560E2A060612046FFF7C6F9E4
:1058E00008E0DD4800686060DB4804604046FEF781
:1058F0006BF900242046C1E72DE9F04704468946AC
:1059000015464FF0000A2078022804D001202870A4
:105910002046BDE8F087CF48007818B10F202870E6
:105920002046F6E7FEF74CF98246A07A10B14FF018
:10593000010801E04FF00008B9F1000F03D0B9F100
:10594000010F49D121E0B8F1000F17D1C4A0606167
:105950006668C24800683060C04806600020207059
:10596000BD480068606000202081BB48046050464C
:10597000FEF72AF900202870002705E05046FEF7C0
:1059800023F94920287027462DE005E00223042250
:1059900000212046FFF7F2F8A07A0028F6D1B0A047
:1059A00060616668AD4800683060AC480660002001
:1059B0002070A9480068606000202081A64804602B
:1059C0005046FEF701F9B8F1010F01D1FEF71DFCB9
:1059D00000202870002706E05046FEF7F5F8072063
:1059E0002870274600BF00BF384692E770B50546CD
:1059F0000026FEF7E5F806466C686068E0606068BF
:105A000020610020E0823046FEF7DEF8002070BD05
:105A10002DE9F0470746884615464FF000093878CB
:105A2000022804D0012028700020BDE8F0878948B2
:105A3000007818B1022028700020F6E78948007825
:105A400018B10D2028700020EFE7FEF7B9F8814665
:105A50007C68E08A98B12169081D20610E68E08A9F
:105A6000401EE082A1682069884201D160682061FF
:105A70004846FEF7A9F8002028703046D5E77A4856
:105A8000006890F8340040F004007749096881F814
:105A9000340000207449096881F8350072480068B4
:105AA000C0F830803846FFF7A9F84846FEF78CF872
:105AB000FEF7ABFBFEF784F881466B48006890F870
:105AC000350020B101280DD002280AD105E0664832
:105AD0000068466A002028700DE000260E2028701D
:105AE00009E000BF394660480068FFF730F800263B
:105AF0000A20287000BF00BF00205B49096881F8B8
:105B000034005949096881F8350057490968C86166
:105B10005549096808625449096848624846FEF7D1
:105B200053F8304681E72DE9F04104460F4615460B
:105B30004FF000082078022804D0012028700020AF
:105B4000BDE8F081FEF73CF88046A07A20B300263D
:105B50007FB1012F0CD107E002230422002120464F
:105B6000FFF70CF8701CC6B2A07A0028F4D109E047
:105B700000BF0223042200212046FEF7FFFF701C15
:105B8000C6B200BF00BF4046FEF71EF8FEF73DFB61
:105B90000E2028703046D3E74046FEF715F8002067
:105BA000287000BFCCE72DE9F04105460E460027DE
:105BB0002878022802D00120BDE8F081FEF700F825
:105BC0000746A87A60B10023042231462846FEF732
:105BD000D5FF3846FDF7F8FFFEF717FB0020EBE78F
:105BE0006C68E08AA18A884204DB3846FDF7ECFF46
:105BF0001E20E1E7E168081DE0600E60E08A401CBD
:105C0000E082D4E90210884201D16068E060384641
:105C1000FDF7DAFF0020CFE72DE9F04105460E46FB
:105C200000272878022802D00120BDE8F081FDF786
:105C3000C7FF0746A87AC8B1002304223146284688
:105C4000FEF79CFF3846FDF7BFFFFEF7DEFA0020A7
:105C5000EBE7000029000020140000205400002081
:105C60003F0000002A0000203C0000206C68E08A11
:105C7000A18A884204DB3846FDF7A6FF1E20D4E740
:105C800061682069884201D1A06820612069001FF5
:105C9000206120690660E08A401CE0823846FDF7FA
:105CA00093FF0020C1E72DE9F04105460F46164657
:105CB0004FF000082878022802D00120BDE8F081CA
:105CC000FDF77EFF8046A87AE8B106F0010050B1EA
:105CD00005E00023042239462846FEF74FFFA87A44
:105CE0000028F6D105E00023042239462846FEF7B5
:105CF00045FF4046FDF768FF06F0040008B9FEF7CF
:105D000084FA0020DAE76C68E08AA18A884204DB22
:105D10004046FDF759FF1E20D0E706F0020058B1BB
:105D200061682069884201D1A06820612069001F54
:105D300020612069076009E0E168081DE0600F60EC
:105D4000D4E90210884201D16068E060E08A401C1A
:105D5000E0824046FDF738FF0020AFE72DE9F0472D
:105D600005460C464FF0000A2878022802D0012090
:105D7000BDE8F087FDF724FF8246A87A207405F17C
:105D80000B0804F10809002705E018F8010B09F8D1
:105D9000010B781CC7B2082FF7D36E68F08A18B1D0
:105DA00030690068206001E000202060F08AA08057
:105DB000B08AE0805046FDF707FF0020D8E72DE9C4
:105DC000F041F0211048FEF791FC00240DE0601C2A
:105DD00086B204EB44000C4901EBC00506EB46001B
:105DE00001EBC0072F60601C84B2092CEFD304EBD9
:105DF0004400054901EBC00500202860084603491E
:105E00000860BDE8F0810000C42A00205400002092
:105E100070B5044600262078032801D0002070BD0C
:105E2000FDF7CEFE0646258915B12089401E20814A
:105E30003046FDF7C9FE2846F1E770B50546002655
:105E4000D748007808B1002070BDFDF7B9FE0646BE
:105E5000D4480468006820B1D24800684068D1493D
:105E600008603046FDF7B0FE4CB10320207025815C
:105E700000206060CCA060612046FEF7F7FE20465F
:105E8000E2E72DE9F0470446884615464FF0000941
:105E90002078032804D0012028702046BDE8F08730
:105EA000BF48007818B10F2028702046F6E7FDF7AC
:105EB00087FE8146A07A08B1012700E00027B8F1EB
:105EC000000F03D0B8F1010F3AD119E08FB9B6A095
:105ED000606100202070B34800686060002020816D
:105EE000B04804604846FDF76FFE00202870002689
:105EF00005E04846FDF768FE49202870264626E062
:105F000005E00223012200212046FEF737FEA07A99
:105F10000028F6D1A4A0606100202070A14800688C
:105F20006060002020819F4804604846FDF74CFED9
:105F3000012F01D1FEF769F900202870002606E044
:105F40004846FDF741FE07202870264600BF00BFE7
:105F50003046A3E72DE9F04105460E4614460027DA
:105F60002878032803D001202070BDE8F0818C48F8
:105F7000007810B102202070F7E78C48007810B14B
:105F80000D202070F1E7FDF71BFE0746288940B180
:105F90002889401E28813846FDF716FE0020207013
:105FA000E3E78348006890F8340040F0010080493E
:105FB000096881F8340000207D49096881F83500BE
:105FC0007B48006806632846FEF718FE3846FDF752
:105FD000FBFDFEF71AF9FDF7F3FD0746744800686C
:105FE00090F8350020B1012809D0022806D102E03E
:105FF000002020700BE00E20207008E000BF294632
:106000006B480068FEF7A3FD0A20207000BF00BFA8
:1060100000206749096881F834006549096881F8FA
:10602000350063490968C8616149096808623846F2
:10603000FDF7CAFD00BF98E72DE9F04104460F4681
:1060400015464FF000082078032804D0012028705E
:106050000020BDE8F081FDF7B3FD8046A07A20B3B3
:1060600000267FB1012F0CD107E00223012200217D
:106070002046FEF783FD701CC6B2A07A0028F4D13A
:1060800009E000BF0223012200212046FEF776FD31
:10609000701CC6B200BF00BF4046FDF795FDFEF77D
:1060A000B4F80E2028703046D3E74046FDF78CFD4B
:1060B0000020287000BFCCE770B50446002520788A
:1060C000032801D0012070BDFDF77AFD0546A07AB6
:1060D00060B10023012219462046FEF74FFD2846F5
:1060E000FDF772FDFEF791F80020ECE720894FF6EE
:1060F000FF71884207D22089401C20812846FDF785
:1061000063FD0020DFE72846FDF75EFD3320DAE778
:106110002DE9F04704460D464FF00009207803288A
:1061200002D00120BDE8F087FDF74AFD8146A07A44
:10613000A87204F10B0705F10208002605E017F824
:10614000010B08F8010B701CC6B2082EF7D320898A
:1061500028804846FDF738FD0020E3E72DE9F041AF
:1061600004460E46154600272078032803D0012058
:106170002870BDE8F081FDF723FD07460020287058
:10618000208908B1268105E0A07A08B9268101E0BE
:10619000492028703846FDF717FD00BFE9E70000E9
:1061A00029000020140000203F0000002A000020E9
:1061B0003C0000202DE9F34F85B088460020019077
:1061C000FDF7FEFC0190FE4850F8280030B1019820
:1061D000FDF7FAFC282007B0BDE8F08F0598FF28EE
:1061E00004D1F848006890F836000590F449059805
:1061F00051F8205025B90198FDF7E6FC2920EAE77F
:10620000012D04D10198FDF7DFFC4320E3E74FEABD
:10621000E80708F0070003900120B84000F0FF09EC
:1062200001210398814001F0FF0A0021E44A05980A
:1062300042F82010104640F8285095F8386095F83C
:106240003A00029095F839B0DF48805D00EA0B0013
:10625000D0B1DD48805D20EA0B00DB498855084657
:10626000805D28B9D948007802998843D7490870D9
:10627000D648007840EA0900D4490870D248C05D89
:1062800040EA0A00D049C855EC69D4B104F10B00CA
:10629000805D20EA0B0004F10B0188550846805D03
:1062A00018B9A07A02998843A072A07A40EA09003E
:1062B000A07204F10B00C05D40EA0A0004F10B017A
:1062C000C855286A30B3286A0490049804681FE00F
:1062D00004F10B00805D20EA0B0004F10B018855EE
:1062E0000846805D18B9A07A02998843A072A07A06
:1062F00040EA0900A07204F10B00C05D40EA0A0008
:1063000004F10B01C8550498001D0490049804681A
:10631000002CDDD185F8368085F83870039885F833
:10632000370085F83A9085F839A00198FDF74CFCC4
:10633000A7480078012801D1FDF767FF00204AE750
:106340002DE9FE4F06460F4690461C464FF00009C9
:10635000FDF736FC81469F48007828B14846FDF796
:1063600033FC3C20BDE8FE8F954850F8240060BB0C
:106370000120934941F824004846FDF725FC0023FD
:10638000424639463046FDF7A2FC82460020009086
:10639000019003460246514602902046FEF77EFCDD
:1063A000054635B98A48007801280CD1FDF72DFF44
:1063B00009E0FDF705FC81460020814941F82400F1
:1063C0004846FDF701FC2846CCE74846FDF7FCFBB4
:1063D0002820C7E702F0010343B102F002032BB10A
:1063E00002E0491E002308C00029FAD170472DE9B8
:1063F000F04F85B081468A4693461C46DDE90F780A
:10640000129D00200390FDF7DBFB0390714800789C
:1064100030B10398FDF7D8FB3C2005B0BDE8F08F04
:10642000674850F8240088BB0120654941F82400E2
:106430000398FDF7C9FB2A4641463846FFF7CAFFD5
:106440002B465A4651464846FDF741FC04901198A8
:10645000CDE9008002953A4620460E9B0499FEF74E
:106460001DFC064636B95A48007801280CD1FDF7C4
:10647000CCFE09E0FDF7A4FB03900020504941F851
:1064800024000398FDF7A0FB3046C6E7FFE703981A
:10649000FDF79AFB2820C0E72DE9F04105460027CB
:1064A0004C48007810B14020BDE8F0813F2D01D16B
:1064B0003E20F9E7FDF784FB0746FF2D03D1414855
:1064C000006890F836503E4850F8254024B93846C8
:1064D000FDF77AFB4320E7E7012C04D13846FDF7AE
:1064E00073FB3D20E0E714F8380F3749085C61780A
:1064F00088432178344A505414F838091146085C0E
:1065000030B994F83A103148007888432F49087020
:10651000E06918B12046E169FEF719FB206A18B15D
:106520002046216AFDF747FEA66A16B13046FEF7FF
:1065300018FD0020206384F8340084F835002648D4
:106540000078FF2804D224480078401C22490870B3
:106550003846FDF739FBFEF7F9FAFDF731FB074640
:106560001D48007820B11C480078401E1A49087068
:106570002046FDF798FB19480078401E174908701F
:1065800000200F4941F82500A06930B90020616959
:10659000886113496069086005E0D4E90501486134
:1065A000D4E9051088610F48006860610D480460F7
:1065B0000DA020653846FDF707FB0548007815E07B
:1065C000F41600203C0000202E0000202D000020AA
:1065D00036000020290000202A000020370000207B
:1065E00048000020400000203F000000012801D1A9
:1065F000FDF70BFE002057E72DE9F0410446002788
:106600003F2C02D13E20BDE8F081FF2C0BD1FDF7DD
:10661000D7FA0746F948006890F83B603846FDF71E
:10662000D3FA3046EFE7FDF7CBFA0746F44850F8C7
:10663000245025B93846FDF7C7FA4320E3E7012D7A
:1066400004D13846FDF7C0FA3D20DCE73F2085F84D
:106650003B003846FDF7B8FA0020D4E72DE9F047B3
:1066600006460F4614464FF00008E648007820B171
:10667000112020700020BDE8F087FDF7A1FA8046C8
:10668000FF2E03D1DD48006890F83660DC4850F8F2
:10669000265035B94046FDF797FA43202070002078
:1066A000E9E7012D06D14046FDF78EFA4320207020
:1066B0000020E0E7286D38603868FDF717FD814657
:1066C0004046FDF781FA002020704846D3E72DE9C7
:1066D000F04106460F4614464FF00008C9480078BE
:1066E00018B112202070BDE8F081FDF769FA8046EC
:1066F000FF2E03D1C148006890F83660C04850F8BA
:1067000026502DB94046FDF75FFA43202070EAE796
:10671000012D05D14046FDF757FA43202070E2E7EE
:106720002F654046FDF750FA0020207000BFDAE7E1
:1067300070B505460026FDF743FA0646B04850F806
:10674000254024B93046FDF73FFA462070BD012CA4
:1067500004D13046FDF738FA4320F7E794F83400C7
:1067600000F0080060B314F8340F00F0F700207058
:1067700014F83409F8B9206BC8B93834A078A249A4
:1067800009780843A04908702078A049085C61781E
:10679000084314F838199D4A50543046FDF714FA4E
:1067A0009B480078012809D1FDF72FFD06E030460F
:1067B000FDF70AFA02E03046FDF706FA0020C5E7C9
:1067C0003046FDF701FA4420C0E72DE9F0470746BF
:1067D0000D464FF0000A002028606860FDF7F0F9D0
:1067E0008246FF2F03D18548006890F836708448B0
:1067F00050F827402CB95046FDF7E6F94320BDE894
:10680000F087012C04D15046FDF7DEF94320F6E76E
:10681000207C00F0010020B95046FDF7D5F9452055
:10682000EDE70026D4F80C90D4F808805046FDF728
:10683000CBF900E0761C58F8041B0029FAD02E6032
:10684000A9EB060068600020D9E72DE9F041054674
:106850004FF00008FDF7B4F98046FF2D05D16748D9
:10686000006890F83650012608E06448006890F807
:106870003600A84201D1012600E00026604850F809
:1068800025402CB94046FDF79FF94820BDE8F0812E
:10689000012C04D14046FDF797F94320F6E794F820
:1068A00038705A48C05D94F8391088435749C85524
:1068B0000846C05D30B994F83A10534800788843D0
:1068C0005149087094F8340040F0080084F834000E
:1068D0004046FDF779F9012E01D1FDF796FC002025
:1068E000D4E72DE9F04105460E460027FDF768F98B
:1068F0000746FF2D03D14148006890F836504048C4
:1069000050F825402CB93846FDF75EF92920BDE83E
:10691000F081012C04D13846FDF756F94320F6E703
:10692000582221463046FEF7AFF93846FDF74CF9BC
:106930000020ECE72DE9F04704460E4617464FF0DD
:106940000009FDF73DF98146FF2C02D12B4805686F
:1069500002E02B4850F8245005F1540050F82680EE
:106960004846FDF731F9002038704046BDE8F08711
:1069700070B504460026FDF723F906462548007841
:1069800030B1962020703046FDF71EF9012070BD11
:10699000204805780078401C1E4908703046FDF7F5
:1069A00013F9002020702846F1E72DE9F04704464E
:1069B0000E46174698464FF00009FDF701F981464B
:1069C000FF2C02D10D48056802E00D4850F8245014
:1069D00005F1540040F826704846FDF7F5F8002010
:1069E00088F80000BDE8F08710B504480068FDF79E
:1069F00064F9FF20FFF750FD10BD00003C000020AF
:106A0000F4160020290000202D0000202E00002078
:106A1000360000205800002070B505460026634867
:106A2000007800B170BD6248007800B1FAE71DB38C
:106A3000FDF7C6F806465F48006890F838405E48A3
:106A4000005D5C49096891F8391088435A49085536
:106A50000846005D40B95748006890F83A1057481A
:106A600000788843554908705248006805633046ED
:106A7000FDF7AAF8FDF7C9FB00BFD3E72DE9F04108
:106A800005460E4617461C464848007810B155206A
:106A9000BDE8F0814648007808B13220F8E74FF4AD
:106AA0007A7060434FF47A71B0FBF1F14FF461609A
:106AB0006843C6EB061200EB8200384400EB40024C
:106AC000C2EBC01001EBC0084046FFF7A5FF002055
:106AD000DEE770B5054600263F2D01D32A2070BDA4
:106AE000FDF76EF80646364850F8254024B9304682
:106AF000FDF76AF84320F2E7012C04D13046FDF798
:106B000063F84320EBE7206B20B93046FDF75CF8D3
:106B10005020E4E70020206394F8340000F03700B0
:106B200040B114F8340F20F037002070012060705D
:106B3000343C02E0002084F8350094F8340000F082
:106B40000800A8B93834A0781C49097808431B49C3
:106B5000087020781849085C6178084314F83819DF
:106B6000154A50543046FDF72FF8FDF74EFB02E072
:106B70003046FDF729F80020B1E770B50025FDF794
:106B80001FF805460F4804682846FDF71DF8204603
:106B900070BD70B504460025FDF712F8054609489A
:106BA00004602846FDF710F870BD000029000020A1
:106BB0002A0000203C0000202E0000202D00002094
:106BC000F41600205C000020F848006808B9002096
:106BD0007047F6480168F54AC86810600020C86030
:106BE0000861F3480088401CF14A1080F148008891
:106BF000401EF04A10800846EAE72DE9F05F06469D
:106C00000F4690469946DDE90ABA0C9DEA4800789D
:106C100020B18B2028700020BDE8F09FFDF766FEB4
:106C2000FFF7D2FF04462CB9FDF7C4FE862028707A
:106C30000020F1E7012084F82500A661E76184F8CF
:106C40002480C4F80490C4F808B0BAF1000F02D14F
:106C5000DAA0206201E0C4F820A0FDF7ABFE00201E
:106C600028702046D8E7002180F8251080F82410ED
:106C7000C161416141608160D0A101620021016177
:106C8000CA490968C160C9490860C9490988491EDB
:106C9000C74A1180C7490988491CC64A11807047F4
:106CA00030B5057D05F00704C54D05EBC4031D682F
:106CB000854205D1C168196039B100250D6104E034
:106CC0000169C268CA6002B11161012580F82550CE
:106CD0000025C56005619D886D1E9D8030BD70B525
:106CE00005460C462878642803D0892020700020AF
:106CF00070BDB148007818B18B2020700020F7E7F4
:106D0000FDF7F4FD95F82500D8B101280FD0022831
:106D10000ED003281BD12846FFF7C2FF2846FFF7F5
:106D2000A2FFFDF747FE002020700120E0E700BF32
:106D30002846FFF798FFFDF73DFE00202070012058
:106D4000D6E7FDF737FE872020700020D0E7FDF75B
:106D500031FE8D2020700020CAE72DE9F041054664
:106D60000E4614462878642804D08920207000201C
:106D7000BDE8F0819048007818B111202070002003
:106D8000F6E7FDF7B3FD95F8250098B1012804D08A
:106D9000022803D0032813D100BF00BF286A306047
:106DA0003068FDF7A3F90746FDF704FE00202070C8
:106DB0003846DDE7FDF7FEFD872020700020D7E78D
:106DC000FDF7F8FD8D2020700020D1E770B5044656
:106DD0000D462078642803D089202870002070BDDB
:106DE0007548007818B18B2028700020F7E7FDF770
:106DF0007DFD94F8250070B301280DD0022825D020
:106E000003282FD16F4960690968461AFDF7D2FD42
:106E1000002028703046E2E794F8240001280CD0C6
:106E2000022809D1A06908B9E66900E0A669FDF762
:106E3000C1FD0020287006E000BFA669FDF7BAFD7D
:106E40000020287000BF00BF3046C8E7FDF7B2FD44
:106E500000202870C3E7FFE7FDF7ACFD872028700E
:106E60000020BCE7FDF7A6FD8D2028700020B6E7C6
:106E700070B505460C462878642803D08920207018
:106E8000002070BD4C48007818B18B202070002085
:106E9000F7E7FDF72BFD95F8256036B1012E05D0FB
:106EA000022E04D0032E06D102E000BF00BF00BFB7
:106EB0000020207002E08D20207000BF00BFFDF791
:106EC00079FD3046DDE770B50B46032580F8255087
:106ED000012B05D13B4EC5693668354445610CE050
:106EE00085692DB9374EC56936683544456104E07A
:106EF000344E8569366835444561057D05F00704E3
:106F00002F4D05EBC4010D682DB908600025C56043
:106F100001258D8006E00A680860C26010618D88D6
:106F20006D1C8D800025056170BD70B505460C4651
:106F30002878642803D089202070002070BD1E4866
:106F4000007818B18B2020700020F7E7FDF7CEFC09
:106F500095F82500E8B1012810D002280FD00328A9
:106F60001DD12846FFF79CFE00212846FFF7ABFF06
:106F7000FDF720FD002020700120DFE700BF002189
:106F80002846FFF7A0FFFDF715FD00202070012027
:106F9000D4E7FDF70FFD872020700020CEE7FDF736
:106FA00009FD8D2020700020C8E70000700000203F
:106FB0006200002060000020290000203F00000047
:106FC00034300020640000202DE9F04105460F46D2
:106FD00090461C462878642804D089202070002020
:106FE000BDE8F0817D48007818B18B20207000202A
:106FF000F6E7FDF77BFC95F82500002832D0012844
:107000002AD0022827D0032832D12846FFF748FE8D
:1070100000202070B7B1032F02D0042F13D108E055
:107020006E681EB12846A968B04701E08F20207025
:107030000CE06E681EB141462846B04701E08F2043
:10704000207003E002E08420207000BF00BFFDF745
:10705000B1FC0120C4E700BFFDF7ACFC8E2020701E
:107060000120BDE7FDF7A6FC872020700020B7E7D0
:10707000FDF7A0FC8D2020700020B1E710B5584826
:107080000068FFF719F80446204610BD08B500BF98
:1070900000BF6A46002152480068FEF75BFFFDF71B
:1070A00025FC50480068401C4E490860084600789E
:1070B00000F007084C4800EBC8073C681AE0E66897
:1070C000484960690968884213D12046FFF7E8FD06
:1070D00094F82400022804D101212046FFF7F3FE92
:1070E00002E0022084F82500656815B12046A168F9
:1070F000A8473446002CE2D1FDF75CFCC9E700B597
:1071000087B0032000218022384BCDE90132CDE940
:1071100003104FF6FD703D23354A00903548FFF7C8
:1071200066F906AA34A13D20FFF7D1FA07B000BDE9
:10713000F8B54FF420713448FDF7D8FA40212A48B9
:10714000FDF7D4FA002515E0681C86B205EB850032
:107150002D4901EBC00406EB860001EBC00764205B
:107160002070002084F82500E760AFF2B0102062A4
:10717000681C85B20F2DE7D305EB8500224901EB92
:10718000C00464202070002084F82500E060AFF285
:10719000D41020620020134908601C490880102088
:1071A0001B49088018481B4908600120FEF745FE6E
:1071B000194908600020FEF740FE094908606A4648
:1071C00016A115480068FCF7CCFF6A4618A10448D0
:1071D0000068FCF7C6FFFFF792FFF8BD290000200A
:1071E0006C0000206400002034300020342E002089
:1071F000303000208D70000075432F4F532D4949CA
:1072000020546D7200000000B42B002062000020AA
:1072100060000020700000206800002075432F4FA0
:10722000532D494920546D724C6F636B0000000070
:1072300075432F4F532D494920546D725369676E22
:10724000616C00000146412903DB5A2901DC01225F
:1072500000E00022012A08D0612903DB7A2901DC41
:10726000012200E00022012A01D1012200E00022D7
:10727000104670470146412903DB5A2901DC0122EF
:1072800000E00022012A08D0612903DB7A2901DC11
:10729000012200E00022012A01D1012200E00022A7
:1072A000012A08D0302903DB392901DC012200E062
:1072B0000022012A01D1012200E00022104670477D
:1072C0000146612903DB7A2901DC012200E000226A
:1072D000104670470146412903DB5A2901DC01228F
:1072E00000E00022104670470146302903DB3929AF
:1072F00001DC012200E000221046704701463029DF
:1073000003DB372901DC012200E000221046704730
:107310000146302901DB392907DD412901DB4629F6
:1073200003DD612903DB662901DC012200E0002284
:10733000104670470146202901D0092901D10122B8
:1073400000E00022104670470146202909D00D298F
:1073500007D00A2905D00C2903D0092901D00B290F
:1073600001D1012200E00022104670470146202989
:1073700003DB7E2901DC012200E000221046704779
:107380000146212903DB7E2901DC012200E00022E5
:10739000104670470146202903DB7E2901DC0122CB
:1073A00000E00022012A35D1202909D00D2907D07B
:1073B0000A2905D00C2903D0092901D00B2901D1B4
:1073C000012200E000222ABB412903DB5A2901DC0B
:1073D000012200E00022012A08D0612903DB7A297A
:1073E00001DC012200E00022012A01D1012200E09B
:1073F0000022012A08D0302903DB392901DC0122CF
:1074000000E00022012A01D1012200E000220AB995
:10741000012200E000221046704701464AB2002ACD
:1074200001DB1F2901DD7F2901D1012200E00022BB
:10743000104670470146412903DB5A2901DC01222D
:1074400000E00022012A02D101F1200200E00A46F8
:10745000D0B270470146612903DB7A2901DC0122A1
:1074600000E00022012A02D1A1F1200200E00A4638
:10747000D0B27047F0B504460B462046FFF7EAFF4E
:1074800005461846FFF7E6FF0646B54201D1012042
:1074900000E0002007463846F0BD0000FD48FE49E8
:1074A00001600146416000218160C160016141616C
:1074B0008161C16101620163C1624162F749816317
:1074C000C1634FF48061016441640146F44A116074
:1074D00070472DE9F04103460C4617460FB9BDE849
:1074E000F08103B9FBE70025002202E02D022543CD
:1074F000521C042AFAD3384603F0030C1946BCF197
:10750000000F08D0624603E001F8014B401E521CF8
:1075100008B1042AF8D30E4601E020C6001F042853
:10752000FBD2314602E001F8014B401E0028FAD19F
:1075300000BFD4E730B505460C4622460021284658
:10754000FFF7C7FF30BD2DE9F04F85B007468846ED
:107550009146B9F1000F02D105B0BDE8F08F07B92F
:10756000FAE7B8F1000F00D1F6E746463D46AE42D5
:1075700005D94A464146384601F088FBECE74C46BF
:107580003819451E08EB0400461EA81B04900498F9
:10759000042834D305F00300029006F003010191A2
:1075A000DDE90110884201D1012000E000200090B7
:1075B0000098012823D10298032810D0029840B2E5
:1075C000039008E016F8010905F80109641E039804
:1075D000401E40B2039014B103980028F2DAA5F1DE
:1075E000030AA6F1030B04E05BF804094AF8040956
:1075F000241F042CF8D20AF103050BF1030604E062
:1076000016F8010905F80109641E002CF8D100BF25
:10761000A2E72DE9F84F80468946154615B90120A5
:10762000BDE8F88FB8F1000F01D10020F8E7B9F1FB
:10763000000F01D10020F3E70124294608EB0502E1
:1076400009EB050302F0030C03F0030BDC4501D149
:10765000012000E0002000900098012829D1BCF111
:10766000000F12D0E2460AE0521E5B1E107893F81B
:1076700000E0704500D00024491EAAF1010A012C47
:1076800003D111B1BAF1000FEED1012C11D1164680
:107690001F4608E0361F3F1F3068D7F800E07045EE
:1076A00000D00024091F012C01D10429F2D2324656
:1076B0003B4608E0521E5B1E107893F800E07045D0
:1076C00000D00024491E012C01D10029F2D120460E
:1076D000A6E7F0B503460D461646DA6BB2FBF6F0A8
:1076E00006FB102CBCF1000F02D0A6EB0C0400E04E
:1076F00000246119586C884201D20020F0BDA142DB
:1077000001D3A94201D20020F8E75718974201D2CD
:107710000020F3E72244DF63586C401A5864104697
:10772000ECE72DE9F04F81468C461C46B9FBF4F09E
:1077300004FB109BBBF1000F02D0A4EB0B0600E092
:107740000026B2FBF4F004FB102BBBF1000F02D0BB
:10775000A4EB0B0300E00023D018ACF1010E00FBFA
:107760000E60871806EB0208B04501D3904502D29F
:107770000020BDE8F08FBCF1010F22D9D5189D4241
:1077800001D3954201D20020F3E7ACF1010000FBE8
:1077900005F1A94203D3994201D3914201D20020BD
:1077A000E7E701EB020A8A4501D3924501D20020A6
:1077B000DFE7474503D38F4201D3574501D200206D
:1077C000D7E73846D5E72DE9FE4F074688461546E8
:1077D0001C46002000901CB900BF01F08DFB00BFCB
:1077E0000DB901AD00BF002028602FB942F27470BE
:1077F00020800020BDE8FE8FB8F1000F04D142F2D6
:10780000757020800020F5E7DFF8889000BF00BF8A
:1078100001F0A4FC009000BF00BFD9F83C0002902A
:10782000D9F844B043463A4601210298FFF779FF60
:10783000064666B900BF00BF009801F093FC00BF88
:1078400000BF2F6042F2E37020800020D2E75E4547
:107850000ED900BF00BF009801F084FC00BF00BF3C
:10786000A6EB0B00286042F2E27020800020C1E706
:10787000424639464846FFF72CFF8246BAF1000FD0
:1078800015D100BF00BF009801F06CFC00BF00BF25
:107890002E6007E07430002048454150BC30002085
:1078A0007400002042F2E27020800020A2E700BFB6
:1078B00000BF009801F056FC00BF00BF42F21070FC
:1078C0002080504696E72DE9FC5F06460D4614469B
:1078D000002000901CB900BF01F00EFB00BF2DB9C5
:1078E00042F2757020800020BDE8FC9FB5F5805FF6
:1078F00004D942F2757020800020F5E726B942F2E3
:10790000117020800020EFE700BF00BF01F026FCCF
:10791000009000BF00BFFE493068084440B1FD49F7
:10792000084418B1FC49084408B900BF0CE000BF86
:1079300000BF00BF009801F015FC00BF00BF42F27D
:10794000887020800020CFE700BFD6F80490D9F8D7
:10795000380008B1484600E0F0488246DAF8447042
:10796000DAF83CB000BF00BF009801F0FBFB00BF9D
:1079700000BF012D0DD9BBFBF5F005FB10B8B8F128
:10798000000F02D0A5EB080000E000200190019854
:107990003F1A42F2107020803846A5E770B50446C1
:1079A0000D462A462146DD48FFF78DFF0646304644
:1079B00070BD70B504460D461DB900BF01F09CFABC
:1079C00000BF1CB942F21170288070BDD0484042FF
:1079D000206000206060A060E06020616061A061C4
:1079E000E0612062A06260632063E0626062A06385
:1079F000E0632064606442F21070288000BFE4E716
:107A00002DE9FF4F91B00446DDE92095002000905C
:107A10001DB900BF01F070FA00BFB9F1000F02D12B
:107A20000DF1100900BF0020C9F8000029462046CA
:107A3000FFF7BFFF288842F21071884202D015B0CC
:107A4000BDE8F08F129828B1139818B942F27E70F1
:107A50002880F4E7149818B942F292702880EEE773
:107A60001E9818B942F293702880E8E71F9818B959
:107A700042F294702880E2E7A948006818B942F2FF
:107A8000E7702880DBE7A54810904FF0000A00BFA0
:107A900000BF01F063FB009000BF00BF12980028F8
:107AA0005BD1109E109E0E96109E3746109EF06B76
:107AB0000B9004231A4614990B98FFF732FE03909B
:107AC000039850B900BF00BF009801F04BFB00BF06
:107AD00000BF42F2E3702880B1E703990B98084495
:107AE0000A90DDE91E2314990A98FFF71AFE8346CF
:107AF000BBF1000F0AD100BF00BF009801F032FBBC
:107B000000BF00BF42F2E370288098E7039800EBC3
:107B10000B0A0398824501D3DA450AD200BF00BFA1
:107B2000009801F01FFB00BF00BF42F2E370288005
:107B300085E71098D0F84480C2457DD900BF00BFCA
:107B4000009801F00FFB00BF00BFAAEB0800C9F8C6
:107B5000000042F2E270288071E712980990DDE996
:107B600012010844401E0890DDE9081081420AD243
:107B700000BF00BF009801F0F5FA00BF00BF42F25D
:107B8000977028805BE7002600200E906448076805
:107B90003AE0B96B1298814205D1396C1398814251
:107BA00001D13E4632E0B86B0790396CB86B08449F
:107BB000401E0690DDE90701814200D226E00799C8
:107BC0000998884203D8DDE9071088420FD2079947
:107BD0000998884203D306990898884207D90699DC
:107BE000099888420ED80699089888420AD300BF9F
:107BF00000BF009801F0B6FA00BF00BF42F27F70EC
:107C000028801CE70E97FF68002FC2D100BF46B93D
:107C100026461298A0631298E06313982064139884
:107C200060641098C06B0B9004231A4614990B984B
:107C3000FFF777FD039000E04CE0039850B900BFD8
:107C400000BF009801F08EFA00BF00BF42F2E3705F
:107C50002880F4E61098D0F84480039840450FD966
:107C600000BF00BF009801F07DFA00BF00BF03987D
:107C7000A0EB0800C9F8000042F2E2702880DEE6BE
:107C8000F06B0A90DDE91E2314990A98FFF749FD6D
:107C90008346BBF1000F0AD100BF00BF009801F07E
:107CA00061FA00BF00BF42F2D9702880C7E6D6F85B
:107CB0004480C3450ED900BF00BF009801F052FABE
:107CC00000BF00BFABEB0800C9F8000042F2D8705B
:107CD0002880B4E61498800002900422029910983B
:107CE000FFF7F7FC0D900D9878BB1098D0F8448002
:107CF00000BF00BF009801F035FA00BF00BF129826
:107D000098B9C2450ED9AAEB0800C9F8000018E0DE
:107D1000B2B0B1BAFEFFFEF8080A0EFC74300020C3
:107D200074000020C9F800A00BE00298404505D976
:107D30000298A0EB0800C9F8000002E00298C9F818
:107D4000000042F2E270288079E6FFE7002001900F
:107D500032E03046DDE91E12FFF7BBFC0C900C98B8
:107D600010BBF06B0A90D6F8448000BF00BF0098AB
:107D700001F0F8F900BF00BF01991498401A05906E
:107D8000DDE91E2305990A98FFF7CBFC8246C24520
:107D900004D9AAEB0800C9F8000001E0C9F800A066
:107DA00042F2D87028804AE6019ADDE90C0141F8D8
:107DB00022000198401C0190149901988842C8D370
:107DC000A6420CD10E98A060E7600E9810B10E98F4
:107DD000C46001E0FE4804605FB1BC6009E0706906
:107DE0000F9026610F98606174610F9808B10F9829
:107DF0000461F848206066600A98A0610A985844B7
:107E0000401EE0610D982062C4F828B01F9860639E
:107E10001E9820631498E0621498606200BF00BF4F
:107E2000009801F09FF900BF00BF42F21070288057
:107E300000BF04E62DE9F04105460C4600271CB9B9
:107E400000BF01F059F800BF2DB942F21170208037
:107E50000020BDE8F08100BF00BF01F07FF90746B8
:107E600000BF00BFDC492868084440B1DB49084432
:107E700018B1DB49084408B902E00DE000BF00BFBB
:107E800000BF00BF384601F06DF900BF00BF42F2ED
:107E9000887020800020DCE700BF6E6A00BF00BF52
:107EA000384601F05FF900BF00BF42F21070208039
:107EB0003046CEE72DE9F04104460E4615464FF018
:107EC00000081DB900BF01F017F800BF2CB942F23D
:107ED000117028800020BDE8F08126B942F293702D
:107EE00028800020F7E700BF00BF01F037F9804687
:107EF00000BF00BFB749206888420BD000BF00BF59
:107F0000404601F02FF900BF00BF42F28870288080
:107F10000020E0E7206BB0420BD200BF00BF40461C
:107F200001F020F900BF00BF42F2937028800020CA
:107F3000D1E7606A58B900BF00BF404601F012F9AE
:107F400000BF00BF42F2DE7028800020C3E7E16A74
:107F5000606A88420BD900BF00BF404601F002F9B9
:107F600000BF00BF42F2957028800020B3E7606A2E
:107F7000401E6062D4E9080150F8217000BF00BFC4
:107F8000404601F0EFF800BF00BF42F210702880B9
:107F90003846A0E72DE9F04704460F4615464FF056
:107FA00000091DB900BF00F0A7FF00BF2CB942F2C5
:107FB000117028800020BDE8F08700BF00BF01F0ED
:107FC000CDF8814600BF00BF8249206888420BD0AF
:107FD00000BF00BF484601F0C5F800BF00BF42F235
:107FE000887028800020E6E7E16A606A88420BD347
:107FF00000BF00BF484601F0B5F800BF00BF42F225
:10800000957028800020D6E7E06AC01B461EE06A13
:10801000B0420BD800BF00BF484601F0A3F800BF34
:1080200000BF42F2957028800020C4E7606AB04229
:108030000BD900BF00BF484601F094F800BF00BF55
:1080400042F2957028800020B5E7206A50F826801B
:1080500000BF00BF484601F085F800BF00BF42F2F4
:10806000107028804046A6E72DE9F04F02460C46E6
:108070009569D2F81CB0AC4201D35C4502D900200E
:10808000BDE8F08F536BB5FBF3F003FB105111B15A
:10809000A3EB010C01E04FF0000C176BB7FBF3F002
:1080A00003FB107109B15E1A00E0002605EB0C0815
:1080B000A4EB080A07EB0609BAFBF9F009FB10A0CC
:1080C00008B9012000E0002086467046D8E72DE977
:1080D000F04704460F4615464FF0000A1DB900BF91
:1080E00000F00AFF00BF24B942F211702880BDE8F9
:1080F000F0871FB942F211702880F8E700BF00BF77
:1081000001F02CF8824600BF00BF32492068884247
:108110000AD000BF00BF504601F024F800BF00BFE6
:1081200042F288702880E2E739462046FFF79CFF3C
:108130008046B8F1010F0AD000BF00BF504601F0E1
:1081400011F800BF00BF42F297702880CFE70026E9
:1081500010E0206A50F82600B8420AD100BF00BFE4
:10816000504600F0FFFF00BF00BF42F29870288029
:10817000BDE7761C606AB042EBD8E16A606A88426B
:108180000AD300BF00BF504600F0ECFF00BF00BFA5
:1081900042F2DD702880AAE74FF00008666A08E026
:1081A000206A50F82690B94502D14FF0010803E04B
:1081B000761CE06AB042F3D800BFB8F1010F11D1CC
:1081C000D4E9080150F82100216A41F8260014E0A2
:1081D00074000020504F4F4CB2B0B1BAFEFFFEF811
:1081E000080A0EFC00BF00BF504600F0BBFF00BFF6
:1081F00000BF42F28870288079E7D4E9080140F88E
:108200002170606A401C606200BF00BF504600F0F1
:10821000A9FF00BF00BF42F21070288000BF66E7D0
:108220002DE9F84F04460F461546002000904FF008
:10823000FF3B1DB900BF00F05FFE00BF2CB942F24A
:10824000117028805846BDE8F88F27B942F21170A6
:1082500028805846F7E700BF00BF00F07FFF00907E
:1082600000BF00BF3D49206888420BD000BF00BF5F
:10827000009800F077FF00BF00BF42F288702880AE
:108280005846E0E739462046FFF7EEFE8046B8F153
:10829000010F0BD000BF00BF009800F063FF00BFCC
:1082A00000BF42F2977028805846CCE7002611E0C4
:1082B000206A50F82600B8420BD100BF00BF0098DA
:1082C00000F050FF00BF00BF42F29870288058466F
:1082D000B9E7761C606AB042EAD8E16A606A88420F
:1082E0000BD300BF00BF009800F03CFF00BF00BFF1
:1082F00042F2DD7028805846A5E74FF00008666A14
:1083000008E0206A50F82690B94502D14FF00108E4
:1083100003E0761CE06AB042F3D800BFB8F1010F69
:108320000FD1E06A401EA0EB060A00BF00BF009814
:1083300000F018FF00BF00BF42F2107028805046C6
:1083400081E700BF00BF009800F00CFF00BF00BF36
:1083500042F288702880584675E70000504F4F4C15
:1083600010B502460B461146002001E0491C401C96
:1083700019B10C780CB19842F8D310BD30B5044651
:108380004FF0FF312046FFF7EBFF0546284630BD92
:1083900070B504460D4616460CB9002070BD0DB9E7
:1083A0000020FBE721462A46002304E010780870ED
:1083B000491C521C5B1C21B11AB1107808B1B342A0
:1083C000F4D301B10AB90020E8E7B34201D200209A
:1083D00008702046E2E770B504460D464FF0FF32C4
:1083E00029462046FFF7D4FF0646304670BD70B5DB
:1083F00003460C4615460BB9002070BD0CB9002091
:10840000FBE70DB91846F8E7194600E0491C11B121
:1084100008780028FAD109B90020EEE722460026A4
:1084200004E010780870491C521C761C21B11AB166
:10843000107808B1AE42F4D301B10AB90020DCE7EC
:10844000002008701846D8E770B504460D464FF076
:10845000FF3229462046FFF7CAFF0646304670BD68
:108460002DE9F04305460B469446BCF1000F02D1BE
:108470000020BDE8F08335B90BB90020F9E7187882
:1084800042421046F5E713B92A781046F1E729462B
:108490001C460F4626467F1C761C4FF0000805E060
:1084A000491C641C7F1C761C08F10108087894F8AC
:1084B0000090484505D1087818B117B10EB1E045D4
:1084C000EED3E04501D10020D3E7087894F800907E
:1084D000484505D0087894F80090A0EB09020BE01D
:1084E000087808B9002207E02FB90EB9002203E08E
:1084F0003078424200E03A781046BAE770B5044658
:108500000D464FF0FF3229462046FFF7A9FF0646E9
:10851000304670BD2DE9F74F82B080460E46049874
:1085200018B9002005B0BDE8F08FB8F1000F09D1EF
:108530000EB90020F6E73078FEF77CFF07467C4254
:108540002046EFE73EB998F80000FEF773FF0546B6
:108550002C462046E6E7C146B246C846C3465646C4
:10856000CDF804A0D8460BF1010B019E701C0190C0
:10857000C84699F80000FEF75DFF054656469AF892
:108580000000FEF757FF07460020009015E009F1B4
:1085900001090AF1010A0BF1010B0198401C01903D
:1085A0000098401C009099F80000FEF743FF054634
:1085B0009AF80000FEF73EFF0746BD420BD199F83E
:1085C000000040B1BBF1000F05D0019818B104992B
:1085D00000988842DBD304990098884201D100209A
:1085E000A0E7BD4201D0EC1B16E00DB9002413E05A
:1085F000BBF1000F0AD1019808B900240CE00199E1
:108600000878FEF717FF07467C4205E09BF800005C
:10861000FEF710FF05462C46204683E770B504465A
:108620000D464FF0FF3229462046FFF773FF0646FE
:10863000304670BD30B504460B4615460CB90020D7
:1086400030BD0BB90020FBE72146002201E0491CA8
:10865000521C31B1087820B10878A84201D09A4262
:10866000F5D309B90020EBE79A4201D30020E7E7F0
:108670000878A84201D00020E2E70846E0E770B59C
:1086800005460C4622464FF0FF312846FFF7D2FF41
:108690000646304670BD2DE9F04305460E461746A6
:1086A00015B90020BDE8F0830EB90020FAE72C468A
:1086B000A6F1010949462046FFF752FE8046444490
:1086C0000CB90020EEE700E0641EAC4202D0207836
:1086D000B842F9D12078B84201D00020E2E7204624
:1086E000E0E770B505460C4622464FF0FF312846BC
:1086F000FFF7D1FF0646304670BD70B504460D4603
:1087000016460CB9002070BD0BB90020FBE72146CE
:108710001A4605E00878A84200D10E70491C521E86
:1087200019B1087808B1002AF4D12046EBE7F0B57A
:1087300004460D4616464FF0FF3332462946204682
:10874000FFF7DBFF07463846F0BD2DE9FF4F064631
:108750000F4615461EB9002004B0BDE8F08F0FB9D2
:108760000020F9E70DB90020F6E7681C00B101E030
:108770004FF0FF30039029463046FFF7F1FD804669
:1087800038460399FFF7ECFD04460CB93046E3E7A1
:10879000444501D90020DFE706EB080BBBF1000FD1
:1087A00001D10020D8E707EB040BBBF1000F01D18A
:1087B0000020D1E7A8EB040002904FF00009002050
:1087C000019000BF06EB0900009022463946009850
:1087D000FFF746FE8246BAF1000F01D1012000E00A
:1087E0000020019009F10109019810B90298814512
:1087F000E8D9BAF1000F01D00020ADE70098ABE74F
:1088000070B504460D464FF0FF3229462046FFF76B
:108810009CFF0646304670BD2DE9FF4F8DB00F46D8
:1088200015461A9E1D9818B9002011B0BDE8F08FAA
:10883000002003900490012F01DA01200390022D03
:1088400001D3242D01D90120039096B33046FEF7C1
:108850008DFD02900298012802D00120039028E0AB
:10886000302E26D0A6F13000C0B207901B98012808
:1088700004D0A6F14100C0B2069003E0A6F1610069
:10888000C0B206900A2D02D80798A84209DB0A2D2B
:1088900009D907980A2804D3A5F10A000699884245
:1088A00001D9012000E0002005900598012800D1A1
:1088B00003901D9C0398002846D1DDF834A0DDF814
:1088C00034A0CDF830A001200B9007E00B98401C9D
:1088D000C0B20B900C98B0FBF5F00C900C98A8422D
:1088E000F4D21098012800D100E0002009900B99E3
:1088F00009980844B84225DC002001900B98B84242
:1089000001DA0B9800E038460A903EB1B8460A9862
:10891000391A0998081AC0B2089006E0DDE9091072
:10892000084400F0FF08002008900898002806DDA1
:10893000302E01D1012000E00020049004E000204E
:10894000049001E001200390039800B1B84644442C
:108950001C9808B100202070641E4FF0000941E00F
:108960000398A8BBBAF1000F02D1B9F1000F1CD1D6
:10897000BAFBF5F005FB10A000F0FF0BBBF10A0FEE
:1089800004D20BF1300004F801090BE01B98012818
:1089900004D00BF1370004F8010903E00BF1570094
:1089A00004F80109BAFBF5FA1AE01098012810D171
:1089B000049808B9019828B1049850B1A8F10100B1
:1089C000484506D12D2004F801090120019007E057
:1089D00003E02EB104F8016902E03F2004F8010928
:1089E00009F10109C145BBD3039808B100201CE778
:1089F0001D981AE72DE9FF5F05460E4617461C46EF
:108A0000DDE90F9ADDF8388000233A4631462846E2
:108A10008DE81007FFF700FF8346584604B0BDE815
:108A2000F09F2DE9FF4F85B0044689461F46DDE9DA
:108A300013AB002C02DA6542012601E02546002630
:108A400012983346CDE902ABCDE90070494628467D
:108A5000079AFFF7E1FE8046404609B0BDE8F08F77
:108A60002DE9FF4F8BB0064689461546B9F1000F38
:108A700002D10DF1240900BFC9F80060189810B99F
:108A800007A8189000BF0021189801701EB9002097
:108A90000FB0BDE8F08F012D01D0242D01D90020A9
:108AA000F6E734462078FEF74FFC039004E0641CA0
:108AB0002078FEF749FC039003980128F7D020782E
:108AC0002B2802D02D280BD103E0641C4FF0000BA3
:108AD00009E00E98012800D1641C4FF0010B02E060
:108AE0004FF0000B00BF00BF0A9425B1082D1CD029
:108AF000102D36D11EE02078302814D1641C207847
:108B0000582802D078280BD100BF10256778384646
:108B1000FEF7FEFB8246BAF1010F00D1641C01E0B2
:108B2000082500BF00E00A251CE02078302800D18D
:108B3000641C17E02078302812D1641C2078582853
:108B400002D078280AD100BF67783846FEF7E0FBEC
:108B50008246BAF1010F00D1641C00E000BF00BFE3
:108B600000E000BF00BF4FF000080020029001901D
:108B700040E027783846FEF77DFB059005980128F0
:108B800036D13846FEF7B0FB06900698012804D18E
:108B9000A7F13000C0B208900FE03846FEF790FB16
:108BA00004900498012804D1A7F15700C0B208909E
:108BB00003E0A7F13700C0B208900898A84214DA81
:108BC000029880B9304850F82500404509D308FB89
:108BD00005F8089880440898804504D20120029046
:108BE00001E001200290641C04E00120019001E0FA
:108BF0000120019001980028BBD00298012801D1E2
:108C00004FF0FF380A98844202D0C9F8004001E0D2
:108C1000C9F80060189880F800B0404638E7F8B509
:108C200004460D461646002003463246294600906B
:108C30002046FFF715FF07463846F8BD2DE9FC41F1
:108C400005460E46174601A801233A4631460090D4
:108C50002846FFF705FF04469DF8040040B9B4F12B
:108C6000004F02D36FF0004000E02046804607E04E
:108C7000B4F1004F02D34FF0004000E06042804664
:108C80004046BDE8FC81000014BC0200002800D171
:108C90007047002900D17047002A00D170472DE9A4
:108CA000F81F00F0030301F00304A34211D1C3F144
:108CB000040303F00303012B1DD3012A00D2F2E0C9
:108CC00011F8014B00F8014BA3F10103A2F10102DD
:108CD000F1E700F0010301F00104A34200D094E0A9
:108CE000012B44D311F8014B00F8014BA3F1010310
:108CF000A2F10102F4E7B2F5B47F26D3B1E8F81F80
:108D0000A0E8F81FB1E8F81FA0E8F81FB1E8F81FC5
:108D1000A0E8F81FB1E8F81FA0E8F81FB1E8F81FB5
:108D2000A0E8F81FB1E8F81FA0E8F81FB1E8F81FA5
:108D3000A0E8F81FB1E8F81FA0E8F81FB1E8F81F95
:108D4000A0E8F81FA2F5B472D5E7282A06D3B1E847
:108D5000F81FA0E8F81FA2F12802F6E7042A06D3BC
:108D600051F8043B40F8043BA2F10402F6E7202A44
:108D700042D331F8023B20F8023B31F8023B20F8A5
:108D8000023B31F8023B20F8023B31F8023B20F86D
:108D9000023B31F8023B20F8023B31F8023B20F85D
:108DA000023B31F8023B20F8023B31F8023B20F84D
:108DB000023B31F8023B20F8023B31F8023B20F83D
:108DC000023B31F8023B20F8023B31F8023B20F82D
:108DD000023B31F8023B20F8023B31F8023B20F81D
:108DE000023B31F8023B20F8023B31F8023B20F80D
:108DF000023BA2F12002BAE7022A06D331F8023B75
:108E000020F8023BA2F10202F6E7102A42D311F841
:108E1000013B00F8013B11F8013B00F8013B11F860
:108E2000013B00F8013B11F8013B00F8013B11F850
:108E3000013B00F8013B11F8013B00F8013B11F840
:108E4000013B00F8013B11F8013B00F8013B11F830
:108E5000013B00F8013B11F8013B00F8013B11F820
:108E6000013B00F8013B11F8013B00F8013B11F810
:108E7000013B00F8013B11F8013B00F8013B11F800
:108E8000013B00F8013B11F8013B00F8013BA2F166
:108E90001002BAE7012A06D311F8013B00F8013BA2
:108EA000A2F10102F6E7BDE8F81F704710B50024F3
:108EB00000BF00BF00F052F9044600BF00BF102100
:108EC000A148FEF737FB00BF00BF204600F04AF97B
:108ED00000BF00BF10BD10B5FFF7E8FF10BD10B513
:108EE00000209A49086001F051F810BD10B5FFF755
:108EF000F6FFFFF7F0FF10BD00BFFEE770B50546B7
:108F00000C46002614B900BFFFF7F6FF15B90A207A
:108F1000208070BD00BF00BF00F020F9064600BFF2
:108F200000BF102288492846FFF732FA00BF00BF71
:108F3000304600F017F900BF00BF0020208000BFBE
:108F4000E7E72DE9F04105460C46002714B900BFBC
:108F5000FFF7D2FF1DB90A202080BDE8F081102163
:108F60002846FFF7FDF90646102E15D200BF00BFB8
:108F700000F0F4F8074600BF00BF102229467248EF
:108F8000FFF706FA00BF00BF384600F0EBF800BF5D
:108F900000BF0020208002E04FF47A70208000BFE4
:108FA000DBE710B501F008F80446204610BD704715
:108FB00000B5014611B900BFFFF79EFF634A106874
:108FC00008B1002201E04FF4FA620A8000BD5F4957
:108FD0000860704770B50546284600F0CAF8044698
:108FE000183C204670BD70B50546284600F0C1F813
:108FF0000446103C204670BD70B50546284600F07A
:10900000B8F8044600BF204670BD30B502460B4696
:109010000024D2F1FF359C4126D24FF6FF74D2F1E5
:10902000FF359C410FD26FF07F44D2F1FF359C4158
:1090300003D2190E464C605C44E0190C444C645C4D
:1090400004F108003EE0FF24D2F1FF359C4105D237
:10905000190A3F4C645C04F1100033E019463C4CA3
:10906000645C04F118002DE04FF6FF750024AD1A82
:109070009C4115D26FF07F450024AD1A9C4107D268
:10908000140E44EA0321324C645C04F1200019E020
:10909000140C44EA03412E4C645C04F1280011E0F6
:1090A0000024D2F1FF059C4107D2140A44EA03616F
:1090B000274C645C04F1300004E01146244C645CED
:1090C00004F1380030BD70B504460CB9082070BDFD
:1090D000204600F051F805462846F8E770B50446EA
:1090E0000CB9102070BD204600F046F80546284611
:1090F000F8E770B504460CB9202070BD204600F09A
:109100003BF805462846F8E72DE9F04304460D46AE
:10911000002184EA01006940084302D14020BDE8F3
:10912000F083E243E843521C40F1000102EA0406E6
:1091300001EA050730463946FFF767FF8046C8F168
:109140003F094846EBE70000BC34002078000020CF
:10915000A8BC020072B6704762B67047EFF3108089
:1091600072B6704780F31088704730BF704720BFD9
:109170007047B0FA80F0704790FAA0F0B0FA80F033
:10918000704790FAA0F0704710B5B0F1005F0AD3B5
:10919000FE4CA04207D8440104EB810303F10852BE
:1091A000002414600CE0B0F1804F09D3F84CA042C9
:1091B00006D8440104EB810303F1844200241460C7
:1091C00010BD10B5B0F1005F0AD3F04CA04207D833
:1091D000440104EB810303F10852012414600CE004
:1091E000B0F1804F09D3EA4CA04206D8440104EB09
:1091F000810303F184420124146010BD2DE9F04184
:1092000004464FF00008102C6BD2DFE804F0080E83
:109210000F1014293E090A0B0C11120D135300BF35
:1092200000BF00BF00BF00BF89E000BF00BF00BF9C
:1092300000BF00BF83E000BF00BFFFF78FFF804685
:1092400000BF00BFD348006820F48030D1490860D7
:1092500000BF00BF4046FFF785FF00BF00BF6EE0C4
:1092600000BF00BFFFF77AFF804600BF00BFC948BC
:10927000006820F40030C749086000BF00BF4046C6
:10928000FFF770FF00BF00BF59E000BF00BFFFF74E
:1092900065FF804600BF00BFBE48006820F4802004
:1092A000BC49086000BF00BF4046FFF75BFF00BF3E
:1092B00000BF44E000BF00BFFFF750FF804600BF83
:1092C00000BF4FF0E020006920F001004FF0E021E6
:1092D000086100BF00BF4046FFF744FF00BF00BF6A
:1092E0002DE04FF0E0204068401C102101EB4010C1
:1092F000C6B2B44222DAA4F11000C11700EBD1616A
:10930000C1F34715C11700EBD1614911A0EB411121
:10931000CFB200BF00BFFFF721FF804600BF00BFF4
:109320000120B840A90001F1E021C1F8800100BF8F
:1093300000BF4046FFF716FF00BF00BF00BF00BFE1
:10934000BDE8F0812DE9F04104464FF00008102CF3
:109350006BD2DFE804F0080E0F1014293E090A0B47
:109360000C11120D135300BF00BF00BF00BF00BFA0
:1093700089E000BF00BF00BF00BF00BF83E000BFA7
:1093800000BFFFF7EBFE804600BF00BF81480068CA
:1093900040F480307F49086000BF00BF4046FFF7BF
:1093A000E1FE00BF00BF6EE000BF00BFFFF7D6FECA
:1093B000804600BF00BF7748006840F40030754920
:1093C000086000BF00BF4046FFF7CCFE00BF00BFF3
:1093D00059E000BF00BFFFF7C1FE804600BF00BFDD
:1093E0006C48006840F480206A49086000BF00BFF4
:1093F0004046FFF7B7FE00BF00BF44E000BF00BF1C
:10940000FFF7ACFE804600BF00BF4FF0E0200069D0
:1094100040F001004FF0E021086100BF00BF40466E
:10942000FFF7A0FE00BF00BF2DE04FF0E020406836
:10943000401C102101EB4010C7B2BC4222DAA4F15B
:109440001000C11700EBD161C1F34715C11700EB44
:10945000D1614911A0EB4111CEB200BF00BFFFF7AF
:109460007DFE804600BF00BF0120B040A90001F191
:10947000E021C1F8000100BF00BF4046FFF772FEC7
:1094800000BF00BF00BF00BFBDE8F0812DE9F04183
:1094900004464FF00008102C19D2DFE804F0080E43
:1094A0000F10111516090A0B0C12130D141700BF1B
:1094B00000BF00BF00BF00BF37E000BF00BF00BF5C
:1094C00000BF00BF00BF00BF00BF00BF2DE04FF0D6
:1094D000E0204068401C102101EB4010C7B2BC42A4
:1094E00022DAA4F11000C11700EBD161C1F34715D6
:1094F000C11700EBD1614911A0EB4111CEB200BF01
:1095000000BFFFF72BFE804600BF00BF0120B04028
:10951000A90001F1E021C1F8800200BF00BF404670
:10952000FFF720FE00BF00BF00BF00BFBDE8F08115
:109530002DE9F04706460D464FF0000A102E73D273
:10954000DFE806F0080E0F10112F45090A0B0C5B1F
:10955000730D89A000BF00BF00BF00BF00BFE5E0E2
:1095600000BF00BFE2E000BF00BFFFF7F7FD82468B
:1095700000BF00BF07480C38046824F0FF042C43E8
:10958000046000BF00BF504606E00000FFFF0F2050
:10959000FFFF0F4024ED00E0FFF7E4FD00BF00BF38
:1095A000C4E000BF00BFFFF7D9FD824600BF00BF87
:1095B000CC48046824F47F4444EA0524046000BFD6
:1095C00000BF5046FFF7CEFD00BF00BFAEE000BFBA
:1095D00000BFFFF7C3FD824600BF00BFC14804685B
:1095E00024F47F0444EA0544046000BF00BF5046F1
:1095F000FFF7B8FD00BF00BF98E000BF00BFFFF756
:10960000ADFD824600BF00BFB648001D046824F0CF
:109610007F4444EA0564046000BF00BF5046FFF782
:10962000A1FD00BF00BF81E043E000BF00BFFFF726
:1096300095FD824600BF00BFAA480830046824F0A8
:10964000FF042C43046000BF00BF5046FFF78AFDB3
:1096500000BF00BF6AE000BF00BFFFF77FFD82468A
:1096600000BF00BF9F480830046824F47F0444EA28
:109670000544046000BF00BF5046FFF773FD00BF04
:1096800000BF53E000BF00BFFFF768FD824600BF88
:1096900000BF94480830046824F07F4444EA05641D
:1096A000046000BF00BF5046FFF75CFD00BF00BF75
:1096B0003CE04FF0E0204068401C102101EB4010DE
:1096C00000F0FF094E4530DAA6F11000C11700EB9B
:1096D0009171C1F38707C11700EB91718910A0EB5D
:1096E000810101F0FF0800BF00BFFFF737FD824690
:1096F00000BF00BFB80000F1E020D0F800444FEAFE
:10970000C801FF20884084434FEAC80105FA01F0F0
:109710000443B80000F1E020C0F8004400BF00BFDF
:109720005046FFF71FFD00BF00BF00BF00BFBDE8F0
:10973000F0872DE9F04706464FF0000A102E70D250
:10974000DFE806F0080F1215182A3D090A0B0C492C
:109750005C0D708400BF00BF00BF00BF00BF624C43
:10976000BCE06FF00204B9E06FF00104B6E04FF026
:10977000FF34B3E000BF00BFFFF7F0FC824600BF3C
:1097800000BF58480568ECB200BF00BF5046FFF765
:10979000E9FC00BF00BFA1E000BF00BFFFF7DEFC97
:1097A000824600BF00BF4F480568C5F3072400BFCD
:1097B00000BF5046FFF7D6FC00BF00BF8EE000BFE1
:1097C00000BFFFF7CBFC824600BF00BF45480568DD
:1097D000C5F3074482E000BF00BFFFF7BFFC82462D
:1097E00000BF00BF3F48001D05682C0E00BF00BF32
:1097F0005046FFF7B7FC00BF00BF6FE000BF00BFDF
:10980000FFF7ACFC824600BF00BF36480830056851
:10981000ECB200BF00BF5046FFF7A4FC00BF00BF82
:109820005CE026E000BF00BFFFF798FC824600BF67
:1098300000BF2C4808300568C5F3074400BF00BFCF
:109840005046FFF78FFC00BF00BF47E000BF00BFDE
:10985000FFF784FC824600BF00BF2248083005683D
:109860002C0E00BF00BF5046FFF77CFC00BF00BFBE
:1098700034E04FF0E0204068401C102101EB401024
:1098800000F0FF094E4527DAA6F11000C11700EBE2
:109890009171C1F38707C11700EB91718910A0EB9B
:1098A000810101F0FF0800BF00BFFFF757FC8246AF
:1098B00000BF00BFB80000F1E020D0F8005400BFA6
:1098C00000BF5046FFF74EFC00BF00BF4FEAC80084
:1098D00025FA00F0C4B200E0034C00BF00BF2046F0
:1098E000BDE8F08718ED00E00080FFFF10B500F044
:1098F00036F800F091FA10BD704710B50446702C90
:1099000004D204F11001C8B2FFF778FC10BD10B505
:10991000FFF720FC10BD10B50446702C04D204F1F2
:109920001001C8B2FFF70EFD10BD70B504460D461C
:109930000026702C10D200BF00BFFFF70FFC0646B8
:1099400000BF00BFF84840F8245000BF00BF3046B9
:10995000FFF708FC00BF00BF70BD00BFFEE710B5F9
:10996000002404E0E0B2F149FFF7DFFF641C702C33
:10997000F8D310BD70B50446002600BF00BFFFF746
:10998000EDFB064600BF00BFFAF762FF00BF00BF55
:109990003046FFF7E7FB00BF00BF702C04D2E2485F
:1099A00050F8245005B1A847FAF768FF70BD10B50C
:1099B0000020FFF7DFFF10BD10B50120FFF7DAFF31
:1099C00010BD10B50220FFF7D5FF10BD10B5032064
:1099D000FFF7D0FF10BD10B50420FFF7CBFF10BD7F
:1099E00010B50520FFF7C6FF10BD10B50620FFF724
:1099F000C1FF10BD10B50720FFF7BCFF10BD10B5AB
:109A00000820FFF7B7FF10BD10B50920FFF7B2FF20
:109A100010BD10B50A20FFF7ADFF10BD10B50B202B
:109A2000FFF7A8FF10BD10B50C20FFF7A3FF10BD76
:109A300010B50D20FFF79EFF10BD10B50E20FFF7EB
:109A400099FF10BD10B50F20FFF794FF10BD10B5A2
:109A50001020FFF78FFF10BD10B51120FFF78AFF10
:109A600010BD10B51220FFF785FF10BD10B51320F3
:109A7000FFF780FF10BD10B51420FFF77BFF10BD6E
:109A800010B51520FFF776FF10BD10B51620FFF7B3
:109A900071FF10BD10B51720FFF76CFF10BD10B59A
:109AA0001820FFF767FF10BD10B51920FFF762FF00
:109AB00010BD10B51A20FFF75DFF10BD10B51B20BB
:109AC000FFF758FF10BD10B51C20FFF753FF10BD66
:109AD00010B51D20FFF74EFF10BD10B51E20FFF77B
:109AE00049FF10BD10B51F20FFF744FF10BD10B592
:109AF0002020FFF73FFF10BD10B52120FFF73AFFF0
:109B000010BD10B52220FFF735FF10BD10B5232082
:109B1000FFF730FF10BD10B52420FFF72BFF10BD5D
:109B200010B52520FFF726FF10BD10B52620FFF742
:109B300021FF10BD10B52720FFF71CFF10BD10B589
:109B40002820FFF717FF10BD10B52920FFF712FFDF
:109B500010BD10B52A20FFF70DFF10BD10B52B204A
:109B6000FFF708FF10BD10B52C20FFF703FF10BD55
:109B700010B52D20FFF7FEFE10BD10B52E20FFF70B
:109B8000F9FE10BD10B52F20FFF7F4FE10BD10B583
:109B90003020FFF7EFFE10BD10B53120FFF7EAFED1
:109BA00010BD10B53220FFF7E5FE10BD10B5332013
:109BB000FFF7E0FE10BD10B53420FFF7DBFE10BD4F
:109BC00010B53520FFF7D6FE10BD10B53620FFF7D3
:109BD000D1FE10BD10B53720FFF7CCFE10BD10B57B
:109BE0003820FFF7C7FE10BD10B53920FFF7C2FEC1
:109BF00010BD10B53A20FFF7BDFE10BD10B53B20DB
:109C0000FFF7B8FE10BD10B53C20FFF7B3FE10BD46
:109C100010B53D20FFF7AEFE10BD10B53E20FFF79A
:109C2000A9FE10BD10B53F20FFF7A4FE10BD10B572
:109C30004020FFF79FFE10BD10B54120FFF79AFEB0
:109C400010BD10B54220FFF795FE10BD10B54320A2
:109C5000FFF790FE10BD10B54420FFF78BFE10BD3E
:109C600010B54520FFF786FE10BD10B54620FFF762
:109C700081FE10BD10B54720FFF77CFE10BD10B56A
:109C80004820FFF777FE10BD10B54920FFF772FEA0
:109C900010BD10B54A20FFF76DFE10BD10B54B206A
:109CA000FFF768FE10BD10B54C20FFF763FE10BD36
:109CB00010B54D20FFF75EFE10BD10B54E20FFF72A
:109CC00059FE10BD10B54F20FFF754FE10BD10B562
:109CD0005020FFF74FFE10BD10B55120FFF74AFE90
:109CE00010BD10B55220FFF745FE10BD10B5532032
:109CF000FFF740FE10BD10B55420FFF73BFE10BD2E
:109D000010B55520FFF736FE10BD10B55620FFF7F1
:109D100031FE10BD10B55720FFF72CFE10BD10B559
:109D20005820FFF727FE10BDCC3400205B990000BF
:109D300010B55920FFF71EFE10BD10B55A20FFF7D1
:109D400019FE10BD10B55B20FFF714FE10BD10B555
:109D50005C20FFF70FFE10BD10B55D20FFF70AFE77
:109D600010BD10B55E20FFF705FE10BD10B55F20D9
:109D7000FFF700FE10BD10B56020FFF7FBFD10BD22
:109D800010B56120FFF7F6FD10BD10B56220FFF79A
:109D9000F1FD10BD10B56320FFF7ECFD10BD10B54F
:109DA0006420FFF7E7FD10BD10B56520FFF7E2FD69
:109DB00010BD10B56620FFF7DDFD10BD10B56720A2
:109DC000FFF7D8FD10BD10B56820FFF7D3FD10BD1B
:109DD00010B56920FFF7CEFD10BD10B56A20FFF762
:109DE000C9FD10BD10B56B20FFF7C4FD10BD10B547
:109DF0006C20FFF7BFFD10BD10B56D20FFF7BAFD59
:109E000010BD10B56E20FFF7B5FD10BD10B56F2069
:109E1000FFF7B0FD10BD00005348C06F20F01C00DC
:109E20005149C8670846C06F40F01000C8674E48E7
:109E3000C03000684D4908404B49C1F8C0004A484D
:109E4000C03000684A4908434749C03108604806A5
:109E50004549B03108604FF04C70086060204549BA
:109E6000086004204049C1F864014248A0380068F5
:109E70003E4908403C49C1F8C0003E48A03800684F
:109E80003D4908433849C1F8C0000846D0F8600190
:109E900040F40000C1F8600100BF36480830006897
:109EA00000F0010080F001000028F6D12E48B0300B
:109EB0000068324908432C49C1F8B00070472DE9C9
:109EC000F043DFF8A4C0DCF8B0C0CCF3007CBCF1F8
:109ED000000F3ED0DFF890C0DCF860C1CCF38A26DA
:109EE000DFF884C0DCF860C1CCF30A0303EB9622F0
:109EF000DFF874C0DCF864C1CCF30424DFF868C078
:109F0000DCF864C10CF01F05DFF85CC0DCF8B0C001
:109F1000CCF3036111B1032904D101E0184902E037
:109F2000184900E000BF00BF01FB02F804F1010C7A
:109F300005F101090CFB09FCB8FBFCF0DFF828C0B7
:109F4000DCF8B0C0CCF3090C0CF10107B0FBF7F062
:109F500000E00020DFF830C0CCF80000BDE8F0835E
:109F6000094800687047000000E00F4010FC10FC3A
:109F70008100010060E10F40850185010300009030
:109F80000024F40040787D017C00002010B51948C1
:109F9000006840F08070174908600020164948604A
:109FA0000846006840F001000860FFF788FF04469B
:109FB0002046FFF70CF810BD0F49486870472DE99F
:109FC000F0478246FFF77BFF4FF0000980460B4ABF
:109FD0000023404649461FF0FBFF064632460B462B
:109FE000504600211FF0F4FF04460D462046294646
:109FF000BDE8F087FCED00E0001000E040420F00FB
:10A0000010B50024FAF724FCF9F7DAFD0446002124
:10A01000FA48F6F735FAFA4A0021F848F6F7BFFA97
:10A020000020F84908700120F74908702046F9F728
:10A03000CBFDFAF723FC10BD10B50024FAF708FC9D
:10A04000F9F7BEFD04460121F048F6F719FAEC4A8B
:10A05000203A0121ED48F6F7A2FA0020EC490870F9
:10A060000120EC4908702046F9F7AEFDFAF706FC2E
:10A0700010BD10B50024FAF7EBFBF9F7A1FD04467B
:10A080000021E248F6F7FCF9DD4A403A0021DF48BA
:10A09000F6F785FA0020E04908700120DF490870D2
:10A0A0002046F9F791FDFAF7E9FB10BD10B5DC4841
:10A0B0000078012801D1002010BDDA48F8F7EAFC49
:10A0C000D848401CF8F7E6FCD748F8F7E3FC08212D
:10A0D000D648F7F727FCD448F8F7DCFC0421D3482E
:10A0E000F7F720FCD048F8F7D5FC0221CF48F7F766
:10A0F00019FCCD48F8F7CEFC0121CC48F7F712FC4B
:10A10000C948401EF8F7C6FC8021C948F7F70AFC89
:10A11000C548401EF8F7BEFC4021C548F7F702FCD1
:10A12000C148401EF8F7B6FC2021C148F7F7FAFBFA
:10A13000BD48401EF8F7AEFC1021BD48F7F7F2FB12
:10A14000B948F8F7A7FC2021B848F7F7EBFBB64869
:10A15000F8F7A0FC1021B548F7F7E4FBB248C01EA1
:10A16000F8F798FC1021B348F7F7DCFBAE48C01EA7
:10A17000F8F790FC2021AF48F7F7D4FBAA48401D20
:10A18000F8F788FC0121AC48F7F7CCFBA648401D46
:10A19000F8F780FC0221A848F7F7C4FBA248401D4D
:10A1A000F8F778FC0421A448F7F7BCFB9E48401D53
:10A1B000F8F770FC0821A048F7F7B4FB00231A4613
:10A1C00019469248F6F76CF90123002219468F4888
:10A1D000F6F766F900231A4619468848F6F760F93B
:10A1E00008218A48F6F77BFA08218448F6F777FABF
:10A1F00000231A4619468548F6F779F901231A46CD
:10A2000000218248F6F773F902231A4600217F489D
:10A21000F6F76DF903231A4600217C48F6F767F933
:10A2200004231A4600217948F6F761F905231A46F6
:10A2300000217648F6F75BF906231A460021734899
:10A24000F6F755F96723072200217048F6F74FF912
:10A250000823002201216D48F6F749F9092301225C
:10A2600011466A48F6F743F90A230222012167489A
:10A27000F6F73DF96B23032201216448F6F737F91D
:10A280004FF48073002211465C48F6F730F940F233
:10A290000113012200215948F6F729F94FF481737F
:10A2A000022200215548F6F722F940F263130322F7
:10A2B00000215248F6F71BF960490E20FFF735FBE5
:10A2C0005F490F20FFF731FB5E492E20FFF72DFB82
:10A2D0000E20FFF720FB0F20FFF71DFB2E20FFF7BE
:10A2E0001AFB00214948F6F7A7F801214748F6F77D
:10A2F000A3F800214148F6F79FF81E20F7F738FF32
:10A300001F20F7F735FF3E20F7F732FF00213F48C7
:10A31000F6F7BAF801213D48F6F7B6F800213748BC
:10A32000F6F7B2F800213948F6F7AAF801213748C4
:10A33000F6F7A6F800213148F6F7A2F80020BBE6B0
:10A3400070B504460D4615B94FF0FF3070BD3E485C
:10A35000005D08287DD2DFE800F0041D363738792B
:10A360007A7B00BF2C4800780028FBD101202A49C5
:10A37000087000202949087000212448F6F780F869
:10A3800000212248F6F71CF900BF24480078002875
:10A39000FBD05EE000BF1E4800780028FBD1012002
:10A3A0001B49087000201B49087001211748F6F767
:10A3B00067F801211548F6F703F900BF1548007842
:10A3C0000028FBD045E044E043E000BF0D480078A2
:10A3D0000028FBD101200B49087000200A490870B1
:10A3E00000210648F6F74CF800210448F6F7E8F893
:10A3F00000BF054800780028FBD02AE00090034009
:10A40000CC3600208400002085000020008003401E
:10A4100082000020830000208000002081000020B6
:10A420009A000020003800F0040800F000400240CC
:10A4300000700040005000400010064073A0000073
:10A4400039A0000001A000008600002001E000E02B
:10A4500000BF00BF094850F8240000EE100AB8EE13
:10A46000400ADFED070A20EE200ADFED060A80EE43
:10A47000201A85ED001A002068E700008C360020C5
:10A4800000404E450000804510B52548F8F702FB16
:10A4900000BF2348F8F781FA0028FAD0F6F7FAF956
:10A4A00004460CB100BFFEE710BD2DE9F0410446A3
:10A4B0000D46164604F0030018B14FF0FF30BDE81A
:10A4C000F0810027F9F77CFB0746324621462846F3
:10A4D000F6F722FA20B1324621462846F6F71CFA52
:10A4E0003846F9F771FB0020E9E72DE9F041044611
:10A4F0000D46164604F0030018B14FF0FF30BDE8DA
:10A50000F0810027F9F75CFB0746324621462846D2
:10A51000F6F7E8F93846F9F757FB0020EFE70000B7
:10A52000005800F02DE9F04104460D4616461F463E
:10A53000082C03DB4FF0FF30BDE8F08100BF04EBD7
:10A540004400F94901EB8000C0780128F7D004EB02
:10A55000440001EB800000790128F0D0002004EBDA
:10A560004401F14A02F8210004EB4400114601EBDA
:10A570008000467004EB440001EB8000877004EB20
:10A58000440001EB8000856014BBE848F8F782FACC
:10A59000E748F8F77FFAE648F8F77CFAE548F7F776
:10A5A0004DFBE548F7F74AFB0421E448F7F77DFA4D
:10A5B0000821E248F7F76AFAA6B9E148854208D1CE
:10A5C000FFF7CEFC804600224146DE48F7F7A1FBAC
:10A5D0000CE0FFF7C5FC804601224146D948F7F759
:10A5E00098FB03E03946D748F7F7C2FB012C33D17B
:10A5F000CE48401CF8F74EFACD48401DF8F74AFA0D
:10A60000CB48401DF8F746FACF48F7F717FBCF487D
:10A61000F7F714FB0121CE48F7F747FA0221CC489F
:10A62000F7F734FAA6B9C648854208D1FFF798FC77
:10A63000804600224146C748F7F76BFB0CE0FFF766
:10A640008FFC804601224146C248F7F762FB03E0D7
:10A650003946C048F7F78CFB022C33D1B348801C35
:10A66000F8F718FAB2480930F8F714FAB048093088
:10A67000F8F710FAB848F7F7E1FAB848F7F7DEFA52
:10A680000221B748F7F711FA0121B548F7F7FEF9AB
:10A69000A6B9AB48854208D1FFF762FC804600228C
:10A6A0004146B048F7F735FB0CE0FFF759FC804610
:10A6B00001224146AB48F7F72CFB03E03946A94895
:10A6C000F7F756FB032C33D19848C01CF8F7E2F992
:10A6D00097480830F8F7DEF995480830F8F7DAF9C6
:10A6E000A148F7F7ABFAA148F7F7A8FA1021A0485C
:10A6F000F7F7DBF920219E48F7F7C8F9A6B990488B
:10A70000854208D1FFF72CFC80460022414699483B
:10A71000F7F7FFFA0CE0FFF723FC804601224146E1
:10A720009448F7F7F6FA03E039469248F7F720FB2A
:10A73000042C33D17D48001DF8F7ACF97C48083073
:10A74000F8F7A8F97A480830F8F7A4F98A48F7F733
:10A7500075FA8A48F7F772FA40218548F7F7A5F9A4
:10A7600080218348F7F792F9A6B97548854208D148
:10A77000FFF7F6FB8046002241468148F7F7C9FA09
:10A780000CE0FFF7EDFB8046012241467C48F7F7DD
:10A79000C0FA03E039467A48F7F7EAFA052C31D1D6
:10A7A0006248401DF8F776F96148F8F773F9604898
:10A7B000F8F770F97348F7F741FA7348F7F73EFA7C
:10A7C00001215E48F7F771F902215C48F7F75EF95D
:10A7D000A6B95B48854208D1FFF7C2FB804600223C
:10A7E00041466A48F7F795FA0CE0FFF7B9FB804657
:10A7F000012241466548F7F78CFA03E03946634881
:10A80000F7F7B6FA062C37D14848801DF8F742F919
:10A810004748401EF8F73EF94548401EF8F73AF918
:10A8200041F60200F7F70AFA41F60240F7F706FA96
:10A8300040214FF04020F7F738F980214FF04020B9
:10A84000F7F724F9A6B93E48854208D1FFF788FBFF
:10A850008046002241464E48F7F75BFA0CE0FFF7CE
:10A860007FFB8046012241464948F7F752FA03E050
:10A8700039464748F7F77CFA072C33D12B48C01DDF
:10A88000F8F708F92A48801CF8F704F92848801CD2
:10A89000F8F700F93F48F7F7D1F93F48F7F7CEF955
:10A8A00001213E48F7F701F902213C48F7F7EEF89D
:10A8B000A6B92348854208D1FFF752FB8046002203
:10A8C00041463748F7F725FA0CE0FFF749FB804689
:10A8D000012241463248F7F71CFA03E03946304876
:10A8E000F7F746FA012004EB44010F4A02F8210071
:10A8F000002021E62DE9F0470546884616461F460A
:10A900004FF00009082D03DB4FF0FF30BDE8F08762
:10A9100036B12FB105EB4500034911F8200010B9FD
:10A920004FF0FF30F2E73DE0DC360020002000F081
:10A93000010800F002080100020C01000050004074
:10A94000A08601000000024002000600020406008A
:10A95000006002400010024002040A0002000A00E7
:10A9600000200640002002400210090002140900E5
:10A97000001006400030024002180900021C0900C5
:10A9800000000C40020001000204010000100C4015
:10A9900000200C400200030002040300007000408D
:10A9A00000300C40F9F70CF98146012005EB450118
:10A9B000FE4A02EB8101087105EB4500114601EBEF
:10A9C00080004078002876D1002D75D100BFF8486E
:10A9D000F7F776FA0028FAD100224146F448F7F753
:10A9E00068FA012F28D13178F148F7F78CFA07215E
:10A9F000EF48F7F777FAEE48F7F776FA58B1002004
:10AA000005EB4501E94A02EB810108714846F9F777
:10AA1000DBF8B81E7AE700BFE548F7F751FA0028DF
:10AA2000FAD105EB4501E14A02EB81010871484684
:10AA3000F9F7CAF8002069E7002445E044B9315D20
:10AA4000DB48F7F760FA0321D948F7F74BFA13E030
:10AA5000781EA04208D1315DD548F7F754FA052198
:10AA6000D348F7F73FFA07E0315DD148F7F74BFAE3
:10AA70000121CF48F7F736FACD48F7F735FAE0B1BC
:10AA8000781EA0420AD0CA48F7F72EFA00F010004C
:10AA9000102803D00421C648F7F724FA002005EB5C
:10AAA0004501C24A02EB810108714846F9F78CF86A
:10AAB0004FF0FF302AE71CE209E000BFBC48F7F77F
:10AAC000FFF90028FAD1641CBC42B7D3A4E3012DDE
:10AAD0007FD100BFB748F7F7F3F90028FAD1002279
:10AAE0004146B448F7F7E5F9012F28D13178B1484C
:10AAF000F7F709FA0721AF48F7F7F4F9AD48F7F788
:10AB0000F3F958B1002005EB4501A84A02EB810199
:10AB100008714846F9F758F8B81EF7E600BFA5488F
:10AB2000F7F7CEF90028FAD105EB45019F4A02EB71
:10AB3000810108714846F9F747F80020E6E600244D
:10AB400044E044B9315D9B48F7F7DDF903219948AA
:10AB5000F7F7C8F913E0781EA04208D1315D954897
:10AB6000F7F7D1F905219348F7F7BCF907E0315D14
:10AB70009048F7F7C8F901218E48F7F7B3F98D48E7
:10AB8000F7F7B2F9D8B1781EA0420AD08948F7F792
:10AB9000ABF900F01000102803D004218548F7F726
:10ABA000A1F9002005EB4501804A02EB8101087103
:10ABB0004846F9F709F84FF0FF30A7E609E000BF73
:10ABC0007C48F7F77DF90028FAD1641CBC42B8D361
:10ABD00022E3022D7FD100BF7748F7F771F90028F3
:10ABE000FAD1002241467448F7F763F9012F28D1C2
:10ABF00031787148F7F787F907216F48F7F772F94D
:10AC00006D48F7F771F958B1002005EB4501674A27
:10AC100002EB810108714846F8F7D6FFB81E75E6C9
:10AC200000BF6548F7F74CF90028FAD105EB45015C
:10AC30005E4A02EB810108714846F8F7C5FF002023
:10AC400064E6002444E044B9315D5B48F7F75BF902
:10AC500003215948F7F746F913E0781EA04208D1BE
:10AC6000315D5548F7F74FF905215348F7F73AF9A1
:10AC700007E0315D5048F7F746F901214E48F7F7F4
:10AC800031F94D48F7F730F9D8B1781EA0420AD013
:10AC90004948F7F729F900F01000102803D00421E3
:10ACA0004548F7F71FF9002005EB45013F4A02EB45
:10ACB000810108714846F8F787FF4FF0FF3025E61D
:10ACC00009E000BF3C48F7F7FBF80028FAD1641C04
:10ACD000BC42B8D3A0E2032D72D100BF3748F7F7CA
:10ACE000EFF80028FAD1002241463448F7F7E1F89E
:10ACF000012F28D131783148F7F705F907212F487E
:10AD0000F7F7F0F82D48F7F7EFF858B1002005EB0A
:10AD10004501264A02EB810108714846F8F754FFC5
:10AD2000B81EF3E500BF2548F7F7CAF80028FAD1A6
:10AD300005EB45011D4A02EB810108714846F8F711
:10AD400043FF0020E2E500244FE044B9315D1B4899
:10AD5000F7F7D9F803211948F7F7C4F813E0781E7C
:10AD6000A04208D1315D1548F7F7CDF80521134809
:10AD7000F7F7B8F807E0315D1048F7F7C4F801219C
:10AD80000E48F7F7AFF80D48F7F7AEF830B3781E76
:10AD9000A0420AD00948F7F7A7F800F010001028E1
:10ADA00003D004210548F7F79DF80AE0DC360020BF
:10ADB000000002400010024000200240003002402B
:10ADC00016E0002005EB4501FE4A02EB8101087107
:10ADD0004846F8F7F9FE4FF0FF3097E500BFFA4814
:10ADE000F7F76EF80028FAD1641CBC42ADD313E229
:10ADF000042D7FD100BFF548F7F762F80028FAD19B
:10AE000000224146F148F7F754F8012F28D1317854
:10AE1000EE48F7F778F80721EC48F7F763F8EB48C6
:10AE2000F7F762F858B1002005EB4501E54A02EB5F
:10AE3000810108714846F8F7C7FEB81E66E500BFF5
:10AE4000E248F7F73DF80028FAD105EB4501DD4A65
:10AE500002EB810108714846F8F7B6FE002055E57F
:10AE6000002444E044B9315DD848F7F74CF8032199
:10AE7000D648F7F737F813E0781EA04208D1315DC5
:10AE8000D248F7F740F80521D048F7F72BF807E04C
:10AE9000315DCE48F7F737F80121CC48F7F722F8B3
:10AEA000CA48F7F721F8D8B1781EA0420AD0C7489F
:10AEB000F7F71AF800F01000102803D00421C34857
:10AEC000F7F710F8002005EB4501BE4A02EB8101BF
:10AED00008714846F8F778FE4FF0FF3016E509E0B4
:10AEE00000BFBA48F6F7ECFF0028FAD1641CBC4258
:10AEF000B8D391E1052D7FD100BFB548F6F7E0FF4B
:10AF00000028FAD100224146B148F6F7D2FF012FBE
:10AF100028D13178AE48F6F7F6FF0721AC48F6F7AE
:10AF2000E1FFAB48F6F7E0FF58B1002005EB450123
:10AF3000A44A02EB810108714846F8F745FEB81EA5
:10AF4000E4E400BFA248F6F7BBFF0028FAD105EB06
:10AF500045019C4A02EB810108714846F8F734FE2E
:10AF60000020D3E4002444E044B9315D9848F6F76A
:10AF7000CAFF03219648F6F7B5FF13E0781EA042FA
:10AF800008D1315D9248F6F7BEFF05219048F6F7EB
:10AF9000A9FF07E0315D8E48F6F7B5FF01218C4827
:10AFA000F6F7A0FF8A48F6F79FFFD8B1781EA042B7
:10AFB0000AD08748F6F798FF00F01000102803D059
:10AFC00004218348F6F78EFF002005EB45017D4AFA
:10AFD00002EB810108714846F8F7F6FD4FF0FF30AB
:10AFE00094E409E000BF7A48F6F76AFF0028FAD136
:10AFF000641CBC42B8D30FE1062D7FD100BF754859
:10B00000F6F75EFF0028FAD1002241467148F6F7B4
:10B0100050FF012F28D131786E48F6F774FF0721D1
:10B020006C48F6F75FFF6B48F6F75EFF58B10020FB
:10B0300005EB4501634A02EB810108714846F8F7C8
:10B04000C3FDB81E62E400BF6248F6F739FF00286E
:10B05000FAD105EB45015B4A02EB810108714846D4
:10B06000F8F7B2FD002051E4002444E044B9315D1A
:10B070005848F6F748FF03215648F6F733FF13E028
:10B08000781EA04208D1315D5248F6F73CFF0521F9
:10B090005048F6F727FF07E0315D4E48F6F733FFDB
:10B0A00001214C48F6F71EFF4A48F6F71DFFD8B1BC
:10B0B000781EA0420AD04748F6F716FF00F01000AD
:10B0C000102803D004214348F6F70CFF002005EBBD
:10B0D00045013C4A02EB810108714846F8F774FDCE
:10B0E0004FF0FF3012E409E000BF3A48F6F7E8FEFF
:10B0F0000028FAD1641CBC42B8D38DE0072D60D182
:10B1000000BF3548F6F7DCFE0028FAD100224146A0
:10B110003148F6F7CEFE012F28D131782E48F6F7C8
:10B12000F2FE07212C48F6F7DDFE2B48F6F7DCFE91
:10B1300058B1002005EB4501224A02EB810108715C
:10B140004846F8F741FDB81E64E400BF2248F6F710
:10B15000B7FE0028FAD105EB45011A4A02EB81013E
:10B1600008714846F8F730FD002053E4002451E010
:10B1700044B9315D1848F6F7C6FE03211648F6F7C4
:10B18000B1FE13E0781EA04208D1315D1248F6F7F7
:10B19000BAFE05211048F6F7A5FE07E0315D0E481E
:10B1A000F6F7B1FE01210C48F6F79CFE0A48F6F7C7
:10B1B0009BFE40B3781EA04218D00748F6F794FED5
:10B1C0000CE029E0DC3600200030024000000C409A
:10B1D00000100C4000200C4000300C4000F010002B
:10B1E000102803D00421FD48F6F77CFE002005EB73
:10B1F0004501FB4A02EB810108714846F8F7E4FC7F
:10B200004FF0FF3006E400BFF448F6F759FE00287F
:10B21000FAD1641CBC42ABD3002005EB4501F04AD7
:10B2200002EB810108714846F8F7CEFC002041E4AA
:10B230002DE9F0470546884617461E464FF000099F
:10B24000082D03DB4FF0FF30BDE8F08737B12EB19A
:10B2500005EB4500E24911F8200010B94FF0FF302E
:10B26000F2E7F8F7ADFC8146012005EB4501DC4A29
:10B2700002EB8101C87005EB4500114601EB80002F
:10B280004078002878D1002D78D100BFD548F6F756
:10B2900017FE0028FAD101224146D248F6F709FEEE
:10B2A000012E29D10721CF48F6F71CFECD48F6F72D
:10B2B0001BFE58B1002005EB4501C94A02EB810194
:10B2C000C8704846F8F780FCB01EBDE700BFC5480F
:10B2D000F6F7F6FD0028FAD1C248F6F716FE3870E8
:10B2E000002005EB4501BE4A02EB8101C8704846CB
:10B2F000F8F76AFC0020A7E700243BE024B90B2103
:10B30000B848F6F7EFFD0BE0701EA04204D105210E
:10B31000B448F6F7E7FD03E00921B248F6F7E2FD8D
:10B32000B048F6F7E1FDD0B1701EA0420AD0AD489A
:10B33000F6F7DAFD00F01000102803D00421A94828
:10B34000F6F7D0FD002005EB4501A54A02EB81018F
:10B35000C8704846F8F738FC4FF0FF3074E700BF7C
:10B36000A048F6F7ADFD0028FAD19E48F6F7CDFDCE
:10B370003855641CB442C1D375E3FFE7012D78D181
:10B3800000BF9948F6F79CFD0028FAD101224146FA
:10B390009548F6F78EFD012E29D107219248F6F740
:10B3A000A1FD9148F6F7A0FD58B1002005EB45013D
:10B3B0008B4A02EB8101C8704846F8F705FCB01EC5
:10B3C00042E700BF8848F6F77BFD0028FAD186489F
:10B3D000F6F79BFD3870002005EB4501804A02EB33
:10B3E0008101C8704846F8F7EFFB00202CE70024E5
:10B3F0003BE024B90B217C48F6F774FD0BE0701E8E
:10B40000A04204D105217848F6F76CFD03E009213C
:10B410007548F6F767FD7448F6F766FDD0B1701E03
:10B42000A0420AD07048F6F75FFD00F01000102827
:10B4300003D004216C48F6F755FD002005EB4501CB
:10B44000674A02EB8101C8704846F8F7BDFB4FF030
:10B45000FF30F9E600BF6448F6F732FD0028FAD164
:10B460006148F6F752FD3855641CB442C1D3FAE284
:10B47000FFE7022D78D100BF5C48F6F721FD0028D8
:10B48000FAD1012241465948F6F713FD012E29D180
:10B4900007215648F6F726FD5448F6F725FD58B122
:10B4A000002005EB45014E4A02EB8101C870484679
:10B4B000F8F78AFBB01EC7E600BF4C48F6F700FD60
:10B4C0000028FAD14948F6F720FD3870002005EB36
:10B4D0004501434A02EB8101C8704846F8F774FB06
:10B4E0000020B1E600243BE024B90B213F48F6F7E9
:10B4F000F9FC0BE0701EA04204D105213B48F6F791
:10B50000F1FC03E009213948F6F7ECFC3748F6F77F
:10B51000EBFCD0B1701EA0420AD03448F6F7E4FC30
:10B5200000F01000102803D004213048F6F7DAFCB0
:10B53000002005EB45012A4A02EB8101C87048460C
:10B54000F8F742FB4FF0FF307EE600BF2748F6F7E2
:10B55000B7FC0028FAD12548F6F7D7FC3855641C0B
:10B56000B442C1D37FE2FFE7032D76D100BF20486C
:10B57000F6F7A6FC0028FAD1012241461C48F6F74E
:10B5800098FC012E36D107211948F6F7ABFC184874
:10B59000F6F7AAFC58B1002005EB4501104A02EB72
:10B5A0008101C8704846F8F70FFBB01E4CE600BF9B
:10B5B0000F48F6F785FC0028FAD10D48F6F7A5FCF0
:10B5C0003870002005EB4501054A02EB8101C87087
:10B5D0004846F8F7F9FA002036E6000000300C4043
:10B5E000DC36002000000240001002400020024033
:10B5F0000030024000243CE024B90B21F748F6F764
:10B6000071FC0BE0701EA04204D10521F348F6F74F
:10B6100069FC03E00921F148F6F764FCEF48F6F70E
:10B6200063FCD8B1701EA0420AD0EC48F6F75CFC6F
:10B6300000F01000102803D00421E848F6F752FC6F
:10B64000002005EB4501E64A02EB8101C87048463F
:10B65000F8F7BAFA4FF0FF30F6E50DE000BFDF482B
:10B66000F6F72EFC0028FAD1DC48F6F74EFC3855E8
:10B67000641CB442C0D3F6E1042D78D100BFD94890
:10B68000F6F71EFC0028FAD101224146D548F6F70C
:10B6900010FC012E29D10721D248F6F723FCD1480E
:10B6A000F6F722FC58B1002005EB4501CC4A02EB2D
:10B6B0008101C8704846F8F787FAB01EC4E500BF9C
:10B6C000C848F6F7FDFB0028FAD1C648F6F71DFC7E
:10B6D0003870002005EB4501C14A02EB8101C870BA
:10B6E0004846F8F771FA0020AEE500243BE024B9A3
:10B6F0000B21BC48F6F7F6FB0BE0701EA04204D10C
:10B700000521B848F6F7EEFB03E00921B548F6F746
:10B71000E9FBB448F6F7E8FBD0B1701EA0420AD0AE
:10B72000B048F6F7E1FB00F01000102803D0042128
:10B73000AC48F6F7D7FB002005EB4501A84A02EB21
:10B740008101C8704846F8F73FFA4FF0FF307BE5BB
:10B7500000BFA448F6F7B4FB0028FAD1A148F6F7D9
:10B76000D4FB3855641CB442C1D37CE1FFE7052DFE
:10B7700078D100BF9C48F6F7A3FB0028FAD101223C
:10B7800041469948F6F795FB012E29D107219648A5
:10B79000F6F7A8FB9448F6F7A7FB58B1002005EB95
:10B7A00045018F4A02EB8101C8704846F8F70CFA50
:10B7B000B01E49E500BF8C48F6F782FB0028FAD19D
:10B7C0008948F6F7A2FB3870002005EB4501844A52
:10B7D00002EB8101C8704846F8F7F6F9002033E51E
:10B7E00000243BE024B90B217F48F6F77BFB0BE0FC
:10B7F000701EA04204D105217B48F6F773FB03E0DD
:10B8000009217948F6F76EFB7748F6F76DFBD0B162
:10B81000701EA0420AD07448F6F766FB00F01000D4
:10B82000102803D004217048F6F75CFB002005EBDC
:10B8300045016B4A02EB8101C8704846F8F7C4F92C
:10B840004FF0FF3000E500BF6748F6F739FB0028EE
:10B85000FAD16548F6F759FB3855641CB442C1D398
:10B8600001E1FFE7062D78D100BF6048F6F728FB1D
:10B870000028FAD1012241465C48F6F71AFB012E56
:10B8800029D107215948F6F72DFB5848F6F72CFB2C
:10B8900058B1002005EB4501514A02EB8101C87007
:10B8A0004846F8F791F9B01ECEE400BF4F48F6F7CE
:10B8B00007FB0028FAD14D48F6F727FB3870002027
:10B8C00005EB4501464A02EB8101C8704846F8F78E
:10B8D0007BF90020B8E400243BE024B90B21434865
:10B8E000F6F700FB0BE0701EA04204D105213F4893
:10B8F000F6F7F8FA03E009213C48F6F7F3FA3B487B
:10B90000F6F7F2FAD0B1701EA0420AD03748F6F727
:10B91000EBFA00F01000102803D004213348F6F7AA
:10B92000E1FA002005EB45012D4A02EB8101C870C8
:10B930004846F8F749F94FF0FF3085E400BF2B483F
:10B94000F6F7BEFA0028FAD12848F6F7DEFA38559D
:10B95000641CB442C1D386E0FFE7072D75D100BF58
:10B960002348F6F7ADFA0028FAD1012241462048D3
:10B97000F6F79FFA012E29D107211D48F6F7B2FAF2
:10B980001B48F6F7B1FA58B1002005EB4501144AFF
:10B9900002EB8101C8704846F8F716F9B01E53E46F
:10B9A00000BF1348F6F78CFA0028FAD11048F6F7D2
:10B9B000ACFA3870002005EB4501094A02EB810121
:10B9C000C8704846F8F700F900203DE4002448E03C
:10B9D00084B90B210648F6F785FA17E000300240DB
:10B9E000DC36002000000C4000100C4000200C4011
:10B9F00000300C40701EA04204D10521FE48F6F72D
:10BA000071FA03E00921FC48F6F76CFAFA48F6F7F8
:10BA10006BFAD8B1701EA0420AD0F748F6F764FA64
:10BA200000F01000102803D00421F348F6F75AFA6A
:10BA3000002005EB4501F14A02EB8101C870484640
:10BA4000F8F7C2F84FF0FF300AE40CE000BFEA4814
:10BA5000F6F736FA0028FAD1E748F6F756FA3855DD
:10BA6000641CB442B4D3002005EB4501E34A02EB69
:10BA70008101C8704846F8F7A7F8002025E42DE9B1
:10BA8000F04104460D4616461F46082C03DB4FF0D6
:10BA9000FF30BDE8F08104EB4400D84911F82000E4
:10BAA00010B94FF0FF30F4E700BF04EB4400D34976
:10BAB00001EB8000C0780128F7D004EB440001EBD3
:10BAC000800000790128F0D0002004EB4401CB4A2B
:10BAD00002F82100FCB900BFC948F6F7F1F90028C7
:10BAE000FAD104EB4400C54901EB8000407818B955
:10BAF000C348F6F754F902E0C148F6F755F9A6B97C
:10BB0000C048854208D1FEF72BFA80460022414604
:10BB1000BB48F6F7FEF80CE0FEF722FA8046012259
:10BB20004146B748F6F7F5F803E03946B448F6F76A
:10BB30001FF9012C2DD100BFB348F6F7C1F9002839
:10BB4000FAD104EB4400AD4901EB8000407818B90C
:10BB5000AD48F6F724F902E0AB48F6F725F9A6B9A7
:10BB6000A848854208D1FEF7FBF9804600224146ED
:10BB7000A548F6F7CEF80CE0FEF7F2F98046012270
:10BB80004146A148F6F7C5F803E039469E48F6F766
:10BB9000EFF8022C2DD100BF9C48F6F791F9002850
:10BBA000FAD104EB4400954901EB8000407818B9C4
:10BBB0009648F6F7F4F802E09448F6F7F5F8A6B9D7
:10BBC0009048854208D1FEF7CBF9804600224146D5
:10BBD0008E48F6F79EF80CE0FEF7C2F98046012287
:10BBE00041468A48F6F795F803E039468748F6F764
:10BBF000BFF8032C2DD100BF8548F6F761F9002866
:10BC0000FAD104EB44007D4901EB8000407818B97B
:10BC10007F48F6F7C4F802E07D48F6F7C5F8A6B904
:10BC20007848854208D1FEF79BF9804600224146BC
:10BC30007748F6F76EF80CE0FEF792F9804601229D
:10BC400041467348F6F765F803E039467048F6F761
:10BC50008FF8042C2DD100BF6E48F6F731F900287B
:10BC6000FAD104EB4400654901EB8000407818B933
:10BC70006848F6F794F802E06648F6F795F8A6B932
:10BC80006048854208D1FEF76BF9804600224146A4
:10BC90006048F6F73EF80CE0FEF762F980460122B4
:10BCA00041465C48F6F735F803E039465948F6F75F
:10BCB0005FF8052C2DD100BF5748F6F701F9002891
:10BCC000FAD104EB44004D4901EB8000407818B9EB
:10BCD0005148F6F764F802E04F48F6F765F8A6B960
:10BCE0004848854208D1FEF73BF98046002241468C
:10BCF0004948F6F70EF80CE0FEF732F980460122CB
:10BD000041464548F6F705F803E039464248F6F75C
:10BD10002FF8062C2DD100BF4048F6F7D1F80028A7
:10BD2000FAD104EB4400354901EB8000407818B9A2
:10BD30003A48F6F734F802E03848F6F735F8A6B98D
:10BD40003048854208D1FEF70BF980460022414673
:10BD50003248F5F7DEFF0CE0FEF702F980460122DB
:10BD600041462E48F5F7D5FF03E039462B48F5F755
:10BD7000FFFF072C2DD100BF1F48F6F7A1F80028C0
:10BD8000FAD104EB44001D4901EB8000407818B95A
:10BD90001948F6F704F802E01748F6F705F8A6B9CF
:10BDA0001848854208D1FEF7DBF88046002241465C
:10BDB0001148F5F7AEFF0CE0FEF7D2F880460122FD
:10BDC00041460D48F5F7A5FF03E039460A48F5F767
:10BDD000CFFF04EB4400094901EB8000467004EBFF
:10BDE000440001EB8000877004EB440001EB80000D
:10BDF0008560012014E0000000300C40DC3600209B
:10BE000000000240A0860100001002400020024015
:10BE10000030024000000C4000100C4000200C409C
:10BE200004EB4401024A02F82100002031E6000040
:10BE3000DC3600202DE9FE4304460F4690461E46A0
:10BE40000A9D042C03DA042D01DB102D03DD4FF0D5
:10BE5000FF30BDE8FE8300BF04EB4400F74901EB6F
:10BE60008000C07A0128F7D0002004EB4401F34A97
:10BE700002F82100002C48D1F148F6F70BFEF148FA
:10BE8000F6F708FEEF48F6F705FEEE48F6F702FE75
:10BE9000EC48F6F7FFFD40F60F00F5F7CFFE40F651
:10BEA0000F40F5F7CBFE41F20F00F5F7C7FE41F268
:10BEB0000F40F5F7C3FE04214FF04020F5F740FE98
:10BEC00008214FF04020F5F73BFE10214FF04020B5
:10BED000F5F736FE20214FF04020F5F731FEFEF752
:10BEE0003FF8814643463A464946D748CDE9006582
:10BEF000F6F784FAD448F6F7ACFA00BF02A9D248A4
:10BF0000F6F7F8FA0028F9D1D6E0012C45D1CC4853
:10BF1000401CF6F7BFFDCB48401CF6F7BBFDC948F7
:10BF2000401CF6F7B7FDC748001DF6F7B3FDC5483E
:10BF3000001DF6F7AFFDC548F5F780FEC448F5F7DC
:10BF40007DFEC448F5F77AFEC348F5F777FE202159
:10BF5000C248F5F7F5FD1021C048F5F7F1FD1021B5
:10BF6000BF48F5F7EDFD2021BD48F5F7E9FDFDF7E8
:10BF7000F7FF814643463A464946BA48CDE900654F
:10BF8000F6F73CFAB748F6F764FA00BF02A9B548DD
:10BF9000F6F7B0FA0028F9D18EE0022C45D1A84876
:10BFA000801CF6F777FDA748C01CF6F773FDA5487F
:10BFB000C01CF6F76FFDA348C01CF6F76BFDA14847
:10BFC000C01CF6F767FDA848F5F738FEA748F5F757
:10BFD00035FEA748F5F732FEA648F5F72FFE0821F3
:10BFE000A548F5F7ADFD0421A348F5F7A9FD022109
:10BFF000A148F5F7A5FD01219F48F5F7A1FDFDF743
:10C00000AFFF814643463A4649469C48CDE9006524
:10C01000F6F7F4F99948F6F71CFA00BF02A9974819
:10C02000F6F768FA0028F9D146E0032C44D1844899
:10C03000C01CF6F72FFD8348401DF6F72BFD814805
:10C04000401DF6F727FD7F48401DF6F723FD7D488C
:10C05000401DF6F71FFD8A48F5F7F0FD8948F5F712
:10C06000EDFD8948F5F7EAFD8848F5F7E7FD082179
:10C070008748F5F765FD04218548F5F761FD022144
:10C080008348F5F75DFD01218148F5F759FDFDF77E
:10C0900067FF814643463A4649467E48CDE90065FA
:10C0A000F6F7ACF97B48F6F7D4F900BF02A9794856
:10C0B000F6F720FA0028F9D104EB44005F4901EBC0
:10C0C000800080F8098004EB440001EB8000857259
:10C0D00004EB440001EB8000466004EB440001EBFC
:10C0E00080000772012004EB4401544A02F8210049
:10C0F0000020AEE6F8B504460E4615460020009036
:10C100000027042C00DA15B94FF0FF30F8BD04EB1E
:10C1100044004A4911F82000012802D04FF0FF30B6
:10C12000F4E7012004EB4401444A02EB8101C872A8
:10C13000F7F746FD0746ACB900BF69464248F6F737
:10C14000D9F90028F9D131463F48F6F7B8F900BFD0
:10C150003D48F6F7E2F90028FAD169463A48F6F781
:10C16000C0F946E0012C15D100BF69463D48F6F7FD
:10C17000C1F90028F9D131463A48F6F7A0F900BFD5
:10C180003848F6F7CAF90028FAD169463548F6F773
:10C19000A8F92EE0022C15D100BF69463748F6F702
:10C1A000A9F90028F9D131463448F6F788F900BFDB
:10C1B0003248F6F7B2F90028FAD169462F48F6F767
:10C1C00090F916E0032C14D100BF69463148F6F708
:10C1D00091F90028F9D131462E48F6F770F900BFE1
:10C1E0002C48F6F79AF90028FAD169462948F6F75B
:10C1F00078F9009828703846F7F7E6FC002004EB41
:10C2000044010E4A02EB8101C87200BF7EE72DE9AE
:10C21000FC4704460E46174698460A9D042C03DB4D
:10C220004FF0FF30BDE8FC87B5B32878042802DB67
:10C230002878102831DD4FF0FF30F3E73C3700203D
:10C24000001C00F0000800F0008000400F14010006
:10C250000F1001000F1004000F14040000500040E4
:10C2600000400240009000400F0C03000F08030044
:10C270000F0403000F0003000070004000A0004006
:10C280000E0C05000E0805000E0405000E0005004A
:10C290000050024000B00040FFE704EB4400A44916
:10C2A00011F8200010B94FF0FF30BBE700BF04EBDE
:10C2B00044009F4901EB8000C07A0128F7D000209C
:10C2C00004EB44019A4A02F821002EB1307804EBC5
:10C2D000440102EB8101087237B1387804EB440164
:10C2E000934A02EB81014872B8F1000F07D004EBCA
:10C2F00044018F4A02EB8101D8F80000486035B153
:10C30000287804EB44018A4A02EB8101887264BBFD
:10C3100000BF8848F6F701F90028FAD18548F6F7FA
:10C320009DF8FDF71DFE814604EB4400804901EBBA
:10C330008000807A04EB44017D4A02EB8101496868
:10C34000CDE9001004EB4400114601EB8000437A74
:10C3500004EB440001EB8000027A49467548F6F789
:10C360004DF87448F6F775F88BE0012C2CD100BF1E
:10C370007148F6F7D2F80028FAD16F48F6F76EF850
:10C38000FDF7EEFD814604EB4400694901EB8000B6
:10C39000807A04EB4401664A02EB81014968CDE9E9
:10C3A000001004EB4400114601EB8000437A04EBDB
:10C3B000440001EB8000027A49465F48F6F71EF818
:10C3C0005D48F6F746F85CE0022C2CD100BF5B48D4
:10C3D000F6F7A3F80028FAD15848F6F73FF8FDF72A
:10C3E000BFFD814604EB4400514901EB8000807A97
:10C3F00004EB44014E4A02EB81014968CDE900108B
:10C4000004EB4400114601EB8000437A04EB440046
:10C4100001EB8000027A49464848F5F7EFFF4748AC
:10C42000F6F717F82DE0032C2BD100BF4448F6F7A0
:10C4300074F80028FAD14248F6F710F8FDF790FD9D
:10C44000814604EB44003A4901EB8000807A04EB1A
:10C450004401374A02EB81014968CDE9001004EB41
:10C460004400114601EB8000437A04EB440001EBE9
:10C470008000027A49463248F5F7C0FF3048F5F7A8
:10C48000E8FF012004EB4401294A02F821000020C2
:10C49000C8E670B504460D46042C02DB4FF0FF30B1
:10C4A00070BD04EB4400224911F8200010B94FF090
:10C4B000FF30F5E774B935B9F72208214FF0402075
:10C4C000F5F72BFA32E0082211464FF04020F5F73D
:10C4D00024FA2BE0012C0CD12DB9EF2210211948A0
:10C4E000F5F71BFA22E0102211461648F5F715FA67
:10C4F0001CE0022C0CD12DB9FB2204211248F5F7C7
:10C500000CFA13E0042211460F48F5F706FA0DE085
:10C51000032C0BD12DB9FB2204210C48F5F7FDF9B2
:10C5200004E0042211460948F5F7F7F90020B7E7BF
:10C530003C370020008000400090004000A00040F8
:10C5400000B0004000500040007000400050024029
:10C5500010B52348F6F79EFA012211462148F4F758
:10C56000B5FF0823012211461E48F5F73CF81C4888
:10C57000F6F790FA012202211A48F4F7A7FF0823E0
:10C58000012202211748F5F72EF810BD704710B5AB
:10C59000FFF7FCFFFFF7DCFFF5F77EFDFDF774FF0B
:10C5A00010BD10B504462CB9012211460D48F5F70F
:10C5B000B4F904E0FE2201210A48F5F7AEF910BDF6
:10C5C00010B504462CB9022211460648F5F7A5F924
:10C5D00004E0FD2202210348F5F79FF910BD000099
:10C5E000030800F00070004010B50024F8F730F99F
:10C5F000F7F7E6FA04460121FE48F7F79DF8FE48F2
:10C60000C069401CFC49C8612046F7F7DDFAF8F71D
:10C6100035F910BD10B50024F8F71AF9F7F7D0FA7C
:10C6200004460121F548F7F787F8F3488069401C74
:10C63000F14988612046F7F7C7FAF8F71FF910BDEE
:10C6400010B50024F8F704F9F7F7BAFA0446012107
:10C65000EB48F7F771F8E8484069401CE649486143
:10C660002046F7F7B1FAF8F709F910BD10B5002424
:10C67000F8F7EEF8F7F7A4FA04460121E148F7F7D6
:10C680005BF8DD480069401CDB4908612046F7F78C
:10C690009BFAF8F7F3F810BD10B50024F8F7D8F8B6
:10C6A000F7F78EFA04460121D748F7F745F8D24844
:10C6B000C068401CD049C8602046F7F785FAF8F7F3
:10C6C000DDF810BD10B50024F8F7C2F8F7F778FAD6
:10C6D00004460121CD48F7F72FF8C7488068401C71
:10C6E000C54988602046F7F76FFAF8F7C7F810BD1C
:10C6F00010B50024F8F7ACF8F7F762FA0446012108
:10C70000C348F7F719F8BC484068401CBA4948606C
:10C710002046F7F759FAF8F7B1F810BD10B5002424
:10C72000F8F796F8F7F74CFA04460121B948F7F7FD
:10C7300003F8B1480068401CAF4908602046F7F78D
:10C7400043FAF8F79BF810BD70B504460D46082C67
:10C7500002DB4FF0FF3070BD34BBAF48F6F79AF9FB
:10C760002221AC48F6F7B4FEFDF7FAFB4FF47A71DC
:10C77000B0FBF1F000FB05F63246FF21A548F6F7C5
:10C7800059FF2320F5F7F4FCA4491320FDF7CDF859
:10C790001320FDF7C0F801219E48F6F7BFFFFF21E7
:10C7A0009C48F6F787FE4CE1012C27D19A48401CA3
:10C7B000F6F770F922219648F6F78AFEFDF7D0FBCE
:10C7C0004FF47A71B0FBF1F000FB05F63246FF2121
:10C7D0008F48F6F72FFF2520F5F7CAFC9049152062
:10C7E000FDF7A3F81520FDF796F801218848F6F724
:10C7F00095FFFF218648F6F75DFE22E1022C27D146
:10C800008548801CF6F746F922218048F6F760FE3D
:10C81000FDF7A6FB4FF47A71B0FBF1F000FB05F6D3
:10C820003246FF217948F6F705FF2720F5F7A0FCEF
:10C830007C491720FDF779F81720FDF76CF80121E6
:10C840007248F6F76BFFFF217048F6F733FEF8E009
:10C85000032C27D17048C01CF6F71CF922216A4826
:10C86000F6F736FEFDF77CFB4FF47A71B0FBF1F082
:10C8700000FB05F63246FF216348F6F7DBFE332066
:10C88000F5F776FC68492320FDF74FF82320FDF7E4
:10C8900042F801215C48F6F741FFFF215A48F6F7BC
:10C8A00009FECEE0042C27D15B48001DF6F7F2F814
:10C8B00022215448F6F70CFEFDF752FB4FF47A7133
:10C8C000B0FBF1F000FB05F63246FF214D48F6F7CC
:10C8D000B1FE4F20F5F74CFC54493F20FDF725F8F9
:10C8E0003F20FDF718F801214648F6F717FFFF2112
:10C8F0004448F6F7DFFDA4E0052C27D14648401D4B
:10C90000F6F7C8F822213E48F6F7E2FDFDF728FBCE
:10C910004FF47A71B0FBF1F000FB05F63246FF21CF
:10C920003748F6F787FE5120F5F722FC40494120B1
:10C93000FCF7FBFF4120FCF7EEFF01213048F6F742
:10C94000EDFEFF212E48F6F7B5FD7AE0062C27D143
:10C950003148801DF6F79EF822212848F6F7B8FDE9
:10C96000FDF7FEFA4FF47A71B0FBF1F000FB05F62B
:10C970003246FF212148F6F75DFE7220F5F7F8FBFD
:10C980002C496220FCF7D1FF6220FCF7C4FF012193
:10C990001A48F6F7C3FEFF211848F6F78BFD50E062
:10C9A000072C4BD11C48C01DF6F774F82221114802
:10C9B000F6F78EFDFDF7D4FA4FF47A71B0FBF1F083
:10C9C00000FB05F63246FF210A48F6F733FE7420D5
:10C9D000F5F7CEFB18496420FCF7A7FF6420FCF7AD
:10C9E0009AFF01210348F6F799FEFF210148F6F767
:10C9F00061FD26E000100E406C37002000000E4064
:10CA0000005003400040034000300340002003403A
:10CA10000010034000000340000400F01DC70000A8
:10CA2000F1C60000C5C6000099C600006DC6000032
:10CA300041C6000015C60000E9C500004FF0FF30F8
:10CA400089E6002087E60246082A00DC11B94FF08B
:10CA5000FF307047024850F8220008600020F8E7D5
:10CA60006C37002070B50024F7F7F2FEF7F7A8F84E
:10CA700004460121F748F6F7D2FF05462946F54856
:10CA8000F6F7D3FF11E0F348F6F771FFF2490870AB
:10CA9000F24890F8BD00012807D1F148006820B1A4
:10CAA00008460078EE4909688847EA48F6F753FFD8
:10CAB0000028E8D12046F7F787F8F7F7DFFE70BDCA
:10CAC00070B50024F7F7C4FEF7F77AF804460121A1
:10CAD000E448F6F7A4FF05462946E248F6F7A5FF25
:10CAE00011E0E048F6F743FFDF490870DB4890F8B3
:10CAF000A500012807D1DD48006820B1084600786C
:10CB0000DA4909688847D748F6F725FF0028E8D1B1
:10CB10002046F7F759F8F7F7B1FE70BD70B500245D
:10CB2000F7F796FEF7F74CF804460121D048F6F7E0
:10CB300076FF05462946CE48F6F777FF11E0CC4848
:10CB4000F6F715FFCB490870C44890F88D0001280E
:10CB500007D1C948006820B108460078C64909686D
:10CB60008847C348F6F7F7FE0028E8D12046F7F7D4
:10CB70002BF8F7F783FE70BD70B50024F7F768FE59
:10CB8000F7F71EF804460121BC48F6F748FF0546B2
:10CB90002946BA48F6F749FF11E0B848F6F7E7FE2C
:10CBA000B7490870AD4890F87500012807D1B5481D
:10CBB000006820B108460078B24909688847AF4844
:10CBC000F6F7C9FE0028E8D12046F6F7FDFFF7F793
:10CBD00055FE70BD70B50024F7F73AFEF6F7F0FF8A
:10CBE00004460121A848F6F71AFF05462946A6483B
:10CBF000F6F71BFF11E0A448F6F7B9FEA349087049
:10CC0000964890F85D00012807D1A148006820B13E
:10CC1000084600789E49096888479B48F6F79BFEBE
:10CC20000028E8D12046F6F7CFFFF7F727FE70BDC2
:10CC300070B50024F7F70CFEF6F7C2FF0446012199
:10CC40009448F6F7ECFE054629469248F6F7EDFEC5
:10CC500011E09048F6F78BFE8F4908707F4890F8F6
:10CC60004500012807D18D48006820B108460078AA
:10CC70008A49096888478748F6F76DFE0028E8D199
:10CC80002046F6F7A1FFF7F7F9FD70BD70B5002457
:10CC9000F7F7DEFDF6F794FF044601218048F6F72A
:10CCA000BEFE054629467E48F6F7BFFE11E07C48E9
:10CCB000F6F75DFE7B490870684890F82D00012862
:10CCC00007D17948006820B108460078764909689C
:10CCD00088477348F6F73FFE0028E8D12046F6F76C
:10CCE00073FFF7F7CBFD70BD70B50024F7F7B0FD0B
:10CCF000F6F766FF044601216C48F6F790FE0546FC
:10CD000029466A48F6F791FE10E06848F6F72FFECC
:10CD1000674908705148407D012807D1654800687F
:10CD200020B1084600786349096888475F48F6F7EC
:10CD300012FE0028E9D12046F6F746FFF7F79EFDE0
:10CD400070BD2DE9F04704460D4616461F46DDF836
:10CD50002080082C03DB4FF0FF30BDE8F087B5F5ED
:10CD6000965F18D0B5F5165F15D0B5F5615F12D096
:10CD7000B5F5964F0FD0B5F5164F0CD04DF6C02037
:10CD8000854208D0B5F5614F05D0B5F5E13F02D039
:10CD90004FF0FF30E1E704EB4400304901EBC00005
:10CDA0004560052E06D0062E0CD0072E12D0082E78
:10CDB00020D117E0002004EB4401284A02EBC10116
:10CDC00088601AE0202004EB4401244A02EBC101F0
:10CDD000886012E0402004EB4401204A02EBC101CC
:10CDE00088600AE0602004EB44011C4A02EBC101A8
:10CDF000886002E04FF0FF30AFE700BF012F02D0A4
:10CE0000022F10D107E0002004EB4401134A02EB8B
:10CE1000C101C8600AE0082004EB44010F4A02EB9C
:10CE2000C101C86002E04FF0FF3096E700BFB8F1E3
:10CE3000000F06D0B8F1010F3ED0B8F1020F4BD170
:10CE400042E0002004EB4401044A02EBC101086106
:10CE500045E0000000300140A3000020C400002095
:10CE6000C000002000200140A2000020BC000020E3
:10CE700000100140A1000020B80000200000014087
:10CE8000A0000020B400002000F000409F0000201F
:10CE9000B000002000E000409E000020AC00002018
:10CEA00000D000409D000020A800002000C00040ED
:10CEB0009C000020A4000020062004EB4401FE4A50
:10CEC00002EBC10108610AE0022004EB4401FA4AC6
:10CED00002EBC101086102E04FF0FF303DE700BF07
:10CEE00000BF04EB4400F44901EBC000007D0128C1
:10CEF000F7D004EB440001EBC000407D0128F0D0E6
:10CF0000002004EB4401EC4A02F83100002C7DD1F2
:10CF1000EA48F5F7BFFDEA48F5F7BCFDE848F5F744
:10CF2000B9FD0120F4F78AFE40F20140F4F786FED5
:10CF300001214FF04020F4F730FE02214FF0402055
:10CF4000F4F72BFEFDF70CF8824604EB4400DA49B7
:10CF500001EBC000806804EB4401DFF85CC30CEB1C
:10CF6000C101C968084304EB44010CEBC101096924
:10CF700040EA010304EB4400614601EBC000514666
:10CF80004268D048F6F754FC04EB4400CA4901EB70
:10CF9000C0004078022816D1C948F5F77BFD012270
:10CFA00002214FF04020F4F791FA4FF484730122EC
:10CFB00002214FF04020F4F716FBFD2202214FF032
:10CFC0004020F4F7AAFCC0490520FCF7AEFC052080
:10CFD000FCF7A1FC1520F5F7CBF860211520F5F73B
:10CFE000A5F85021B748F6F712FD0121B548F6F72C
:10CFF00016FD81464946B348F6F717FD00BFB14814
:10D00000F6F7B5FC0028FADAE0E3FFE7012C7DD162
:10D01000AA48401CF5F73EFDA948401CF5F73AFD2B
:10D02000A748401CF5F736FD4FF00110F4F706FE57
:10D03000A648F4F703FE0121A548F4F7AEFD02214E
:10D04000A348F4F7AAFDFCF78BFF824604EB4400EB
:10D05000994901EBC000806804EB4401DFF858C235
:10D060000CEBC101C968084304EB44010CEBC1019E
:10D07000096940EA010304EB4400614601EBC0008A
:10D08000514642689348F6F7D3FB8D480930F5F7CF
:10D0900001FD012210219048F4F718FA0C23012217
:10D0A00010218D48F4F79FFA04EB4400824901EB0C
:10D0B000C0004078022819D181480A30F5F7EAFC0F
:10D0C000EF2210218448F4F728FC012211468348FE
:10D0D000F4F7FCF90C23012211468048F4F783FA97
:10D0E000FE2201217D48F4F718FC04E010221146CD
:10D0F0007948F4F712FC7A490620FCF716FC062062
:10D10000FCF709FC1620F5F733F800E017E0602182
:10D110001620F5F70BF850216E48F6F778FC012140
:10D120006C48F6F77CFC814649466A48F6F77DFC78
:10D1300000BF6848F6F71BFC0028FADA46E3022C29
:10D140007CD15E48801CF5F7A5FC5D48F5F7A2FC94
:10D150005B48F5F79FFC41F60100F4F76FFD41F6DF
:10D160000140F4F76BFD40214FF04020F4F715FD2E
:10D1700080214FF04020F4F710FDFCF7F1FE8246CD
:10D1800004EB44004C4901EBC000806804EB44010F
:10D19000DFF824C10CEBC101C968084304EB44016A
:10D1A0000CEBC101096940EA010304EB440061464C
:10D1B00001EBC000514642684A48F6F739FB04EBE0
:10D1C00044003D4901EBC0004078022813D13C489F
:10D1D000401DF5F75FFC012210214348F4F776F972
:10D1E0000C23012210214048F4F7FDF9EF22102111
:10D1F0003D48F4F792FB3D492120FCF796FB2120A6
:10D20000FCF789FB3120F4F7B3FF60213120F4F7FC
:10D210008DFF50213348F6F7FAFB01213148F6F72C
:10D22000FEFB814649462F48F6F7FFFB00BF2D481D
:10D23000F6F79DFB0028FADAC8E2FFE7032C7CD161
:10D240001E48C01CF5F726FC1D48F5F723FC1C48BA
:10D25000F5F720FC41F20100F4F7F0FC41F2014047
:10D26000F4F7ECFC10214FF04020F4F796FC20215D
:10D270004FF04020F4F791FCFCF772FE824604EB7D
:10D2800044000D4901EBC000806804EB4401DFF865
:10D2900028C00CEBC101C968084304EB44010CEB46
:10D2A000C101096940EA010304EB4400614601EB56
:10D2B000C000514642681BE0C4000020001800F086
:10D2C000000800F000C00040E9CC000001040100AB
:10D2D0000050004000D000400010064000200640F2
:10D2E0008DCC000000E000400050024031CC000036
:10D2F000FE48F6F79DFA04EB4400FD4901EBC0003F
:10D300004078022816D1FB48F5F7C4FB0122022120
:10D310004FF04020F4F7DAF84FF484730122022131
:10D320004FF04020F4F75FF9FD2202214FF040203A
:10D33000F4F7F3FAF049382000E01FE0FCF7F5FAC3
:10D340003820FCF7E8FA4820F4F712FF6021482063
:10D35000F4F7ECFE5021E548F6F759FB0121E348CC
:10D36000F6F75DFB81464946E048F6F75EFB00BFF5
:10D37000DE48F6F7FCFA0028FADA27E2042C7ED120
:10D38000DE48F5F787FBDB48F5F784FBD948F5F76E
:10D3900081FB40F60100F4F751FC40F60140F4F740
:10D3A0004DFC04214FF04020F4F7F7FB08214FF02B
:10D3B0004020F4F7F2FBFCF7D3FD824604EB440077
:10D3C000CB4901EBC000806804EB4401DFF820C3C7
:10D3D0000CEBC101C968084304EB44010CEBC1012B
:10D3E000096940EA010304EB4400614601EBC00017
:10D3F00051464268C248F6F71BFA04EB4400BC49A8
:10D4000001EBC0004078022816D1BA48F5F742FB7C
:10D41000012202214FF04020F4F758F84FF48473B2
:10D42000012202214FF04020F4F7DDF8FD22022115
:10D430004FF04020F4F771FAB2493920FCF775FA41
:10D440003920FCF768FA4920F4F792FE6021492060
:10D45000F4F76CFE5021AA48F6F7D9FA0121A84842
:10D46000F6F7DDFA81464946A548F6F7DEFA00BF31
:10D47000A348F6F77CFA0028FADAA7E1FFE7052CC3
:10D480007DD19E48401CF5F705FB9A48801CF5F7B6
:10D4900001FB9848801CF5F7FDFA9B48F4F7CEFB9A
:10D4A0009A48F4F7CBFB40219948F4F776FB8021AA
:10D4B0009748F4F772FBFCF753FD824604EB4400F7
:10D4C0008B4901EBC000806804EB4401DFF820C207
:10D4D0000CEBC101C968084304EB44010CEBC1012A
:10D4E000096940EA010304EB4400614601EBC00016
:10D4F000514642688748F6F79BF904EB44007C49A3
:10D5000001EBC0004078022816D17A48F5F7C2FA3C
:10D51000012202214FF04020F3F7D8FF4FF484732B
:10D52000012202214FF04020F4F75DF8FD22022194
:10D530004FF04020F4F7F1F977493A20FCF7F5F97C
:10D540003A20FCF7E8F94A20F4F712FE60214A205D
:10D55000F4F7ECFD50216F48F6F759FA01216D48B8
:10D56000F6F75DFA814649466A48F6F75EFA00BF6B
:10D570006848F6F7FCF90028FADA27E1FFE7062CFD
:10D580007DD15E48801CF5F785FA5A480D30F5F7D5
:10D5900081FA58480D30F5F77DFA6048F4F74EFBF4
:10D5A0005F48F4F74BFB01215E48F4F7F6FA0221DD
:10D5B0005C48F4F7F2FAFCF7D3FC824604EB440033
:10D5C0004B4901EBC000806804EB4401DFF820C147
:10D5D0000CEBC101C968084304EB44010CEBC10129
:10D5E000096940EA010304EB4400614601EBC00015
:10D5F000514642684C48F6F71BF904EB44003C499D
:10D6000001EBC0004078022816D13A48F5F742FAFB
:10D61000012202214FF04020F3F758FF4FF48473AA
:10D62000012202214FF04020F3F7DDFFFD2202210D
:10D630004FF04020F4F771F93C493B20FCF775F9B5
:10D640003B20FCF768F94B20F4F792FD60214B205A
:10D65000F4F76CFD50213448F6F7D9F9012132482E
:10D66000F6F7DDF9814649462F48F6F7DEF900BFA7
:10D670002D48F6F77CF90028FADAA7E0FFE7072C37
:10D680007ED11E48C01CF5F705FA1A48801CF5F734
:10D6900001FA1848801CF5F7FDF92548F4F7CEFA91
:10D6A0002448F4F7CBFA10211948F4F776FA202130
:10D6B0001748F4F772FAFCF753FC824604EB440077
:10D6C0000B4901EBC000806804EB4401DFF820C087
:10D6D0000CEBC101C968084304EB44010CEBC10128
:10D6E000096940EA010304EB440025E000F0004032
:10D6F000C4000020000800F0D5CB0000041800F0A2
:10D700000000014079CB000001180200011C02005A
:10D7100000600040001001401DCB000001000D0022
:10D7200001040D000050064000200140C1CA000065
:10D730000110020001140200614601EBC0005146D5
:10D740004268FB48F6F774F804EB4400F94901EB32
:10D75000C0004078022818D1F748F5F79BF901225C
:10D7600002214FF04020F3F7B1FE4FF48473012201
:10D7700002214FF04020F3F736FFFD22022100E0A6
:10D7800024E04FF04020F4F7C8F8EC493C20FCF7C7
:10D79000CCF83C20FCF7BFF84C20F4F7E9FC602102
:10D7A0004C20F4F7C3FC5021E148F6F730F9012191
:10D7B000DF48F6F734F981464946DD48F6F735F992
:10D7C00000BFDB48F6F7D3F80028FADA012004EBB3
:10D7D0004401D84A02F831000020FFF7BEBA2DE913
:10D7E000F04104460E4617460025A846082C02DBE9
:10D7F000681EBDE8F08104EB4400CE4911F830000A
:10D80000012802D04FF0FF30F3E700BF04EB4400E3
:10D81000C84901EBC000007D0128F7D0012004EBCE
:10D820004401C44A02EBC1010875F6F7C9F9804604
:10D8300054BB04EB4400BF4901EBC0004078022810
:10D8400005D1022211464FF04020F4F766F804E0BB
:10D85000715DBB48F6F7A8F86D1CBD42F8D300BF58
:10D86000B748F6F7B3F80028FAD104EB4400B14901
:10D8700001EBC0004078022805D1FD2202214FF0C3
:10D880004020F4F74AF835E1012C28D104EB44009C
:10D89000A84901EBC0004078022804D101221146BA
:10D8A000A848F4F73AF804E0715DA748F6F77CF869
:10D8B0006D1CBD42F8D300BFA348F6F787F80028D7
:10D8C000FAD104EB44009B4901EBC00040780228E8
:10D8D000D9D1FE2201219B48F4F71FF80AE1022C5E
:10D8E00028D104EB4400934901EBC00040780228A2
:10D8F00004D1102211469548F4F70FF804E0715D49
:10D900009348F6F751F86D1CBD42F8D300BF90481C
:10D91000F6F75CF80028FAD104EB4400854901EBE6
:10D92000C00040780228AED1EF2210218748F3F7DB
:10D93000F4FFDFE0032C2AD104EB44007D4901EB26
:10D94000C0004078022805D1022211464FF0402045
:10D95000F3F7E3FF04E0715D7E48F6F725F86D1CF0
:10D96000BD42F8D300BF7B48F6F730F80028FAD163
:10D9700004EB44006F4901EBC00040780228ADD1B0
:10D98000FD2202214FF04020F3F7C7FFB2E0042C44
:10D990002AD104EB4400674901EBC000407802281B
:10D9A00005D1022211464FF04020F3F7B6FF04E004
:10D9B000715D6948F5F7F8FF6D1CBD42F8D300BFF3
:10D9C0006548F6F703F80028FAD104EB44005949FA
:10D9D00001EBC0004078022805D1FD2202214FF062
:10D9E0004020F3F79AFF85E0052C2AD104EB440090
:10D9F000504901EBC0004078022805D102221146AF
:10DA00004FF04020F3F789FF04E0715D5348F5F7CC
:10DA1000CBFF6D1CBD42F8D300BF5048F5F7D6FFD1
:10DA20000028FAD104EB4400424901EBC0004078E1
:10DA300002285FD1FD2202214FF04020F3F76DFF55
:10DA400058E0062C2AD104EB44003A4901EBC0000F
:10DA50004078022805D1022211464FF04020F3F70A
:10DA60005CFF04E0715D3E48F5F79EFF6D1CBD4212
:10DA7000F8D300BF3A48F5F7A9FF0028FAD104EB24
:10DA800044002C4901EBC0004078022832D1FD222D
:10DA900002214FF04020F3F740FF2BE0072C29D163
:10DAA00004EB4400234901EBC0004078022805D173
:10DAB000022211464FF04020F3F72FFF04E0715D82
:10DAC0001B48F5F771FF6D1CBD42F8D300BF184825
:10DAD000F5F77CFF0028FAD104EB4400154901EB6F
:10DAE000C0004078022805D1FD2202214FF04020DD
:10DAF000F3F713FF4046F6F767F8002004EB440104
:10DB00000C4A02EBC101087500BF72E610B502466F
:10DB1000082A00DA11B94FF0FF3010BD02EB4200C5
:10DB2000044B13F8300001281CD04FF0FF30F4E70D
:10DB300000300140C4000020000800F065CA000069
:10DB400000C000400020064000D0004000500240CD
:10DB500000E0004000F000400000014000100140E3
:10DB60000020014000BF02EB4200FE4B03EBC0006F
:10DB7000407D0128F7D0012002EB4203F94C04EB71
:10DB8000C3035875082A1DD2DFE802F004070A0D06
:10DB900010131619F448016017E0F448016014E00E
:10DBA000F348016011E0F34801600EE0F2480160C3
:10DBB0000BE0F248016008E0F148016005E0F1483F
:10DBC000016002E04FF0FF30A7E700BF0020A4E7AC
:10DBD0000146082902DB4FF0FF30704701EB41009E
:10DBE000E04A12F83000012802D04FF0FF30F4E78D
:10DBF000082925D2DFE801F004080C1014181C20B5
:10DC00000020D94A10601EE00020D84A10601AE0B7
:10DC10000020D74A106016E00020D64A106012E0BB
:10DC20000020D54A10600EE00020D44A10600AE0BF
:10DC30000020D34A106006E00020D24A106002E0C3
:10DC40004FF0FF30C9E700BF002001EB4102C54B98
:10DC500003EBC202507500BFBFE72DE9F047044651
:10DC60000D4616461F46DDF82080082C03DB4FF0DA
:10DC7000FF30BDE8F087B5F5965F18D0B5F5165FB3
:10DC800015D0B5F5615F12D0B5F5964F0FD0B5F54B
:10DC9000164F0CD04DF6C020854208D0B5F5614F27
:10DCA00005D0B5F5E13F02D04FF0FF30E1E704EBDE
:10DCB0004400AC4901EBC0004560052E06D0062E9D
:10DCC0000CD0072E12D0082E20D117E0002004EB34
:10DCD0004401A44A02EBC10188601AE0202004EB51
:10DCE0004401A04A02EBC101886012E0402004EB2D
:10DCF00044019C4A02EBC10188600AE0602004EB09
:10DD00004401984A02EBC101886002E04FF0FF3005
:10DD1000AFE700BF012F02D0022F10D107E0002093
:10DD200004EB44018F4A02EBC101C8600AE0002005
:10DD300004EB44018B4A02EBC101C86002E04FF0E2
:10DD4000FF3096E700BFB8F1000F06D0B8F1010F21
:10DD50000BD0B8F1020F18D10FE0002004EB440102
:10DD6000804A02EBC101086112E0062004EB440185
:10DD70007C4A02EBC10108610AE0022004EB440185
:10DD8000784A02EBC101086102E04FF0FF3070E712
:10DD900000BF00BF04EB4400724901EBC000407DAE
:10DDA0000128F7D004EB440001EBC000007D0128FE
:10DDB000F0D0002004EB44016A4A02F8310014BBA1
:10DDC000FCF7CEF8814604EB4400664901EBC00045
:10DDD000806804EB4401DFF88CC10CEBC101C96819
:10DDE000084304EB44010CEBC101096940EA01035B
:10DDF00004EB4400614601EBC000494642686248BA
:10DE0000F5F716FD1EE1012C22D1FCF7A9F8814699
:10DE100004EB4400534901EBC000806804EB44016B
:10DE2000DFF840C10CEBC101C968084304EB4401B1
:10DE30000CEBC101096940EA010304EB44006146AF
:10DE400001EBC000494642685048F5F7F1FCF9E0A3
:10DE5000022C22D1FCF784F8814604EB44004149AE
:10DE600001EBC000806804EB4401DFF8F8C00CEB64
:10DE7000C101C968084304EB44010CEBC101096905
:10DE800040EA010304EB4400614601EBC00049464F
:10DE900042683F48F5F7CCFCD4E0032C22D1FCF7D4
:10DEA0005FF8814604EB44002E4901EBC000806816
:10DEB00004EB4401DFF8ACC00CEBC101C9680843B6
:10DEC00004EB44010CEBC101096940EA010304EBD6
:10DED0004400614601EBC000494642682D48F5F711
:10DEE000A7FCAFE0042C22D1FCF73AF8814604EB02
:10DEF00044001C4901EBC000806804EB4401DFF8DA
:10DF000064C00CEBC101C968084304EB44010CEB8D
:10DF1000C101096940EA010304EB4400614601EBD9
:10DF2000C000494642681C48F5F782FC8AE0052C8F
:10DF30003FD1FCF715F8814604EB4400094901EB99
:10DF4000C000806804EB4401DFF818C00CEBC1018D
:10DF5000C968084304EB44010CEBC101096940EABC
:10DF600001031BE0C4000020A4000020A800002042
:10DF7000AC000020B0000020B4000020B800002059
:10DF8000BC000020C000002000C0004000D00040C5
:10DF900000E0004000F000400000014004EB4400BD
:10DFA000614601EBC000494642682A48F5F740FC4B
:10DFB00048E0062C22D1FBF7D3FF814604EB440056
:10DFC000254901EBC000806804EB4401DFF888C0FC
:10DFD0000CEBC101C968084304EB44010CEBC1011F
:10DFE000096940EA010304EB4400614601EBC0000B
:10DFF000494642681948F5F71BFC23E0072C21D15C
:10E00000FBF7AEFF814604EB4400134901EBC0006F
:10E01000806804EB4401DFF840C00CEBC101C96823
:10E02000084304EB44010CEBC101096940EA010318
:10E0300004EB4400614601EBC000494642680848D1
:10E04000F5F7F6FB012004EB4401034A02F8310026
:10E0500000200EE600100140C40000200020014016
:10E060000030014010B54FF08040F5F747FDFBF759
:10E0700077FF044621464FF08040F5F74BFD4FF007
:10E080008040F5F737FD10BD10B5F6F7E1FB2448E9
:10E090000078401C22490870084600781E2802DDDE
:10E0A0000120204908701F48007828B94FF08040AF
:10E0B000F5F757FDFFF7D6FFF6F7E0FB10BD10B5FB
:10E0C0004FF07040F4F7E6FC2220F4F751F84FF0DF
:10E0D0008040F5F713FDFBF743FF044621464FF060
:10E0E0008040F5F717FD4FF08040F5F7F9FC4FF051
:10E0F0008040F5F7FFFC0C491220FBF716FC1220BC
:10E10000FBF709FC4FF08040F5F7E5FC10BD00205F
:10E1100003490870704701200249087070470000E9
:10E12000840100208501002089E00000F8B5044644
:10E130000D4608208DF800008DF80150A07D0223C7
:10E140006A466F21E769B84746B2002E02DA4FF0FF
:10E15000FF30F8BD0020FCE7F8B504460D46072067
:10E160008DF800008DF80150A07D02236A466F21D2
:10E17000E769B84746B2002E02DA4FF0FF30F8BD2B
:10E180000020FCE710B5044614B94FF0FF3010BD75
:10E19000A06908B1E06910B94FF0FF30F7E79021AE
:10E1A0002046FFF7D9FF00212046FFF7BFFF0020E0
:10E1B000EDE77CB504460520019000200090A07D8D
:10E1C000012301AA6F21E669B04745B2002D02DAAA
:10E1D0004FF0FF307CBDA07D01236A466F21A66908
:10E1E000B04745B2002D02DA4FF0FF30F2E79DF85C
:10E1F000000000F00F009DF80010090901EB8101FB
:10E2000000EB4100FC49098801EBC10202EB01115E
:10E2100000EB810020810020DCE77CB5044604206F
:10E22000019000200090A07D012301AA6F21E669E2
:10E23000B04745B2002D02DA4FF0FF307CBDA07D23
:10E2400001236A466F21A669B04745B2002D02DA64
:10E250004FF0FF30F2E79DF8000000F00F009DF84E
:10E260000010C1F3001101EB810100EB4101E171EC
:10E270000020E3E77CB504460320019000200090D5
:10E28000A07D012301AA6F21E669B04745B2002DA8
:10E2900002DA4FF0FF307CBDA07D01236A466F217A
:10E2A000A669B04745B2002D02DA4FF0FF30F2E721
:10E2B0009DF8000000F00F009DF80010C1F301115F
:10E2C00001EB810100EB4101A1710020E3E77CB586
:10E2D00004460220019000200090A07D012301AAA5
:10E2E0006F21E669B04745B2002D02DA4FF0FF30EA
:10E2F0007CBDA07D01236A466F21A669B04745B267
:10E30000002D02DA4FF0FF30F2E79DF8000000F038
:10E310000F009DF80010C1F3011101EB810100EB2A
:10E32000410161710020E3E77CB5044601200190C2
:10E3300000200090A07D012301AA6F21E669B0476B
:10E3400045B2002D02DA4FF0FF307CBDA07D0123E5
:10E350006A466F21A669B04745B2002D02DA4FF038
:10E36000FF30F2E79DF8000000F00F009DF800106C
:10E37000C1F3021101EB810100EB41012171002089
:10E38000E3E77CB50446002001900090A07D0123C6
:10E3900001AA6F21E669B04745B2002D02DA4FF0BD
:10E3A000FF307CBDA07D01236A466F21A669B0477E
:10E3B00045B2002D02DA4FF0FF30F2E79DF8000081
:10E3C00000F00F009DF80010C1F3021101EB810174
:10E3D00000EB4101E1700020E3E770B505462846F7
:10E3E000FFF7CFFF44B2002C02DA4FF0FF3070BDD0
:10E3F0002846FFF799FF44B2002C02DA4FF0FF30B5
:10E40000F5E72846FFF763FF44B2002C02DA4FF02D
:10E41000FF30ECE72846FFF72DFF44B2002C02DA6C
:10E420004FF0FF30E3E72846FFF7F7FE44B2002C39
:10E4300002DA4FF0FF30DAE72846FFF7BAFE44B2BF
:10E44000002C02DA4FF0FF30D1E70020CFE7F8B51B
:10E450000446608A642190FBF1F067490880608A75
:10E46000098801EBC10202EB0111A0EB810060827F
:10E4700005208DF80000608A0A2190FBF1F201FB73
:10E4800012010A2290FBF2F041EA0010C0B28DF8AE
:10E490000100A07D02236A466F21E669B04745B2BC
:10E4A000002D02DA4FF0FF30F8BD0020FCE7F8B590
:10E4B000044604208DF80000607C0A2190FBF1F2F4
:10E4C00001FB12010A2290FBF2F041EA0010C0B2F7
:10E4D0008DF80100A07D02236A466F21E669B047EE
:10E4E00045B2002D02DA4FF0FF30F8BD0020FCE706
:10E4F000F8B5044603208DF80000207C0A2190FB2B
:10E50000F1F201FB12010A2290FBF2F041EA001045
:10E51000C0B28DF80100A07D02236A466F21E66932
:10E52000B04745B2002D02DA4FF0FF30F8BD0020B1
:10E53000FCE7F8B5044602208DF80000E07B0A21D4
:10E5400090FBF1F201FB12010A2290FBF2F041EA8A
:10E550000010C0B240F080008DF80100A07D0223C1
:10E560006A466F21E669B04745B2002D02DA4FF0E6
:10E57000FF30F8BD0020FCE7F8B5044601208DF817
:10E580000000A07B0A2190FBF1F201FB12010A229C
:10E5900090FBF2F041EA0010C0B28DF80100A07DBE
:10E5A00002236A466F21E669B04745B2002D02DAC0
:10E5B0004FF0FF30F8BD0020FCE7F8B5044600201E
:10E5C0008DF80000607B0A2190FBF1F201FB120143
:10E5D0000A2290FBF2F041EA0010C0B28DF801006F
:10E5E000A07D02236A466F21E669B04745B2002D3F
:10E5F00004DA4FF0FF30F8BD860100200020FAE772
:10E6000070B505462846FFF7D8FF44B2002C02DA61
:10E610004FF0FF3070BD2846FFF7AEFF44B2002C2C
:10E6200002DA4FF0FF30F5E72846FFF782FF44B2E9
:10E63000002C02DA4FF0FF30ECE72846FFF758FFD6
:10E6400044B2002C02DA4FF0FF30E3E72846FFF730
:10E650002EFF44B2002C02DA4FF0FF30DAE72846F2
:10E66000FFF7F5FE44B2002C02DA4FF0FF30D1E79D
:10E670000020CFE730B589B0044600254FF6FF7083
:10E6800005903EA103C9CDE903010020009001904F
:10E69000029014B9401E09B030BD20788DF80C00EE
:10E6A00005AA062103A8A3699847BDF81400000A2B
:10E6B0008DF81300BDF81400C0B28DF812000821C7
:10E6C00003A82269904709216846E26890470546F9
:10E6D000002D02DA4FF0FF30DDE79DF800002178D1
:10E6E000884207D19DF80100032803D19DF802005C
:10E6F000042802D04FF0FF30CDE74FF6FF700590B1
:10E7000005AA07216846A36998479DF807009DF868
:10E71000081040EA0120BDF81410884202D04FF0E2
:10E72000FF30B8E79DF804009DF8031040EA01208F
:10E73000069006980790BDF91C0000EE100AB8EE8E
:10E74000C00AF2EE040A80EE201A84ED021A9DF847
:10E7500006009DF8051040EA0120069006980890F2
:10E76000BDF9200000EE100AB8EEC00AF2EE040A6D
:10E7700080EE201A84ED011A00208CE701030000CE
:10E780000002C40B1CB5044614B9F748019001E01F
:10E79000F6480190002001AB02460146009003209C
:10E7A000FDF735FD1CBD38B50446002000906A46D3
:10E7B00021460320FDF79EFC9DF8000038BD10B5F2
:10E7C000044621460320FDF764FE10BD10B501206C
:10E7D000FFF7F5FFFF20FFF7E6FF10BD38B5002477
:10E7E00000BFFF20FFF7DFFF0546FF2D01D100200E
:10E7F00038BD641C6FF07F40B4FBF0F100FB1140AA
:10E8000050B90820DA4B0022114600900320FDF792
:10E8100011FB0020FFF7D3FF6FF070408442E0D37C
:10E820000120E5E710B50020FFF7C9FFFFF7D6FF8D
:10E8300008B9002010BDFFF7C9FF0120FAE72DE954
:10E84000F04105460C4617464FF00008FFF7BEFFA3
:10E85000FFF7E8FF10B1FF20BDE8F08145F0400070
:10E86000FFF7A1FF200EFFF79EFFC4F30740FFF75D
:10E870009AFFC4F30720FFF796FFE0B2FFF793FF7C
:10E880003846FFF790FF0C2D02D1FF20FFF78BFFDA
:10E890004FF01F0800BFFF20FFF785FF064606F078
:10E8A000800030B1B8F10000A8F1010101F0FF08CB
:10E8B000F1D13046D0E77CB50820AD4B002211469F
:10E8C00000900320FDF7B6FA0020FFF778FF002044
:10E8D000FFF758FF002505E0FF20FFF764FF04461F
:10E8E000681C85B2642DF7DB4020FFF75CFF002039
:10E8F000FFF759FF0020FFF756FF0020FFF753FFF7
:10E900000020FFF750FF9520FFF74DFF142600BFB2
:10E91000952200210846FFF792FF0446012C04D0FF
:10E92000301EA6F101018EB2F2D10020914908708B
:10E93000012C4AD187224FF4D5710820FFF77FFFC1
:10E94000012847D1002506E0FF20FFF72CFF01A991
:10E950004855681C85B2042DF6DB9DF80600012899
:10E9600079D19DF80700AA2875D14FF6FE7600BF31
:10E97000012200213720FFF762FF012291072920A1
:10E98000FFF75DFF044624B1301EA6F101018EB2EF
:10E99000EED1002E5FD0012200213A20FFF74FFF79
:10E9A000002858D1002506E0FF20FFF7FCFE01A952
:10E9B0004855681C85B2042DF6DB9DF8040000F074
:10E9C000400018B106206B49087044E004206949F2
:10E9D000087040E0012200213720FFF730FF0122BC
:10E9E00000212920FFF72BFF0446012C17DC022011
:10E9F000604908704FF6FE7600BF012200213720E3
:10EA0000FFF71DFF012200212920FFF718FF044610
:10EA1000BCB1301EA6F101018EB2EED111E0012091
:10EA2000544908704FF6FE7600BF012200211046BF
:10EA3000FFF705FF044624B1301EA6F101018EB296
:10EA4000F3D12EB1012251021020FFF7F8FE10B1D0
:10EA5000002048490870FFF7B9FE0120FFF792FE39
:10EA60004448007808B100207CBD0CB12046FBE78B
:10EA7000AA20F9E770B505464FF6FF7401E0601E65
:10EA800084B2FF20FFF78FFEA84201D0002CF6D100
:10EA90000CB9FF2070BD0020FCE770B504460D46A0
:10EAA000FE20FFF7E7FF08B1012070BD04E0FF2062
:10EAB000FFF779FE2070641C281EA5F101018DB2BC
:10EAC000F5D1FF20FFF76FFEFF20FFF76CFE00205F
:10EAD000EBE72DE9F04106460F461546254800783C
:10EAE000062800D07F02012D0CD1012239461120C9
:10EAF000FFF7A5FE0446FCB969023046FFF7CDFFDB
:10EB0000044619E0012239461220FFF798FE044618
:10EB100000BF4FF400713046FFF7BFFF044606F513
:10EB20000076681EC0B2051E01D0002CF1D0012273
:10EB300000210C20FFF783FEFFF748FE2046BDE8CA
:10EB4000F0812DE9F04106460D46FFF747FE0746E6
:10EB500017B10120BDE8F0812846FFF724FEFD2D06
:10EB600022D000240DE00000400D0300003FAB0167
:10EB700040420F0088010020305DFFF714FE601C4A
:10EB800084B2B4F5007FF7DBFF20FFF70CFEFF2017
:10EB9000FFF709FEFF20FFF706FE074607F01F00FC
:10EBA000052801D00220D5E70020D3E72DE9F04168
:10EBB00006460F4615464A480078062800D07F02D0
:10EBC000012D0CD1012239461820FFF738FE0446EA
:10EBD0006CBBFE213046FFF7B4FF044627E04048F7
:10EBE0000078012809D0012200213720FFF727FEF5
:10EBF000012229461720FFF722FE0122394619205B
:10EC0000FFF71DFE044694B900BFFC213046FFF714
:10EC100098FF044606F50076681EC0B2051E01D0B6
:10EC2000002CF2D0FD210020FFF78BFF0446FFF7F8
:10EC3000CDFD2046BDE8F08170B5054601220021DA
:10EC40000920FFF7FCFD044624B910212846FFF7F0
:10EC500024FF0446FFF7BAFD0CB1012070BD00206F
:10EC6000FCE770B510211F481BF0C9FC1D48FFF7D9
:10EC7000E3FF08B1002070BD1A48007800F0C00022
:10EC8000402809D11748407A1649097A00EB01203B
:10EC9000401C84B2A50220E01248407900F00F0029
:10ECA0001049897A00EBD1100E49497A01F003012D
:10ECB00000EB4100861C0B48007A80110949C97994
:10ECC00000EB81000749897901F0030100EB812005
:10ECD000441CA6F1090004FA00F52846CBE7000021
:10ECE000880100208C37002010B500231A466649A1
:10ECF0000120FBF717FC0446002C02DA4FF0FF302E
:10ED000010BD012061498875614888616148C8610A
:10ED10000846FFF737FA0446002C02DA4FF0FF30BE
:10ED2000EEE70020ECE770B50446E18857484182E1
:10ED30006179417421790174E178C173A17881739B
:10ED400061784173FFF75CFC0546002D02DA4FF055
:10ED5000FF3070BD0020FCE770B504464B48FFF75C
:10ED60003CFB0546002D02DA4FF0FF3070BD4748EE
:10ED70000089E0804548C0796071444880792071FD
:10ED800042484079E07041480079A0703F48C0781F
:10ED900060700020EAE770B504463C48FFF71DFBB1
:10EDA0000546002D02DA4FF0FF3070BDE18837488C
:10EDB0000089814201DD0220F7E7E18833480089BC
:10EDC000814201DA0120F0E761793048C07981425F
:10EDD00001DD0220E9E761792C48C079814201DA3E
:10EDE0000120E2E7217929488079814201DD022072
:10EDF000DBE7217925488079814201DA0120D4E7D7
:10EE0000E17822484079814201DD0220CDE7E178B6
:10EE10001E484079814201DA0120C6E7A1781B48EB
:10EE20000079814201DD0220BFE7A178174800790F
:10EE3000814201DA0120B8E761781448C078814244
:10EE400001DD0220B1E761781048C078814201DA23
:10EE50000120AAE70020A8E710B58CB00446E0889E
:10EE6000A0F26C7006906079401E059020790490A5
:10EE7000E0780390A07802906078019001A81BF0E0
:10EE800066FC0CB010BD0000801A06009C37002004
:10EE900031B20000F5A80000014609B90020704712
:10EEA0000120FCE770B5054665B9FFF704FD04468F
:10EEB00034B10120FFF766FCFF20FFF774FC01E08E
:10EEC000002070BD00BF0120FBE72DE9F0410646A0
:10EED0000F4690461C4614B90420BDE8F0816EB977
:10EEE000E2B241463846FFF7F4FD054625B1FF2062
:10EEF000FFF759FC0120F0E70020EEE70420ECE7E3
:10EF00002DE9F04105460E461746984665B908F0CA
:10EF1000FF0239463046FFF749FE044614B9002087
:10EF2000BDE8F0810120FBE70420F9E72DE9F0417D
:10EF300006460F4615462EBB37B1012F1AD0022FB9
:10EF40000FD0032F1BD111E00020FFF738FCFFF793
:10EF500045FC08B9002400E001240120FFF72FFC44
:10EF60000FE04FF40070288000240AE00820288079
:10EF7000002406E0FFF775FE2860002401E0042469
:10EF800000BF00E001242046BDE8F0810EB56846D0
:10EF9000FFF7E2FEC0B9BDF80600A0F2BC70400663
:10EFA0009DF8051040EA41509DF8041040EA0140E8
:10EFB0009DF8031040EAC1209DF8021040EA41107C
:10EFC0009DF8011008430EBD0048FCE72252A556EB
:10EFD000014648780A7842EA002070470146C8781E
:10EFE0008A7842EA00204A7842EA00200A7842EA17
:10EFF0000020704700F8011B091200F8011B704740
:10F0000000F8011B090A00F8011B090A00F8011B9E
:10F01000090A00F8011B704730B503460C463AB1A7
:10F0200000BF14F8015B03F8015B551E2A1EF8D1DE
:10F0300030BD10B5034600BF03F8011B541E221E4D
:10F04000FAD110BDF0B503461D460C46002000BFA6
:10F0500015F8017B14F801CBA7EB0C00561E321EED
:10F0600001D00028F4D0F0BD024600E0521C107818
:10F0700010B110788842F9D110787047014609B173
:10F08000002070470020FCE7014609B100207047CE
:10F090000020FCE72DE9F0410646356815F8014BE4
:10F0A0002046FFF7EBFF60B115F8017B3846FFF70C
:10F0B000EBFF18B94FF0FF30BDE8F08107EB0420FB
:10F0C00084B24CB140F2B511204603F056FA044622
:10F0D00014B94FF0FF30EFE7A04635604046EBE74C
:10F0E0002DE9F04107460C46164640F2B511384668
:10F0F00003F026FA0546FF2D0BDD022E02D200207A
:10F10000BDE8F081281204F8010B04F8015B02202D
:10F11000F6E705B10EB90020F2E704F8015B012023
:10F12000EEE770B504460025E078E8B16078012389
:10F1300004F13801626BFFF7E3FEA0B90020E07034
:10F14000A16A606B401A216A88420DD2A078022819
:10F150000AD1236A616BCA186078012304F138016F
:10F16000FFF7CEFE00E00125284670BD70B50446CD
:10F170000D460026606BA84210D02046FFF7D1FF55
:10F1800006465EB9607801232A4604F13801FFF78C
:10F190009CFE10B14FF0FF3501266563304670BD0F
:10F1A00070B504462046FFF7BCFF0546002D38D158
:10F1B000207803282ED1207901282BD1420200216A
:10F1C00004F13800FFF735FF4AF6552104F23620E6
:10F1D000FFF710FFF74904F13800FFF711FFF64978
:10F1E00004F50770FFF70CFF04F508706169FFF77D
:10F1F00007FF04F509702169FFF702FF606A401CF0
:10F2000060636078012304F13801626BFFF778FED8
:10F2100000202071607800221146FFF787FE00B1C0
:10F220000125284670BD0246891ED069801E88428D
:10F2300001D8002070475389106B03FB0100F9E7E8
:10F240002DE9F04781460C46D9F80050022C02D334
:10F25000E869A04202D84FF001085EE04FF0FF38A5
:10F260002878012804D002282CD0032851D13CE072
:10F27000264606EB5606A86A00EB56212846FFF7FD
:10F2800075FF00B148E03046761CC0F3080105F177
:10F290003800475CA86A00EB56212846FFF766FF56
:10F2A00000B139E0C6F3080105F13800405C47EAD7
:10F2B000002704F0010008B1380901E0C7F30B0092
:10F2C000804629E0A86A00EB14212846FFF74EFF8C
:10F2D00000B121E040F2FF1101EA440205F13801DA
:10F2E0005018FFF775FE804616E0A86A00EBD411AF
:10F2F0002846FFF73BFF00B10EE040F2FF1101EAA4
:10F30000840205F138015018FFF768FE20F07048BC
:10F3100002E04FF0010800BF00BF4046BDE8F087A3
:10F320002DE9F04704460D4616464FF00209022D1E
:10F3300074D3E069A84271D92078012804D002284A
:10F3400049D003280DD15EE02F4607EB5707A06A8E
:10F3500000EB57212046FFF709FF8146B9F1000F66
:10F3600000D075E038467F1CC0F3080104F1380076
:10F3700001EB000805F0010028B1F1B298F8000097
:10F3800061F31F1000E0304688F800000120E070B3
:10F39000A06A00EB57212046FFF7E8FE8146B9F14D
:10F3A000000F00D054E0C7F3080104F1380001EB6E
:10F3B000000805F0010010B1C6F3071006E098F848
:10F3C000000000F0F000C6F30321084388F80000B5
:10F3D0000120E0703CE0A06A00EB15212046FFF719
:10F3E000C5FE8146B9F1000F00D031E0B1B240F264
:10F3F000FF1202EA450304F138029818FFF7FAFDFC
:10F400000120E07024E0A06A00EBD5112046FFF750
:10F41000ADFE8146B9F1000F01D019E019E040F2CC
:10F42000FF1101EA850204F138015018FFF7D6FDFB
:10F4300066F31B00064640F2FF1101EA850204F163
:10F44000380150183146FFF7DBFD0120E07000BFA6
:10F4500000BF4846BDE8F0872DE9F04781460E46DB
:10F4600017464FF00008D9F80040022E02D3E06999
:10F47000B04202D80220BDE8F08767B100BF4FF06C
:10F48000FF3239462046FFF74BFF8046B8F1000FA8
:10F4900001D04046EFE700BF31464846FFF7D0FEB7
:10F4A000054605B922E0012D01D10220E3E7681CE1
:10F4B00008B90120DFE7002231462046FFF730FF80
:10F4C0008046B8F1000F01D04046D4E7E069801EC5
:10F4D0006169814206D26069401C6061207940F018
:10F4E000010020712E46E069B042D5D800BF00204F
:10F4F000C1E72DE9F04782468846DAF80040B8F1C6
:10F50000000F06D1276917B1E069B84215D8012765
:10F5100013E041465046FFF793FE0546022D02D206
:10F520000120BDE8F087681C08B92846F9E7E069C2
:10F53000A84201D92846F4E74746606908B9002087
:10F54000EFE70026474518D17E1CE069B04200D89D
:10F55000022631465046FFF773FE0546012D01D0C5
:10F56000681C08B92846DCE73DB12569022D03D3A4
:10F57000E069A84200D92F46002606BB3E4600BFE0
:10F58000761CE069B04204D80226BE4201D90020B0
:10F59000C7E731465046FFF753FE054605B90DE073
:10F5A000012D01D0681C08B92846BAE7BE42E7D150
:10F5B0000020B6E7525261417272416100BF4FF0C4
:10F5C000FF3231462046FFF7ABFE8146B9F1000F0E
:10F5D00008D1B8F1000F05D0324641462046FFF76A
:10F5E0009FFE8146B9F1000F0DD12661E069801EB2
:10F5F0006169814202D86069401E6061207940F0F3
:10F600000100207107E0B9F1010F02D14FF0FF3086
:10F6100000E001200646304683E7F0B503460D467C
:10F620001E68986A021D680A7789B0FBF7F400BF6C
:10F6300002CA09B90020F0BD8C4200D202E0641A6F
:10F64000121DF5E700BF10682044F4E72DE9F047EC
:10F65000044689462046FFF764FD10B10120BDE84D
:10F66000F08749462046FFF7DEFD074667634FF403
:10F670000072002104F13800FFF7DBFC60894FF4D1
:10F680000041B1EB402F01D8084601E060894002FB
:10F6900006464FF0000800E07608B6F5007F05D971
:10F6A000304602F041FFB0F10008F5D0B6F5007F1A
:10F6B00017D9324600214046FFF7BBFC760A0025E9
:10F6C00000E035446089A84207D97A19607833464A
:10F6D0004146FFF715FC0028F3D0404602F02AFF10
:10F6E00010E004F138080126002500E03544608967
:10F6F000A84207D97A19607833464146FFF700FCE3
:10F700000028F3D06089A84201D00120A7E700209B
:10F71000A5E72DE9F04104460D462668B5F5001F22
:10F7200002D205F01F0010B10220BDE8F081256172
:10F73000A7681FB93078032800DBF76A47B930891A
:10F74000B0EB551F01D80220EFE7F06AA0611CE082
:10F7500070894FEA402811E039462046FFF770FDD6
:10F760000746781C08B90120DFE7022F02D3F069B1
:10F77000B84201D80220D8E7A5EB08054545EBD2F1
:10F7800039463046FFF74FFDA0616761A06908B9AF
:10F790000220CAE7A06900EB5520A061C5F308016B
:10F7A00006F138000844E0610020BEE72DE9F04191
:10F7B000044688462768206900F12006B6F5001F38
:10F7C00001D30020A061A06910B90420BDE8F08138
:10F7D000C6F30800002845D1A069401CA0616069FB
:10F7E00038B93889B0EB561F3CD80020A0610420FE
:10F7F000ECE77889401E00EA562098BB20466169F4
:10F80000FFF71EFD0546012D01D80220DEE7681C2A
:10F8100008B90120DAE7F869A8421DD8B8F1000F4D
:10F8200003D10020A0610420D0E720466169FFF7E2
:10F8300060FE05460DB90720C8E7012D01D1022061
:10F84000C4E7681C08B90120C0E729463846FFF71D
:10F85000FDFE08B10120B9E7656129463846FFF78A
:10F86000E2FCA0612661C6F3080107F138000844F4
:10F87000E0610020AAE72DE9F04104460E46D4F8E5
:10F88000008000212046FFF744FF0546EDB9002720
:10F8900000BF4046A169FFF769FC054605B113E0CA
:10F8A000E0690078E52802D0E069007820B9781C8A
:10F8B0000746B04201D107E0002701212046FFF7AB
:10F8C00075FF0546002DE4D000BF042D00D10725AB
:10F8D0002846BDE8F08170B505460C4604F11A00D3
:10F8E000FFF776FB06462878032805D104F11400BB
:10F8F000FFF76EFB46EA0046304670BD70B506461F
:10F900000C461546A9B204F11A00FFF773FB3078D4
:10F91000032804D1290C04F11400FFF76BFB70BD20
:10F920002DE9F04780460C4604F11A00FFF750FB22
:10F9300010B10020BDE8F087207800F03F00401EA5
:10F9400000EB800101EBC0054FF00109002621E02A
:10F95000F849895D0819FFF73BFB0746B9F1000F2D
:10F9600011D0FF2D0BD8384602F01AFE82462946E8
:10F970006D1C38F8110002F013FE824501D0002002
:10F98000D8E7B94605E04FF6FF70874201D0002066
:10F99000D0E7761C0D2EDBD3207800F0400038B184
:10F9A000B9F1000F04D038F8150008B10020C1E704
:10F9B0000120BFE72DE9F04780460C4604F11A000C
:10F9C000FFF706FB10B10020BDE8F087207820F09B
:10F9D0004000401E00EB800101EBC0054FF0010923
:10F9E000002619E0D349895D0819FFF7F1FA0746A7
:10F9F000B9F1000F09D0FF2D01D90020E4E7B94685
:10FA000028466D1C28F8107005E04FF6FF708742FD
:10FA100001D00020D8E7761C0D2EE3D3207800F02B
:10FA2000400048B1B9F1000F06D0FF2D01D90020E8
:10FA3000CAE7002028F815000120C5E72DE9F047A6
:10FA400007460C461546984684F80D800F20E07254
:10FA500000202073002104F11A00FFF7CBFA681E82
:10FA600000EB800101EBC00900200646824600BF82
:10FA70004FF6FF70864204D0484609F1010937F875
:10FA80001060AC4911F80A1008193146FFF7B2FAB4
:10FA90000EB94FF6FF760AF1010082460D28E7D332
:10FAA0004FF6FF70864202D037F8190008B945F0CA
:10FAB00040052570BDE8F0872DE9FF4F83B08046F3
:10FAC00091461E460B2240460499FFF7A5FA052EE3
:10FAD00018D9374611E039F802BB00250BE058462B
:10FAE00067F35F0007464FEA6B0B07F4803008B1FD
:10FAF000914847406D1C102DF1D3B9F80000002843
:10FB0000E9D13E46072500BF06F00F0000F1300A9C
:10FB1000BAF1390F03DD0AF1070000F0FF0A2846A9
:10FB20006D1E01A901F800A03609002EECD17E203F
:10FB3000485500240AE018F80400FFF79FFA20B1A6
:10FB4000681EA04200D107E0641C641CAC4203D2D2
:10FB500018F804002028EED100BF00BF082D04D201
:10FB600028466D1C01A9085C00E020202146641C89
:10FB700008F80100082CF1D307B0BDE8F08F30B5CC
:10FB8000014600200B2200BF431003EBC01411F804
:10FB9000015B6319D8B2531E1A1EF5D130BD2DE991
:10FBA000F05F044689460426D4F800A04FF0FF0811
:10FBB000C34653E05046A169FFF7D8FA064606B19E
:10FBC0004FE0E06905780DB904264AE0E069C07AA3
:10FBD00000F03F07A771E52D0AD02E2D08D027F0A1
:10FBE0002000082801D1012000E00020484502D073
:10FBF0004FF0FF082BE00F2F1DD105F0400038B16A
:10FC0000E06990F80DB005F0BF05A8462069E062F4
:10FC100045450CD1E069407B584508D1E169DAF8E7
:10FC20000C00FFF7C7FE10B1A8F1010000E0FF20B3
:10FC300000F0FF080BE0B8F1000F04D1E069FFF716
:10FC40009EFF584502D04FF0FF30E06209E00021EE
:10FC50002046FFF7ABFD064606B102E0A06900288A
:10FC6000A8D100BF0EB10020A0613046BDE8F09FD2
:10FC70002DE9F0470446D4F800A000212046FFF704
:10FC800048FD064616B13046BDE8F0874FF0FF0844
:10FC9000C1464FF0FF30E06200BF5046A169FFF758
:10FCA00065FA064606B162E0E06905780DB90426FA
:10FCB0005DE0E069C07A00F03F07A771E52D04D050
:10FCC00007F0080038B10F2F05D04FF0FF084FF0B4
:10FCD000FF30E06244E00F2F22D12B20005D00F0C6
:10FCE000400030BB05F0400038B1E06990F80D905D
:10FCF00005F0BF05A8462069E06245450CD1E069E2
:10FD0000407B484508D1E169DAF80C00FFF708FEAE
:10FD100010B1A8F1010000E0FF2000F0FF081FE093
:10FD2000B8F1000F0AD1E069FFF729FF484505D176
:10FD30001DE015E0ACBD0200211001002B20005D8C
:10FD400000F0010038B90B2204F12001E069FFF74F
:10FD500079F900B90BE04FF0FF084FF0FF30E06297
:10FD600000212046FFF722FD0646002E95D000BF59
:10FD7000304689E72DE9FE4F044626682B20005DBA
:10FD800000F0A00010B10620BDE8FE8F4FF0000982
:10FD900001E009F10109F06830F819000028F8D1F4
:10FDA0000C2204F120016846FFF736F99DF80B009C
:10FDB00000F0010028B340212B2001554FF001082D
:10FDC0000EE04346694604F12000F268FFF774FE36
:10FDD0002046FFF74DFF054605B104E008F1010894
:10FDE000B8F1640FEDD300BFB8F1640F01D1072063
:10FDF000CAE7042D01D02846C6E79DF80B102B203A
:10FE000001559DF80B0000F0020030B109F10C0023
:10FE10000D21B0FBF1F0401C00E0012007463946FF
:10FE20002046FFF728FD05464DBB781E071E26D04D
:10FE30002069A0EB47112046FFF76BFC0546F5B99A
:10FE400004F12000FFF79BFE824600BF3046A16907
:10FE5000FFF78CF9054605B110E0FAB2E1695346A7
:10FE6000F068FFF7EBFD0120F07000212046FFF75E
:10FE70009DFC054615B9781E071EE7D100BFC5B920
:10FE80003046A169FFF772F9054695B92022002195
:10FE9000E069FFF7CEF80B2204F12001E069FFF7DB
:10FEA000BBF82B20005D00F01800E1690873012009
:10FEB000F070284668E72DE9F04104462668276976
:10FEC000E06A401C08B9002003E02046E16AFFF721
:10FED00020FC0546E5B900BF3046A169FFF746F9A9
:10FEE000054605B110E000BFE520E169087001207A
:10FEF000F0702069B84200D306E000212046FFF7E9
:10FF000055FC0546002DE7D000BF042D00D1022589
:10FF10002846BDE8F0812DE9F05F07460C46D7F88A
:10FF200000B00020A075B86908B9BDE8F09FF86A74
:10FF3000401CA8B30025A946A84622E0404608F187
:10FF40000108DBF80C2032F81060B9F1000F07D17E
:10FF5000B6F5584F04DBB6F5604F01DAB14610E054
:10FF6000C5F1FF0204F11603591946EA0940FFF7EB
:10FF7000B7F806460EB9002509E035444FF00009F0
:10FF800000BFDBF80C0030F818000028D6D100BF05
:10FF9000B9F1000F00D00025002104F116004155F1
:10FFA0000020054680461BE0404608F10108FA693A
:10FFB000165C202E00D113E0052E00D1E526B8F105
:10FFC000090F07D10C2D05D22E2228466D1C04F1F5
:10FFD00009010A5428466D1C04F109010E5400BFA2
:10FFE000B8F10B0FE0D3002104F109004155A07DC9
:10FFF000B0BB35B93F2228466D1C04F116010A54E6
:020000040001F9
:1000000025E00020054680464FF0080A19E004F17B
:10001000090010F808602E2E01D14FF0100A412E71
:1000200009DB5A2E07DCF869007B00EA0A0010B1F0
:1000300006F1200086B204F11600465508F10108C9
:100040006D1C04F1090010F808000028DFD1002120
:1000500004F116004155F869007B08B90020607270
:10006000F869C07A2072F96901F11C00FEF7B6FF49
:100070002060F96901F11600FEF7AAFFE080F96936
:1000800001F11800FEF7A4FFA08000BF4DE72DE9A5
:10009000F34F83B08146049800680090D9F80000BF
:1000A000C768002500BF6846FEF7F4FF029002987B
:1000B000401C18B9062005B0BDE8F08F0298B0F5D5
:1000C000803F05D30298020C28466D1C27F81020AB
:1000D000029884B2202C03DB2F2C01D05C2C00D1A1
:1000E00011E0802C06DA2146FEA0FEF7BDFF08B124
:1000F0000620E0E7FF2D01D30620DCE728466D1C33
:1001000027F81040CFE700BF202C01DA04260CE0CE
:10011000002602E00098401C0090009800782F28EC
:10012000F8D0009800785C28F4D000990498016019
:10013000012D04D1681E37F810002E280BD0022D97
:1001400024D1681E37F810002E281FD1A81E37F8BA
:1001500010002E281AD1002027F8150080460AE04A
:10016000A84501D22E2100E0202109F1200000F84D
:10017000081008F10108B8F10B0FF1D346F0200187
:1001800009F1200000F80810002094E708E0681E3C
:1001900037F81040202C02D02E2C00D002E06D1E2B
:1001A000002DF4D100BF002027F815000DB906205E
:1001B00081E74FF0000A01E00AF1010A37F81A005E
:1001C0002028F9D0BAF1000F03D137F81A002E28F1
:1001D00001D146F0030600E06D1E25B1681E37F818
:1001E00010002E28F8D10B22202109F12000FEF763
:1001F00020FF4FF00008C3460820019000BF504682
:100200000AF1010A37F8104004B968E0202C03D045
:100210002E2C04D1AA4502D046F00306EFE7019840
:10022000804501D2AA4516D101980B2802D146F08B
:10023000030654E0AA4501D046F00306AA4500D9BA
:100240004DE0AA464FF008080B2001904FEA8B6062
:100250004FEA106BD3E7802C0EDB46F0020640F22B
:10026000B511204602F06CF9044604F0800018B184
:1002700004F07F009E490C5CFF2C10DD0198401EAD
:10028000404504D846F00306DDF80480B7E72212A3
:10029000404608F1010809F120010A5418E024B190
:1002A000214694A0FEF7E0FE18B15F2446F0030655
:1002B0000EE0412C03DB5A2C01DC4BF0020B612CCD
:1002C00006DB7A2C04DC4BF0010BA4F1200084B295
:1002D000404608F1010809F120010C548FE700BFE6
:1002E00099F82000E52802D1052089F8200001981E
:1002F000082803D14FEA8B604FEA106B0BF00C001B
:100300000C2803D00BF00300032801D146F00206AD
:1003100006F0020048B90BF0010008B146F01006E3
:100320000BF0040008B146F008062B2000F8096025
:100330000020C0E62DE9F3410446276801980078C3
:100340002F2806D0019800785C2802D0B869A060F8
:100350000DE002E00198401C0190019800782F28E0
:10036000F8D0019800785C28F4D00020A0600198B3
:100370000078202808D280212B200155002120461A
:10038000FFF7C7F9054637E000BF01A92046FFF790
:100390007EFE054605B12EE02046FFF769FC0546C6
:1003A0002B20065D95B1042D0FD106F0200040B141
:1003B00006F0040000B9E8E780212B200155002554
:1003C00003E006F0040000B9052514E006F004007F
:1003D00000B110E0A07900F0100008B905250AE08E
:1003E000208AC0F3080207F1380011183846FFF7D9
:1003F00072FAA060C9E700BF2846BDE8FC8170B56D
:1004000004464FF0FF3026683146324601B970BDD0
:1004100000BF12F8013B202B01D33A2BF9D13A2B24
:1004200011D101250E78302E08DB0E78392E05DC2F
:100430008E1C964202D10E78A6F13005012D01DA0C
:1004400028462260E3E72D4E307800BFDFE72DE934
:10045000F041044688460020E070401E606341463B
:100460002046FEF783FE10B10420BDE8F08104F2BF
:100470003620FEF7ADFD074694F83850EB2D03D03B
:10048000E92D01D0E82D4AD14AF65520874208D1FE
:1004900008221BA104F18A00FEF7D4FD08B9002050
:1004A000E3E704F14300FEF793FD0646701E30407B
:1004B00060BBB6F5007F32DBB6F5007F2FDC452050
:1004C000055D1DB3681E284000BB4820005D012863
:1004D00003D04820005D022821D104F14900FEF735
:1004E00077FD14E0222A3A3C3E3F7C7F000000006A
:1004F000B9BD02002B2C3B3D5B5D0000920100204A
:1005000046415433322020200000000007E030B183
:1005100004F14E00FEF75CFD08B10020A5E74AF6A5
:100520005520874201D102209FE703209DE72DE956
:10053000FF4107460D4600213846FFF788FF064673
:10054000022E06D0032E00D21DB9304604B0BDE8FD
:10055000F08100BF00240AE007F5FB7101EB0411F4
:1005600001F10800FEF73AFD4DF82400641C042C4C
:10057000F2D30DB1681E00E00020044600BF5DF814
:10058000240028B15DF824103846FFF760FF00E032
:10059000032006462DB9022E03D3601C044604280E
:1005A000EDD33046D2E72DE9F74F84B0002105980E
:1005B00001600498FFF723FF03900398002803DAF3
:1005C0000B2007B0BDE8F08FFE49039851F820409A
:1005D0000CB90C20F5E705980460069800F0FE00C1
:1005E0000690207878B16078FEF756FC074607F051
:1005F000010040B9069820B107F0040008B10A20B4
:10060000DFE70020DDE7002020700398607060784D
:10061000FEF748FC074607F0010008B10320D0E7C9
:10062000069820B107F0040008B10A20C9E70021AC
:100630002046FFF77CFF0546042D01D10120C0E7CD
:10064000022D01D30D20BCE7D4F8349004F143000F
:10065000FEF7BEFCB0F5007F01D00D20B1E704F13C
:100660004E00FEF7B5FC064626B904F15C00FEF725
:10067000B5FC064626624820005DA070A0780128DF
:1006800004D0A078022801D00D209AE7A078464334
:100690004520005D6081608918B16089411E084075
:1006A00008B10D208DE704F14900FEF791FC20818F
:1006B000207A00F00F0008B10D2082E704F14B0012
:1006C000FEF786FC8246BAF1000F04D104F158000F
:1006D000FEF784FC824604F14600FEF779FC83466F
:1006E000BBF1000F01D10D206BE70BEB0600218958
:1006F00000EB111002900298824501D20D2060E7B4
:100700000298AAEB00006189B0FBF1F8B8F1000F84
:1007100001D10D2055E70025AB48804500D80325C1
:100720004FF6F570804500D8022540F6F5708045FB
:1007300000D801250DB90D2043E708F10200E06162
:10074000C4F8249009EB0B00A0620298484420638F
:10075000032D13D104F16200FEF73AFC08B10D201D
:100760002FE7208908B10D202BE704F16400FEF784
:1007700035FCE062E0698000019014E0208908B94E
:100780000D201EE7A06A3044E062022D02D1E0692C
:10079000400007E0207F00F00100E16901EB41012A
:1007A00000EB51000190216A019800F2FF10B1EBBB
:1007B000502F01D20D2004E74FF0FF30606120611F
:1007C00080202071032D2DD104F16800FEF700FC7C
:1007D000012827D109F101012046FEF7C7FC08BB1B
:1007E0000020207104F23620FEF7F2FB4AF6552174
:1007F000884217D104F13800FEF7F0FB73498842B4
:1008000010D104F50770FEF7E9FB7149884209D160
:1008100004F50870FEF7E2FB606104F50970FEF76D
:10082000DDFB206125706B480088401C80B269495F
:100830000880E0800020A06100BFC2E670B50446D9
:100840000D4609268CB1206878B12068007860B127
:10085000A0882168C988884207D121684878FEF7B6
:100860001BFB00F0010000B900260EB9206800E073
:1008700000202860304670BDF7B582B01646039858
:10088000019001A8FFF7BBFD0546002D02DA0B2001
:1008900005B0F0BD4B4850F825400CB10020207049
:1008A000029810B10020029908704649029841F858
:1008B00025000EB90020EBE7002202A903A8FFF7EC
:1008C00072FE07463846E3E72DE9F74F90B004463D
:1008D00016461CB9092013B0BDE8F08F06F03F069C
:1008E000324603A911A8FFF75EFE0546002D68D128
:1008F000039804904FF4007001F016FE8346BBF19C
:10090000000F01D11120E6E70398C0F80CB004A84D
:100910001199FFF70FFD05462DB99DF83B0000F03A
:10092000800000B1062506F01C00002862D045B109
:10093000042D03D104A8FFF71DFA054646F008066A
:100940000AE09DF8160000F0110008B1072503E049
:1009500006F0040000B10825002D5CD106F0080067
:10096000002858D0FEF712FB01900B9901F10E0000
:100970000199FEF745FB0B9901F116000199FEF76D
:100980003FFB0B990398FEF7A6FF814620200B99A9
:10099000C87200220B990398FEF7B0FF0B9901F182
:1009A0001C000021FEF72CFB01200399C870B9F14F
:1009B000000F30D00398D0F834A00022494604A894
:1009C0000AE093E08C010020F5FFFF0F52526141D5
:1009D0007272416190010020FEF73EFD054645B967
:1009E00051460398FEF7C2FB0546A9F101000399A1
:1009F000086110E07DB99DF8160000F0100008B104
:100A0000042508E006F0020028B19DF8160000F069
:100A1000010000B107254DB906F0080008B146F005
:100A200040060398406B20620B986062002D5AD1FB
:100A30000B990398FEF74FFFA0600B9901F11C0082
:100A4000FEF7CCFAE0600020A062039820600398D3
:100A5000C088A080267400206074E06160614FF45B
:100A60000072002104F12C00FEF7E3FA06F02000EA
:100A700058B3E06848B3E068606103984089400279
:100A80000290A768D4F80C800DE039462046FEF7A6
:100A9000D7FB0746012F00D80225781C00B9012595
:100AA0000298A8EB000815B902988045EDD8A76117
:100AB0005DB9C8F3080040B139460398FEF7B3FBAF
:100AC0008246BAF1000F01D102250CE00AEB582052
:100AD000E061E26903994878012304F12C01FEF7F3
:100AE000F4F900B10125584601F024FD0DB10020B4
:100AF00020602846EFE62DE9FF4F85B004461546F5
:100B00009A46DDF818B00020CAF8000003A9204674
:100B1000FFF794FE0490049810B9607C049018B11B
:100B2000049809B0BDE8F08F207C00F0010008B9FE
:100B30000720F6E76169E068401A01900198854254
:100B400000D9019DA8E0A08AC0F30800002874D154
:100B500003984089401E616900EA5129B9F1000FEC
:100B60001FD1606910B9A06802900CE0A06A28B19A
:100B700020466169FEF751FD029004E02046A1691C
:100B8000FEF75EFB02900298022802D202206074F7
:100B9000C7E70298401C10B901206074C1E70298B1
:100BA000A061A1690398FEF73EFB064616B9022034
:100BB0006074B6E74E444FEA5528B8F1000F29D0CB
:100BC00009EB080003994989884203D903984089B1
:100BD000A0EB090803994878434632465946FEF788
:100BE00074F910B1012060749BE7207C00F0800054
:100BF00068B1E069801B404509D2E169891B0BEBB4
:100C000041204FF4007204F12C01FEF705FA4FEA7F
:100C1000482737E0E069B04220D0207C00F0800017
:100C200080B1E26903994878012304F12C01FEF7B1
:100C300067F918B10120607473E710E0207C00F0C0
:100C40007F002074039948780123324604F12C0177
:100C5000FEF73BF910B10120607462E7E661A08AFB
:100C6000C0F30800C0F50077AF4200D92F46A08A34
:100C7000C0F3080204F12C0011183A465846FEF75A
:100C8000CBF900BFED1BDAF800003844CAF80000C9
:100C9000BB44606938446061002D7FF454AF00208C
:100CA0003FE72DE9FF4F83B0044615469B46049865
:100CB00000900020CBF8000001A92046FFF7BEFD00
:100CC0000290029810B9607C029018B1029807B0A7
:100CD000BDE8F08F207C00F0020008B90720F6E79D
:100CE00000BF606928446169884202D26069C0F12E
:100CF000FF35C3E0A08AC0F3080000287DD1019829
:100D00004089401E616900EA512ABAF1000F26D1DC
:100D1000606938B9A76897B900212046FEF7E9FB5A
:100D200007460CE0A06A28B120466169FEF775FC11
:100D3000074604E02046A169FEF7DBFB074607B93A
:100D40009FE0012F02D102206074C0E7781C10B927
:100D500001206074BBE7A761A06800B9A760207C90
:100D600000F0800078B1E26901994878012304F12C
:100D70002C01FEF7C5F810B101206074A7E7207CB4
:100D800000F07F002074A1690198FEF74CFA064636
:100D900016B9022060749AE756444FEA5529B9F112
:100DA000000F2BD00AEB090001994989884203D929
:100DB00001984089A0EB0A09019948784B463246D0
:100DC0000099FEF79DF810B1012060747FE7E0699B
:100DD000801B48450ED2E069801B009A02EB40213F
:100DE0004FF4007204F12C00FEF716F9207C00F09D
:100DF0007F0020744FEA49282BE013E0E069B042FD
:100E00000FD0E168606988420BD2019948780123CC
:100E1000324604F12C01FEF758F810B1012060743D
:100E200055E7E661A08AC0F30800C0F50078A84540
:100E300000D9A846A18AC1F3080204F12C01501878
:100E400042460099FEF7E8F8207C40F080002074CC
:100E500000BFA5EB0805DBF800004044CBF800001C
:100E6000009840440090606940446061E1686069B6
:100E7000884201D9606900E0E068E060002D7FF4FD
:100E800039AF00BF207C40F04000207400201EE7F6
:100E9000F8B5044669462046FFF7D0FC0646002E0A
:100EA00044D1207C00F0400000283FD0207C00F09E
:100EB000800070B1E26900994878012304F12C01A7
:100EC000FEF71EF808B10120F8BD207C00F07F007D
:100ED0002074FEF75BF80746216A0098FEF746F992
:100EE00006461EBB656AE87A40F02000E872294693
:100EF000A2682068FEF702FD05F11C00E168FEF71C
:100F00007FF8394605F11600FEF77AF8002105F161
:100F10001200FEF76FF801200099C8700098FEF7E4
:100F20003FF90646207C00F0BF0020743046CBE736
:100F300038B505462846FFF7ABFF04463CB969467D
:100F40002846FFF77BFC04460CB9002028602046A9
:100F500038BD31B56846FFF752FA0446002C01DA75
:100F60000B2038BDFB490C700020FAE731B58EB07C
:100F7000002201A90EA8FFF716FB044674BB0198D6
:100F800002904FF4007001F0CFFA054615B9112018
:100F90000FB030BD0198C56002A80E99FFF7CAF9DD
:100FA0000446ACB99DF8330000F0800018B10199F7
:100FB000049888610CE09DF80E0000F0100030B13C
:100FC00009990198FEF787FC0199886100E00524E2
:100FD000284601F0AFFA042C00D105242046D7E7BB
:100FE0002DE9F04F89B004460D4607A92046FFF7CA
:100FF00025FC0890089808B9607C0890089818B1FA
:10100000089809B0BDE8F08FA06A00287CD0681C61
:10101000002843D1D4F8289059F8040B02900220FC
:101020000190A76867B300BF039700200490019860
:10103000801C019000BF05970498401C049039461D
:101040002046FEF7FDF80746012F02D80220607403
:10105000D7E7781C10B901206074D2E70598401CCE
:101060008742E8D0DDE90101884205D8049849F8B3
:10107000040B039849F8040B0798C069B842D3D809
:101080000198A16A0860DDE90101884203D80020C7
:10109000C9F80000FAE011200890F7E0E068A842E3
:1010A00000D2E5686561002DF4D0691E2046FEF788
:1010B000B4FAA061A1690798FEF7B5F88246BAF1C3
:1010C000000F02D1022060749BE707984089401E00
:1010D000691E00EA51208244A08AC0F3080000285B
:1010E000D8D0E0695045D5D0207C00F0800080B198
:1010F000E26907994878012304F12C01FDF700FF0C
:1011000018B1012060747CE712E0207C00F07F00C1
:101110002074079948780123524604F12C01FDF709
:10112000D4FE10B1012060746BE7C4F81CA0ADE0E0
:10113000E068A84204D2207C00F0020000B9E56813
:10114000606906904FF0000BC4F814B0002D6AD00F
:10115000079840894FEA4028069890B1681EB0FB76
:10116000F8F10698401EB0FBF8F0814209D30698CA
:10117000401EA8F101018843606160692D1AA669CB
:1011800012E0A6687EB900212046FEF7B2F90646B5
:10119000012E02D10220607433E7701C10B90120C7
:1011A00060742EE7A660A661D6B325E0A5EB08051E
:1011B000606940446061207C00F0020040B100BFE3
:1011C00031462046FEF795F9064636B9002515E06A
:1011D00031462046FEF734F80646701C10B901204F
:1011E00060740EE7012E03D90798C069B04202D897
:1011F0000220607405E7A6614545D7D800BF606945
:1012000028446061C5F3080050B131460798FEF7E5
:101210000AF88346BBF1000F03D102206074F0E6A8
:1012200001E00BEB552BE1686069884205D96069E4
:10123000E060207C40F040002074A08AC0F30800E9
:1012400020B3E069584521D0207C00F0800078B1BF
:10125000E26907994878012304F12C01FDF750FE5B
:1012600010B101206074CCE6207C00F07F00207477
:101270000799487801235A4604F12C01FDF725FE11
:1012800010B101206074BCE6C4F81CB00898B8E640
:1012900073B582B0044614B9092004B070BD0022B1
:1012A00001A903A8FFF77FF90546002D30D1019869
:1012B00020604FF4007001F037F906460EB9112096
:1012C000EBE70198C66020460399FFF733F805461F
:1012D000C5B92B20005D00F0800050B9A07900F066
:1012E000100028B1E1690198FEF7F5FAA06000E06E
:1012F00005253DB90198C088A08000212046FEF751
:1013000008FA0546304601F015F9042D00D10525EF
:101310000DB1002020602846BFE738B50446694675
:101320002046FFF78BFA05460DB9002020602846BD
:1013300038BDF8B507460E4669463846FFF77EFACF
:1013400004465CBB46B900213846FEF7E2F9044684
:1013500024E00000920100204FF4007001F0E4F856
:1013600005460DB91120F8BD0098C560002138462A
:10137000FEF715FC0446042C00D100245CB931466C
:101380003846FEF7C8FD00213846FEF70FFA04463E
:10139000042C00D10024284601F0CCF82046E2E7D6
:1013A00073B58CB00E46002269460CA8FFF7FBF817
:1013B0000546FDB94FF4007001F0B6F8044614B9C3
:1013C00011200EB070BD0098C46068460C99FEF7FD
:1013D000B1FF05465DB99DF82B0000F0800008B113
:1013E000062504E01EB131466846FEF794FD20460E
:1013F00001F0A0F82846E4E72DE9F74F86B08846CB
:101400009246002205A906A8FFF7CDF88146B9F15A
:10141000000F68D10598CAF8000005984169C069B5
:10142000801E814204D805984069C8F800005AE03F
:1014300000250598007801281BD102260598019007
:1014400000BF314601A8FDF7FBFE0746781C10B926
:101450004FF001090CE0012F02D14FF0020907E023
:1014600007B96D1C701C06460599C9698842E8D306
:101470002FE00598C6690598D0F828B0002400BF71
:1014800054B959460BF1010B0598FDF76FFE8146E3
:10149000B9F1000F00D01BE005980078022808D1B0
:1014A000059938310819FDF793FD00B96D1CA41C8E
:1014B00009E0059938310819FDF790FD20F07040DA
:1014C00000B96D1C241DC4F30804701E061ED7D17C
:1014D00000BFC8F80050059845610598007940F0B4
:1014E000010005990871484609B0BDE8F08FF8B5CC
:1014F000044669462046FFF7A1F9054615B9607C08
:10150000051E01D02846F8BD207C00F0020008B975
:101510000720F8E7E168606988423FD2606940B916
:1015200000222046A168FDF797FF05460020A06035
:1015300016E02046A169FDF783FE06460025701CD3
:1015400000B90125012E00D102254DB90098C069CE
:10155000B04205D931462046A269FDF77DFF054618
:101560006069E060207C40F04000207495B9207CE8
:1015700000F0800070B1E26900994878012304F11D
:101580002C01FDF7BDFC08B1012503E0207C00F033
:101590007F00207415B165742846B4E72846B2E789
:1015A00071B599B000250222694619A8FEF7FBFF24
:1015B0000446002C60D100980D904FF4007000F0AC
:1015C000B3FF064616B911201AB070BD0098C66068
:1015D0000DA81999FEF7AEFE04462CB99DF85F00E0
:1015E00000F0200000B10624002C42D19DF85F00DD
:1015F00000F0800008B1062405E09DF83A0000F0F4
:10160000010000B1072414BB14990098FEF763F998
:1016100005469DF83A0000F01000C0B100988069BE
:10162000A84201D1072412E00098019003950021FF
:1016300001A8FEF76EF804464CB9002101A8FEF798
:10164000AEFA044604B90724042C00D1002484B95E
:101650000DA8FEF730FC044634B92DB1002229460E
:101660000DA8FDF7F9FE04461CB90098FDF798FD9A
:101670000446304600F05EFF2046A5E72DE9F14123
:1016800091B00222694611A8FEF78DFF0446002C96
:101690007ED1009805904FF4007000F045FF06469B
:1016A0001EB9112012B0BDE8F0810098C66005A8EF
:1016B0001199FEF73FFE044604B90824042C05D115
:1016C0009DF83F0000F0200000B10624042C6AD1F0
:1016D00000980190002101A8FDF70BFF05460024AA
:1016E00005B90724012D00D10224681C00B901248A
:1016F000FDF74CFC8046BCBB29460098FDF7A6FFD1
:1017000004468CBB0B22202100983830FDF791FC59
:101710002E20009981F838001021009880F843109D
:10172000414600984E30FDF76BFC2A46009938314F
:101730000098FEF7E3F820220099383100985830DD
:10174000FDF76AFC2E21009880F85910079F3A4651
:10175000009958310098FEF7D1F801200099C8701F
:1017600005A8FEF707FB0446C4B90C9901F1160061
:101770004146FDF745FC2A460C990098FEF7BEF855
:1017800010200C99C87201200099C8702CB900E093
:101790000CE00098FDF704FD044604E00022294611
:1017A00001A8FDF759FE304600F0C4FE204679E757
:1017B0002DE9F341A2B023A8FEF721FE022209A9D8
:1017C00022A8FEF7F0FE0446002C7DD10998169061
:1017D0004FF4007000F0A8FE07461FB9112024B096
:1017E000BDE8F0810998C76016A82299FEF7A2FD0E
:1017F00004462CB99DF8830000F0A00000B1062437
:10180000002C6ED1202201A81D99FDF705FC302285
:1018100016A90AA8FDF700FC0AA82399FEF78AFD7D
:1018200004465CB918990C98884205D11A990E980B
:10183000884201D1042000E008200446042C46D14F
:101840000AA8FEF797FA0446002C40D1119D1322F6
:101850000DF1110105F10D00FDF7DEFB9DF80F0004
:10186000E872E87A00F0100018B9E87A40F0200039
:10187000E87201200999C870E87A00F0100030B3CE
:101880000C991898884222D029460998FEF723F827
:10189000804641460998FDF7C6FC06460EB902246B
:1018A00015E031460998FDF761FC0446099800F1FE
:1018B000580564B968782E2809D129460C9A0998E8
:1018C000FEF71CF8012000E00EE00999C87044B949
:1018D00016A8FEF7F0FA04461CB90998FDF760FC5B
:1018E0000446384600F026FE204678E72DE9FF4FF3
:1018F00085B09A4603AA01210598FDF717FB18B198
:10190000012009B0BDE8F08FDDF80C904FF03F08E2
:10191000082701E07806070E37B1B9FBF7F0B0FBF6
:10192000F8F0B0F5806FF5D807B9FF274FF40072D3
:1019300000215046FDF77DFB0AF5DF764FF0000BE6
:10194000444669E0069850F82B50642D07D801D121
:10195000484603E06420B9FBF0F06843054660198F
:10196000484501D8601901D3A9EB040505B959E030
:10197000214606F10800FDF743FB294606F10C005D
:10198000FDF73EFB07983071B4FBF8F0B0FBF7F0C1
:101990000490B4FBF8F0B0FBF7F107FB1100C0B204
:1019A0000290B4FBF8F008FB1040401CC0B201905C
:1019B00002987070C021049801EA900001990843D0
:1019C000B0700498F0706019401EB0FBF8F0B0FBE6
:1019D000F7F004906019401EB0FBF8F0B0FBF7F18F
:1019E00007FB1100C0B202906019401EB0FBF8F175
:1019F00008FB1100401CC0B2019002987071C02118
:101A0000049801EA900001990843B0710498F071BC
:101A100010360BF1010B2C44BBF1040F02D20CB1B8
:101A20004C458FD300BF4AF655210AF5FF70FDF7EC
:101A3000E1FA0123002251460598FDF761FA08B149
:101A400001205EE700205CE72DE9FF4F99B00F46CB
:101A5000154619A8FEF7D3FC03900398002803DA73
:101A60000B201DB0BDE8F08FFC49039851F8200011
:101A700028B10021F94A039852F820000170039818
:101A8000C0B216900020159007B9F54F1698FDF7D3
:101A900009FA0290029800F0010008B10320E0E783
:101AA000029800F0040008B10A20DAE77868139081
:101AB000139838B913AA03211698FDF737FA08B11D
:101AC00001201390139840B11398B0F5004F04D83B
:101AD0001398401E1399084008B1012013904FF449
:101AE0000079387800F00F0018907878012804DB2E
:101AF0007878022801DC787800E001200690B96847
:101B000089B1B968B1F5004F0DD848464FEAE9717F
:101B100009EBD1614911BA68B2FBF1F301FB132162
:101B200009B9B96801E04FF400710591F868B0F1A6
:101B3000807F05D8F868411E084008B9F86800E0C1
:101B4000002007900798B0FBF9F007901C98B0FBB5
:101B5000F9F01490149808B9112082E72C462CB99A
:101B6000149901FB09F000F0DFFC04460CB91120C8
:101B700077E700201190109000BF11AA012116985C
:101B8000FDF7D4F928B115B9204600F0D3FC0120A7
:101B900067E7189800F0080040B911983F2805D968
:101BA0003F201090DDE91001081A1190119880284B
:101BB00005D215B9204600F0BDFC0E2051E700BF4C
:101BC00000BF0798802801D980200790189800F05E
:101BD000020030B1189800F0010010B94FF003086E
:101BE0000CE0189800F0010028B915B9204600F063
:101BF000A1FC132035E74FF0020800BF00BF00BF73
